:020000040000FA
:1000000000040020810A000015070000610A0000BA
:100010001F07000029070000330700000000000050
:10002000000000000000000000000000A50A000021
:100030003D070000000000004707000051070000D6
:100040005B070000650700006F07000079070000EC
:10005000830700008D07000097070000A10700003C
:10006000AB070000B5070000BF070000C90700008C
:10007000D3070000DD070000E7070000F1070000DC
:10008000FB070000050800000F0800001908000029
:10009000230800002D080000370800004108000078
:1000A0004B080000550800005F08000069080000C8
:1000B000730800007D080000870800009108000018
:1000C0009B080000A5080000AF080000B908000068
:1000D000C3080000CD080000D7080000E1080000B8
:1000E000EB080000F5080000FF0800000909000007
:1000F000130900001D090000270900003109000054
:100100003B0900001FB500F003F88DE80F001FBD8C
:1001100000F0ACBC40F6FC7108684FF01022401CA7
:1001200008D00868401C09D00868401C04D0086842
:1001300000F037BA9069F5E79069F9E7704770B554
:100140000B46010B184400F6FF70040B4FF0805073
:100150000022090303692403406943431D1B104621
:1001600000F048FA29462046BDE8704000F042BA47
:10017000F0B54FF6FF734FF4B4751A466E1E11E0DA
:10018000A94201D3344600E00C46091B30F8027B3B
:10019000641E3B441A44F9D19CB204EB134394B25D
:1001A00004EB12420029EBD198B200EB134002EBB2
:1001B000124140EA0140F0BDF34992B00446D1E952
:1001C0000001CDE91001FF224021684600F0F4FB58
:1001D00094E80F008DE80F00684610A902E004C8FB
:1001E00041F8042D8842FAD110216846FFF7C0FF7C
:1001F0001090AA208DF8440000F099F9FFF78AFFCB
:1002000040F6FC7420684FF01025401C0FD0206889
:1002100010226946803000F078F92068401C08D030
:100220002068082210A900F070F900F061F9A869AF
:10023000EEE7A869F5E74FF080500369406940F6A2
:10024000FC71434308684FF01022401C06D0086838
:1002500000F58050834203D2092070479069F7E788
:100260000868401C04D00868401C03D00020704778
:100270009069F9E70420704770B504460068C34DE3
:10028000072876D2DFE800F033041929631E250021
:10029000D4E9026564682946304600F062F92A46CE
:1002A0002146304600F031F9AA002146304600F0E0
:1002B00057FB002800D0032070BD00F009FC4FF46C
:1002C000805007E0201D00F040F90028F4D100F034
:1002D000FFFB60682860002070BD241D94E80700C3
:1002E000920000F03DFB0028F6D00E2070BDFFF715
:1002F000A2FF0028FAD1D4E901034FF0805100EBAE
:10030000830208694D69684382420ED840F6F8704E
:1003100005684FF010226D1C09D0056805EB8305B8
:100320000B6949694B439D4203D9092070BD55694A
:10033000F4E70168491C03D00068401C02D003E0C8
:100340005069FAE70F2070BD2046FFF735FFFFF731
:1003500072FF0028F7D1201D00F0F7F80028F2D135
:1003600060680028F0D100F0E2F8FFF7D3FE00F05B
:10037000BFF8072070BD10B50C46182802D0012028
:10038000086010BD2068FFF777FF206010BD41684E
:10039000054609B1012700E0002740F6F8742068FF
:1003A0004FF01026401C2BD02068AA68920000F065
:1003B000D7FA38B3A86881002068401C27D020688D
:1003C000FFF7BDFED7B12068401C22D026684FF051
:1003D0008050AC686D68016942695143A9420DD9EA
:1003E000016940694143A14208D92146304600F0E5
:1003F000B8F822462946304600F087F800F078F831
:100400007069D2E700F093F8FFF784FEF6E77069B1
:10041000D6E77669DBE740F6FC7420684FF01026DB
:10042000401C23D02068401C0CD02068401C1FD0EA
:100430002568206805F18005401C1BD027683879A5
:10044000AA2819D040F6F8700168491C42D001680A
:10045000491C45D00168491C3ED001680968491C07
:100460003ED00168491C39D000683EE0B069DAE747
:10047000B569DEE7B769E2E710212846FFF778FEA5
:100480003968814222D12068401C05D0D4F8001080
:1004900001F18002C03107E0B169F9E730B108CA63
:1004A00051F8040D984201D1012000E000208A4259
:1004B000F4D158B1286810B1042803D0FEE72846CB
:1004C000FFF765FF3149686808600EE0FFF722FE1C
:1004D00000F00EF87169BBE77169BFE7706904E06D
:1004E0004FF480500168491C01D000F0CBFAFEE7C0
:1004F000BFF34F8F26480168264A01F4E06111439B
:100500000160BFF34F8F00BFFDE72DE9F0411746B3
:100510000D460646002406E03046296800F054F8EF
:10052000641C2D1D361DBC42F6D3BDE8F08140F69B
:10053000FC700168491C04D0D0F800004FF48051D1
:10054000FDE54FF010208069F8E74FF080510A690F
:10055000496900684A43824201D810207047002050
:10056000704770B50C4605464FF4806608E0284693
:1005700000F017F8B44205D3A4F5806405F5805562
:10058000002CF4D170BD0000F40A0000000000202F
:100590000CED00E00400FA05144801680029FCD0C5
:1005A0007047134A0221116010490B68002BFCD0E0
:1005B0000F4B1B1D186008680028FCD0002010603D
:1005C00008680028FCD07047094B10B501221A605A
:1005D000064A1468002CFCD0016010680028FCD08A
:1005E0000020186010680028FCD010BD00E4014015
:1005F00004E5014070B50C46054600F073F810B9EB
:1006000000F07EF828B121462846BDE8704000F091
:1006100007B821462846BDE8704000F037B8000012
:100620007FB5002200920192029203920A0B000B06
:100630006946012302440AE0440900F01F0651F80C
:10064000245003FA06F6354341F82450401C8242F8
:10065000F2D80D490868009A10430860081D016827
:10066000019A1143016000F03DF800280AD00649C4
:1006700010310868029A10430860091D0868039A3F
:10068000104308607FBD00000006004030B50F4CED
:10069000002200BF04EB0213D3F800582DB9D3F8A1
:1006A000045815B9D3F808581DB1521C082AF1D3C3
:1006B00030BD082AFCD204EB0212C2F80008C3F8CD
:1006C00004180220C3F8080830BD000000E0014013
:1006D0004FF08050D0F83001082801D0002070473A
:1006E000012070474FF08050D0F83011062905D016
:1006F000D0F83001401C01D0002070470120704725
:100700004FF08050D0F830010A2801D00020704707
:100710000120704708208F490968095808471020B0
:100720008C4909680958084714208A4909680958FA
:100730000847182087490968095808473020854923
:100740000968095808473820824909680958084744
:100750003C20804909680958084740207D490968BC
:100760000958084744207B49096809580847482028
:1007700078490968095808474C207649096809589A
:10078000084750207349096809580847542071499F
:1007900009680958084758206E49096809580847E8
:1007A0005C206C4909680958084760206949096854
:1007B00009580847642067490968095808476820AC
:1007C00064490968095808476C2062490968095852
:1007D000084770205F4909680958084774205D4937
:1007E00009680958084778205A490968095808478C
:1007F0007C205849096809580847802055490968EC
:10080000095808478420534909680958084788202F
:1008100050490968095808478C204E490968095809
:10082000084790204B4909680958084794204949CE
:10083000096809580847982046490968095808472F
:100840009C204449096809580847A0204149096883
:1008500009580847A4203F49096809580847A820B3
:100860003C49096809580847AC203A4909680958C1
:100870000847B0203749096809580847B420354966
:10088000096809580847B8203249096809580847D3
:10089000BC203049096809580847C0202D4909681B
:1008A00009580847C4202B49096809580847C82037
:1008B0002849096809580847CC2026490968095879
:1008C0000847D0202349096809580847D4202149FE
:1008D000096809580847D8201E4909680958084777
:1008E000DC201C49096809580847E02019490968B3
:1008F00009580847E4201749096809580847E820BB
:100900001449096809580847EC2012490968095830
:100910000847F0200F49096809580847F4200D4995
:10092000096809580847F8200A490968095808471A
:10093000FC2008490968095808475FF48070054998
:10094000096809580847000003480449024A034B54
:100950007047000000000020000B0000000B0000AA
:1009600040EA010310B59B070FD1042A0DD310C82C
:1009700008C9121F9C42F8D020BA19BA884201D97E
:10098000012010BD4FF0FF3010BD1AB1D30703D0C6
:10099000521C07E0002010BD10F8013B11F8014B7C
:1009A0001B1B07D110F8013B11F8014B1B1B01D198
:1009B000921EF1D1184610BD02F0FF0343EA032254
:1009C00042EA024200F005B87047704770474FF0A6
:1009D00000020429C0F0128010F0030C00F01B800C
:1009E000CCF1040CBCF1020F18BF00F8012BA8BF1A
:1009F00020F8022BA1EB0C0100F00DB85FEAC17CDE
:100A000024BF00F8012B00F8012B48BF00F8012B90
:100A100070474FF0000200B51346944696462039C1
:100A200022BFA0E80C50A0E80C50B1F12001BFF4A7
:100A3000F7AF090728BFA0E80C5048BF0CC05DF80D
:100A400004EB890028BF40F8042B08BF704748BF5B
:100A500020F8022B11F0804F18BF00F8012B7047CF
:100A6000014B1B68DB6818470000002009480A4951
:100A70007047FFF7FBFFFFF745FB00BD20BFFDE719
:100A8000064B1847064A1060016881F308884068E1
:100A900000470000000B0000000B000017040000DE
:100AA000000000201EF0040F0CBFEFF30881EFF3ED
:100AB0000981886902380078182803D100E0000015
:100AC000074A1047074A12682C3212681047000084
:100AD00000B5054B1B68054A9B58984700BD0000B0
:100AE0007703000000000020F00A0000040000006E
:100AF000001000000000000000FFFFFF0090D00386
:10100000B00F0020D1AE0100C1B0000037AE01002A
:10101000C1B00000C1B00000C1B00000000000007D
:101020000000000000000000000000005DAF0100B3
:10103000C1B0000000000000C1B00000C1B000005D
:10104000C5AF0100CBAF0100C1B00000C1B00000CE
:10105000C1B00000C1B00000C1B00000C1B00000CC
:10106000D1AF0100C1B00000C1B00000D7AF010096
:10107000C1B00000DDAF0100E3AF0100E9AF010046
:10108000C1B00000C1B00000C1B00000C1B000009C
:10109000C1B00000C1B00000C1B00000C1B000008C
:1010A000C1B00000EFAF0100C1B00000C1B000004E
:1010B000C1B00000C1B00000C1B00000C1B000006C
:1010C000F5AF0100C1B00000C1B00000C1B0000028
:1010D000C1B00000C1B00000C1B00000C1B000004C
:1010E000C1B00000C1B00000C1B00000C1B000003C
:1010F000C1B00000C1B00000C1B00000C1B000002C
:10110000C1B00000C1B0000000F002F819F0CFFE3D
:101110000AA090E8000C82448344AAF10107DA4552
:1011200001D119F0C4FEAFF2090EBAE80F0013F0B6
:10113000010F18BFFB1A43F00103184730A3010049
:1011400050A301000A4410F8014B14F00F0508BF2A
:1011500010F8015B240908BF10F8014B6D1E05D083
:1011600010F8013B6D1E01F8013BF9D1641E03D05C
:10117000641E01F8015BFBD19142E4D3704700008B
:101180000023002400250026103A28BF78C1FBD890
:10119000520728BF30C148BF0B6070471FB500F031
:1011A00003F88DE80F001FBD19F07EBE70B51B4C13
:1011B00005460A202070A01C00F0D7F85920A08016
:1011C00029462046BDE8704006F012BF06F020BF59
:1011D00070B50C461249097829B1A0F160015E2969
:1011E00008D3012013E0602804D0692802D043F21C
:1011F00001000CE020CC0B4E94E80E0006EB8000C2
:10120000A0F58050241FD0F8806E2846B04720609B
:1012100070BD0120704706207047000008000020C4
:101220001C00002024B001003249884201D2012074
:1012300070470020704770B50446A0F500002E4EA0
:10124000B0F1786F02D23444A4F5000429488442F6
:1012500001D2012500E0002500F043F848B125B98E
:10126000B44204D32548006808E0012070BD002086
:1012700070BD002DF9D1B442F9D321488442F6D291
:10128000F3E710B50446A0F50000B0F1786F03D283
:1012900019480444A4F5000400F023F84FF08041FD
:1012A00030B11648006804E08C4204D2012003E00B
:1012B00013488442F8D2002080F0010010BD10B520
:1012C00020B1FFF7DEFF08B1012010BD002010BDE6
:1012D00010B520B1FFF7AFFF08B1012010BD00200D
:1012E00010BD084808490068884201D101207047B4
:1012F0000020704700C001000000002020000020F6
:10130000080000205C000020BEBAFECA10B50446EA
:101310000021012000F042F800210B2000F03EF8EF
:101320000021082000F03AF80421192000F036F8D6
:1013300004210D2000F032F804210E2000F02EF8D8
:1013400004210F2000F02AF80421C84300F026F8F9
:101350000621162000F022F80621152000F01EF8C4
:101360002046FFF723FF002010BD4FF4817101805C
:101370007047FFF72BBF1148704710487047104A5D
:1013800010B514680E4B0F4A08331A60FFF720FFA0
:101390000B48001D046010BD704770474907090ED7
:1013A000002804DB00F1E02080F80014704700F012
:1013B0000F0000F1E02080F8141D704703F900428F
:1013C000100502400100000130B5FF4D0446062C17
:1013D000A9780ED2DFE804F0030E0E0E0509FFDF38
:1013E00008E0022906D0FFDF04E0032902D0FFDF76
:1013F00000E0FFDFAC7030BDF34810B5407E41081F
:10140000F14800F11A0005D00DF068FBBDE810406E
:1014100006F08EBC0DF049FBF8E730B50446A1F1AB
:1014200020000D460A2847D2DFE800F005070C1916
:10143000202532373C41FFDF3FE0207820283CD197
:10144000FFDF3AE0E0488078052836D0207824286D
:1014500033D0252831D023282FD0FFDF2DE020786E
:1014600022282AD0232828D8FFDF26E02078222827
:1014700023D0FFDF21E0207822281ED024281CD092
:1014800026281AD0272818D0292816D0FFDF14E0E4
:101490002078252811D0FFDF0FE0207825280CD0F8
:1014A000FFDF0AE02078252807D0FFDF05E020785D
:1014B000282802D0FFDF00E0FFDF257030BD1FB518
:1014C0000022ADF800200C88ADF802404B88ADF842
:1014D0000430CA88ADF808208988ADF806100021CC
:1014E000ADF80A10ADF80C1080B14FF6FF70062170
:1014F000844201D1ADF80210834201D1ADF804104D
:10150000824203D14FF44860ADF8080068460DF000
:10151000E2FB06F00DFC04B010BD70B514460D469C
:101520000646FFF788FE60B90DB1A54201D90C202F
:1015300070BD002409E000BF56F82400FFF77BFED1
:1015400008B1102070BD641CE4B2AC42F4D300209A
:1015500070BD2DE9F04105461F4690460E46002419
:101560000068FFF7B5FE30B9A98828680844401E16
:10157000FFF7AEFE10B11020BDE8F081286800280A
:10158000A88802D0B84202D850E00028F4D0092040
:10159000F2E72968085DB8B1671CCA5D152A2ED02C
:1015A0003CDC152A3AD2DFE802F039122222282840
:1015B0002A2A313139393939393939393939220019
:1015C000085D30BB641CA4B2A242F9D833E0022803
:1015D000DDD1A01C085C88F80000072801D2400774
:1015E00001D40A20C8E7307840F0010015E0C1437B
:1015F000C90707E0012807D010E00620BCE7010773
:10160000A1F180510029F5D01846B5E7307881075F
:1016100001D50B20B0E740F0020030702868005D73
:10162000384484B2A888A04202D2B0E74FF44853AD
:1016300082B2A242ADD800209EE710B502785408CD
:1016400009D0012243F20223012C07D0022C0DD035
:10165000032C13D10FE00020087005E080790324EB
:10166000B4EB901F0AD10A70002010BD8079B2EB54
:10167000901F03D1F7E780798009F4D0184610BD98
:1016800008B500208DF800004F4890F8221051B1A5
:1016900090F8230002280FD003280FD0FFDF00BFEF
:1016A0009DF8000008BD48486946193001F0CCF9A2
:1016B0000028F5D0FFDFF3E7032000E001208DF8DC
:1016C0000000EDE738B50C460546694601F0BCF967
:1016D00000280DD19DF80010207861F3470020709C
:1016E00055F8010FC4F80100A888A4F805000020EF
:1016F00038BD38B51378C0B1022816D033A46D4672
:10170000246800944C7905EB9414247864F347031F
:10171000137003280ED003F0FE0010700868C2F8A2
:1017200001008888A2F8050038BD23F0FE0313707D
:101730000228EED1D8B240F00100EEE702210EF00F
:10174000E7BC38B50C460978222901D2082038BDFB
:10175000ADF800008DF8022068460DF0FEF906F0A5
:10176000E7FA050003D121212046FFF756FE28465F
:1017700038BD1CB500208DF80000CDF80100ADF893
:101780000500114890F82200022801D0012000E055
:1017900000208DF8070068460DF048FA002800D0B8
:1017A000FFDF1CBD2DE9FF478CB00025BDF834607C
:1017B00082461C4690468DF81C50700703D5606821
:1017C000FFF739FD90B903E09C0100200302FF01FF
:1017D000FE4F4FF0010997F8220058B197F8230007
:1017E000022807D16068FFF773FD18B1102010B010
:1017F000BDE8F087300702D5A089802815D870078A
:1018000004D4B8F1000F01D0387E70B1E07DC0F390
:1018100000108DF81B00617D072041B1012906D021
:101820000229E4D00429E2D117E00720DFE78DF890
:1018300017908DF819908DF81580606878B107A918
:10184000FFF7FBFE0028D2D1606850F8011FCDF8E9
:101850000F108088ADF8130005E00620C7E7CDF82B
:101860000F50ADF81350E07B0028F6D1207C002803
:10187000F3D1607C0028F0D1A07C0028EDD1E07C81
:10188000C006EAD18DF800A0BDF83400ADF8020022
:10189000A0680190A0680290CDA0D0E90010CDE929
:1018A0000A10E07C0AA901EB501000788DF80C00BA
:1018B000FFF7E6FE8DF80D009DF81C008DF80E0078
:1018C0008DF818508DF816508DF81A5009A96846F1
:1018D0000DF050FA06F02CFA89E7F0B58FB000242D
:1018E0008DF830408DF814408DF8344006468DF860
:1018F0002840019402940394049419B10FC901ADD6
:1019000085E80F00B14DA878052801D004280CD136
:1019100001986968884200D120B90398E968884233
:1019200003D110B108200FB0F0BD1F273B460DAA10
:1019300005A903A8FFF70DFE0028F4D13B460AAA2B
:101940000CA901A8FFF705FE0028ECD19DF81400B2
:10195000C00701D00A20E6E7A88A410708D4A97D7C
:1019600031B19DF82810890702D043F20120DAE74F
:101970009DF82810C90709D0400707D4288818B156
:1019800044F25061884201D90720CCE78DF8184015
:101990008DF81960BDF80800ADF81A00019807909D
:1019A00006A80DF0F2F906F0C3F90028BBD18DF8B6
:1019B00020408DF82160BDF81000ADF8220003989A
:1019C000099008A80DF003FA06F0B2F90028AAD190
:1019D00001AC2D1D94E80F0085E80F000020A2E760
:1019E00070B50646FFF7AAFE054606F083FB040025
:1019F00000D1FFDF6680207820F00F00801C20F0EF
:101A0000F000203020700320207295F83E006072B4
:101A1000BDE8704006F072BB2DE9F04385B00400CC
:101A200000D1FFDF2078694E20F00F00801C20F0ED
:101A3000F0007030207060680178C91F14292AD224
:101A4000DFE801F04DF3290AF3F33AF2292966F2AF
:101A5000F2F129F2F2F0EFF286883046FFF76EFEDF
:101A60000546304608F0D9F8C0B16068807985F83D
:101A70003E0021212846FFF7D0FC304603F002FA51
:101A8000304604F0C1FB3146012012F073F9A87F03
:101A900020F01000A87705B0BDE8F083207820F092
:101AA000F00020302070032020726680606880790A
:101AB000607206F023FBDCE785882846FFF73EFED0
:101AC00000B9FFDF60688078012800D0FFDF606820
:101AD000817905B02846BDE8F04308F066BA8688EB
:101AE0003046FFF72BFE050000D1FFDF06F006FBB6
:101AF00060683146C08828816068008968816068B4
:101B00004089A881012012F035F90020A875C2E7AC
:101B1000807828B10228BED03C28BCD0FFDFBAE7CD
:101B200006F0ECFA6568A879AD1C00B9FFDFF7781C
:101B3000B5F80290B046384606F073F8060000D1BA
:101B4000FFDF0022022148460EF0D9FA040000D13E
:101B5000FFDF22212046FFF760FCA17F012060F318
:101B60000101A177298B2181698B6181A98BA181D9
:101B700084F822708DF80800B0680090F068019039
:101B80006A46032148460EF0BAFA00B9FFDFB08872
:101B9000ADF81000B0788DF8120004AA052148466F
:101BA0000EF0ADFA00B9FFDFB088ADF80C00F078A8
:101BB0008DF80E0003AA042148460EF0A0FA00B9E1
:101BC000FFDF062105F1120006E000009C01002065
:101BD000070605040302010000F053FF30B36879E3
:101BE000800700D5FFDF6979E07D61F34700E0758C
:101BF000D5F80600A0616889A083062105F10C00D4
:101C000000F03FFFE0B198F819104A08617862F3DC
:101C100047016170D8F81A10C4F80210B8F81E0015
:101C200017E028E020E033E02DE017E0E07D20F031
:101C3000FE00801CE075D5F81200A061E88ADBE7A1
:101C4000607820F0FE00801C6070E868C4F8020034
:101C5000288AE0800320FFF7B7FB1CE705B0204689
:101C6000BDE8F04301F092BC06F048FA16F8240FE4
:101C700040F0020005E006F041FA16F8240F40F0AB
:101C80000400307007E705B0BDE8F04306F036BA4F
:101C9000B178052909D00429DFD106F02FFA0220F6
:101CA00005B0BDE8F043FFF78FBB80780028D4D0A3
:101CB000F07800F0B0FE06F021FA0320F0E72DE9FD
:101CC000F047054600780027000991460C463E463D
:101CD000012871D0022870D007280AD00A286DD0B8
:101CE000FFDF00BFA9F800600CB1278066800020EC
:101CF0007EE5D5F804C0DFF8508804F108009CF8B0
:101D000000204FF0010AD21F4FF6FF71142A76D23D
:101D1000DFE802F00AF9F9F9F9F9F91DF9F926C035
:101D2000889DF91061D476EE12271026BCF80400C5
:101D30002146F3E01C270A26ECB3BCF80200A08081
:101D4000686800792072686840796072CAE71B276A
:101D5000092684B30320207268684088A080C1E708
:101D60009CF802103C29BDD010272C260CF1020C47
:101D70000CB3BCF80210A180BCF818106182BCF84A
:101D800018102182BCF81A10A182BCF81C10E18244
:101D90009CF8053002460CF106011846FFF7A9FC35
:101DA0009CF8040001289DD184F80FA00020207623
:101DB00008F1040003E00BE0A8E0B2E0EAE090E8FC
:101DC0000E00D8F81000C4E90930C4E9071289E709
:101DD000A9F800608BE720271126002CF8D0A180FD
:101DE000686804F10A02807820726868807A6072FC
:101DF00069680B1DC8781946FFF77BFC72E782E023
:101E000021270A26002CE3D0BCF80200A0806868D5
:101E10000079207268684079607298F8241021F087
:101E2000040162E022270B26002CD1D0BCF804006C
:101E3000A0806868807820726868807900F030FE41
:101E400060726868C07900F02BFEA0724AE726270E
:101E50001C26002CBCD0A1806868C07860726868BD
:101E60008079A07208F1040090E80E00D8F8100004
:101E7000C4E90530C4E90312686880783C2803D0BF
:101E8000432804D0FFDF2DE784F808A02AE70220CA
:101E9000207227E724271026002C99D0BCF80200D6
:101EA000A0806868007920816868007A608168682D
:101EB000C088A08168684089E08113E72327102645
:101EC000002C85D0BCF80200A08068688088208142
:101ED0006868C088608168680089A08168684089F6
:101EE000E08198F8241021F0020188F82410F9E626
:101EF0002F272A26002C86D0A18069682222891CDF
:101F00000BF039FAEEE64A46214644E0287A0228E8
:101F100001D0FFDFE6E612271026688800F09EFD5C
:101F2000E0E6287AB0B3012835D0022833D0032860
:101F300001D0FFDFD6E611270926002C8AD0B5F89C
:101F400002804046FFF7FAFB90F822A0A4F8048034
:101F5000687A2072042140460EF0ECF805214046D4
:101F60000EF0E8F8002140460EF0E4F8012140466A
:101F70000EF0E0F8032140460EF0DCF80221404666
:101F80000EF0D8F8062140460EF0D4F8504600F086
:101F900042FDA7E6FFE72846BDE8F04701F02CBC6C
:101FA00070B5012801D0FFDF70BD8DB22846FFF764
:101FB000C5FB040000D1FFDF20782128F4D006F013
:101FC00099F880B1017821F00F01891C21F0F0010E
:101FD000103101700221017245800020A075BDE81A
:101FE000704006F08BB821462846BDE870401322A9
:101FF000FFF7A7BB2DE9F04116460C00804600D143
:10200000FFDF307820F00F00801C20F0F00010304F
:1020100030702078022802D0FFDFBDE8F081404612
:10202000FFF78CFB050000D1FFDFA1884FF6FF70A2
:102030000027814202D1E288824203D0814201D14D
:10204000E08840B106F05AF894E80F00083686E8B8
:102050000F00AF75E1E7A87D0128DED178230022CB
:10206000414611F0DDFD0220A875D6E738B50C46D3
:1020700024283CD006DC20280CD021280CD0222893
:1020800006D12FE0252826D0262819D03F2836D083
:10209000072038BD062038BD6068FFF710F9A0B9E9
:1020A000618820886A460DF00AF805F041FE002894
:1020B000F1D161680029EED0BDF800200A8038BD5A
:1020C000206820B1FFF704F908B1102038BD204680
:1020D0000DF0B2F80FE0A07800F0010120880DF0BB
:1020E0001FF808E00868BDE8384001F0BABD618813
:1020F00020880CF07DFFBDE8384005F019BE087857
:1021000000F001008DF8000068460CF0DBFD05F0E2
:102110000FFE38BD70B505460C460846FFF7B1F80E
:1021200008B1102070BD202D07D0212D0DD0222DFB
:102130000BD0252D09D0072070BD2088A11C0CF0E4
:102140005BFDBDE8704005F0F3BD062070BDFE48A4
:102150001930704708B528220021FB480BF035F9EB
:102160000120FFF731F9F84968461A3105F058FFA8
:10217000F5489DF80020417E62F3470121F00101FE
:102180004176002180F822104FF461710184022110
:1021900080F82310FFF730F900B1FFDF00F0AEFC4C
:1021A00001F0C6F908BD10B50C46402200212046BA
:1021B0000BF00BF9A07F20F00300A0772020207007
:1021C0000020A07584F8230010BD70472DE9FC4164
:1021D0000746FFF730F810B11020BDE8FC81DA4E59
:1021E00006F11901D6F819000090B6F81D50ADF8A7
:1021F0000450F47F8DF806403846FFF763FA002854
:10220000EBD1FFF7F9F80028E7D0009946F8191F3D
:10221000B580B471E1E710B50446FFF732F808B1B4
:10222000102010BDC848C8492246407E1A314008D7
:10223000FFF75FFA002010BD3EB504460D46084684
:10224000FFF71FF808B110203EBD14B143F204009F
:102250003EBDBD488078052803D0042801D0082061
:102260003EBD694602A80BF036FB2A4669469DF83A
:102270000800FFF73EFA00203EBDFEB50D46040003
:102280004FF0000711D00822FFF747F9002811D1BD
:10229000002608E054F826006946FFF7CEF900282A
:1022A00008D1761CF6B2AE42F4D30CF053FB10B159
:1022B00043F20320FEBDA44E3776FCB100271AE09E
:1022C00054F8270002A9FFF7B8F900B1FFDF9DF825
:1022D00008008DF8000054F8270050F8011FCDF8D1
:1022E00001108088ADF8050068460CF058FB00B17D
:1022F000FFDF7F1CFFB2AF42E2D335760020FEBD88
:102300002DE9F0478AB01546894604001DD00F46D6
:1023100008222946FFF701F9002810D1002612E013
:1023200054F826006946103000F08EFB002806D1D4
:102330003FB157F82600FEF77EFF10B110200AB01B
:10234000D6E4761CF6B2AE42EAD30026A5F1010827
:102350001CE000BF06F1010A0AF0FF0712E000BF0F
:1023600054F82600017C4A0854F827100B7CB2EB85
:10237000530F05D10622113011310AF0CFFF58B1A9
:102380007F1CFFB2AF42EBD30AF0FF064645E1DB0C
:102390004E4624B1012003E043F20520CFE70020A0
:1023A0000CF01CFB10B90CF025FB10B143F204201B
:1023B000C5E75CB300270DF1170825E054F82700A6
:1023C0006946103000F040FB00B1FFDF54F82700F1
:1023D000102250F8111FCDF801108088ADF80500CB
:1023E00054F827100DF107000AF0C5FF96B156F812
:1023F0002710102240460AF0BEFF68460CF0B4FADF
:1024000000B1FFDF7F1CFFB2AF42D7D3FFF7B1F9B6
:10241000002094E7404601F018FCEEE730B585B0A7
:102420000446FEF708FF18B96068FEF751FF10B1C7
:10243000102005B030BD60884AF2B811884206D835
:102440002078414D28B1012806D0022804D0072069
:10245000EFE7FEF7D1FF18E06078022804D00328E8
:1024600002D043F20220E4E785F82300C1B2002045
:102470000090ADF8040002292CD0032927D0FFDFFB
:1024800068460CF02BFB05F053FC0028D1D16068A6
:1024900001F0CEFB207858B101208DF800000DF13D
:1024A000010001F0D2FB68460CF093FE00B1FFDFA3
:1024B000207885F82200FFF75CF9608860B12884F5
:1024C00080B20CF083FA00B1FFDF0020B1E78DF895
:1024D0000500D5E74020FAE74FF46170EFE710B54B
:1024E0000446FEF7CEFE20B9606838B1FEF7E7FE7D
:1024F00008B1102010BD606801F0A7FB124830F849
:10250000201F6180C178617080782070002010BD2C
:102510002DE9F843144689460646FEF7B2FEB8B9DF
:102520004846FEF7D5FE98B92046FEF7D1FE78B9A9
:10253000054DA878012800D154B13178FF2909D080
:1025400061B143F2040001E09C010020BDE8F88382
:102550001020F8E7012801D00420F4E7CCB30528C7
:1025600011D004280FD06946204600F0A4FA0028B4
:10257000E9D1217D49B1012909D0022909D00329D6
:1025800009D00720DFE70820DDE7024604E001224A
:1025900002E0022200E00322804623461746002084
:1025A0000099FFF7FFF80028CDD1A0892880A07BF3
:1025B000E875BDF80000A882AF75BDF800100907E6
:1025C00001D5A18931B1A1892980C00704D0032098
:1025D00003E006E08021F7E70220FEF7F5FE86F82B
:1025E00000804946BDE8F8430020FFF776B92DE9A1
:1025F000FC41FF4C06460D46A078022803D0032874
:1026000001D00820E9E516B143F20400E5E5062013
:102610000DF032FD10B9A078032849D00FF098FCD6
:10262000074610F0F7FE381A00F0FF0806200DF0FC
:102630001BFD074606200DF01FFD391AA07804285F
:1026400009D000221144A8EB010111F0FF0F04D0C2
:10265000032804D00DE00122F4E71320BDE528464D
:1026600005F0DFFA10B3407810B3284605F0E4FD1A
:10267000E570FFF705F80BF070F801208DF8000009
:102680008DF801008DF802602088ADF80400E07D2F
:102690008DF8060068460CF06EFC05F049FB00283A
:1026A000B0D1A078032805D0042010E0052094E5DF
:1026B000122092E5E07805F0B4FA040000D1FFDFC3
:1026C000607800B9FFDF6078401E60700520FEF77B
:1026D0007BFE002081E51CB510B143F204001CBD57
:1026E000C34CA078042803D0052801D008201CBDC5
:1026F00000208DF8000001218DF801108DF80200F6
:1027000068460CF038FC05F013FB0028EFD1A078E8
:10271000052805D05FF00200FEF756FE00201CBD24
:10272000E07800F078F90320F6E72DE9FC418046D7
:102730000D4603260846FEF7CBFD08B110204CE5F8
:102740004046FEF7FBFF040004D02078222804D284
:10275000082042E543F202003FE5A07F00F00307B6
:102760003DB1012F0AD000202946FEF7A8FE060041
:10277000E5D1012F04D0FFDF30462EE50120F3E73D
:10278000A07D2946022801D011B107E0112024E5DF
:10279000684600F0E7FA0028D1D16946404607F0C4
:1027A000E4FB0600E8D10120A075E5E770B50C4612
:1027B0000546FEF7C3FF010005D022462846BDE8C6
:1027C0007040FEF7BEBF43F2020070BD10B5012895
:1027D00007D1874B9B78012B00D011B143F2040045
:1027E00010BD0CF025F9BDE8104005F0A1BA012399
:1027F00000F01BB900231A46194600F016B970B54F
:10280000064615460C460846FEF73BFD18B9284615
:10281000FEF737FD08B1102070BD2A46214630462C
:102820000CF035FC05F084FA0028F5D121787F29D9
:10283000F2D1052070BD7CB505460C460846FEF772
:10284000FAFC08B110207CBD2846FEF777FF20B1C6
:102850000078222804D208207CBD43F202007CBD0F
:10286000634890F82400400701D511207CBD2178F1
:10287000C80802D16078C20801D007207CBD890851
:1028800001D1800801D006207CBDADF80050207831
:102890008DF8020060788DF803000220ADF8040086
:1028A00068460BF02BFF05F043FA7CBD70B586B08F
:1028B00014460D460646FEF741FF28B1007822284F
:1028C00005D2082006B070BD43F20200FAE72846A0
:1028D000FEF7FEFC20B944B12046FEF7F0FC08B13B
:1028E0001020EFE700202060A080414890F82400ED
:1028F000800701D51120E5E703A930460BF03BFF27
:1029000018B100BF05F014FADCE7ADF80060BDF8BF
:102910001400ADF80200BDF81600ADF80400BDF8D3
:102920001000BDF81210ADF80600ADF808107DB12A
:10293000298809B1ADF80610698809B1ADF802100F
:10294000A98809B1ADF80810E98809B1ADF80410FB
:10295000DCB1BDF80610814201D9081A2080BDF80B
:102960000210BDF81400814201D9081A6080BDF838
:102970000800BDF80410BDF816200144BDF812008F
:102980001044814201D9081AA08068460BF090FFDC
:10299000B8E770B505460C460846FEF772FC08B16C
:1029A000102070BD214628460CF068F9BDE8704043
:1029B00005F0BEB93EB505460C460846FEF761FC7B
:1029C00008B110203EBD0020009001900290ADF8AB
:1029D00000502089ADF8080020788DF8020060686A
:1029E00001902089ADF808006089ADF80A0001E087
:1029F0009C01002068460CF04FF905F099F93EBDA6
:102A00000EB5ADF800000020019068460CF044F9C6
:102A100005F08EF90EBD10B505F003F9040000D1E4
:102A2000FFDF6078401C607010BD1CB5ADF8000081
:102A30008DF802308DF803108DF8042068460CF0F4
:102A4000F5FA05F075F91CBD0278520804D0012A88
:102A500002D043F202207047FEF7EFBD70B50C00C4
:102A600006460DD0FEF76AFE050000D1FFDFA68006
:102A700028892081288960816889A081A889E081CE
:102A800070BD10B500231A4603E0845C2343521C3A
:102A9000D2B28A42F9D30BB1002010BD012010BD83
:102AA00000B530B1012803D0022801D0FFDF00209B
:102AB00000BDFF2000BD00220A8092B222F0600219
:102AC0000A800078062817D2DFE800F0160306090E
:102AD0000C1142F0110007E042F01D0009E042F045
:102AE000150006E042F0100040F0020001E042F064
:102AF000100008800020704707207047FD48002123
:102B000001604160018170472DE9FF4F93B09B4602
:102B1000209F160004460DD01046FEF78CFB18B11E
:102B2000102017B0BDE8F08F31460120FEF7C7FC3A
:102B30000028F6D101258DF842504FF4C050ADF871
:102B40004000002210A9284603F024FE0028E8D106
:102B50008DF84250A8464FF428500025ADF84000AB
:102B60001C222946684607950AF02FFC9DF81C0098
:102B70000DF11C0A20F00F00401C20F0F000103076
:102B80008DF81C0020788DF81D0061789DF81E00DE
:102B90000DF1400961F3420040F001008DF81E0084
:102BA0009DF8000008AA40F002008DF8000020897E
:102BB000ADF83000ADF832506089ADF83400CDF892
:102BC0002CA060680E900AA9CDF82890684603F002
:102BD000D6FB0028A5D16068FEF771FB40B16068A4
:102BE000FEF776FB20B9607800F00300022801D0E0
:102BF000012000E00020BF4C08AA0AA92072BDF8FD
:102C0000200020808DF8428042F60120ADF840007F
:102C10009DF81E0020F00600801C20F001008DF8B9
:102C20001E000220ADF83000ADF8340014A80E905C
:102C3000684603F0A4FB002889D1BDF8200060801D
:102C400036B1211D304600F059F90028C2D109E003
:102C5000BBF1000F05D00AF033F9E8BB0AF030F9F8
:102C6000D0BBA58017B1012F43D04AE08DF8428038
:102C700042F6A620ADF8400046461C2200216846D8
:102C800007950AF0A2FB9DF81C00ADF8346020F017
:102C90000F00401C20F0F00010308DF81C009DF853
:102CA0001D0020F0FF008DF81D009DF81E0020F093
:102CB000060040F00100801C8DF81E009DF8000009
:102CC0008DF8446040F002008DF80000CDE90A9ACA
:102CD000ADF8306011A800E011E00E9008AA0AA932
:102CE000684603F04CFB0028A6D1BDF82000E08028
:102CF00008E00AF0E5F810B90AF0E2F808B103209C
:102D00000FE7E58000200CE73EB50446794D08202A
:102D1000ADF80000A88828B12046FEF78CFA18B15B
:102D200010203EBD06203EBD21460120FEF7C7FB18
:102D30000028F8D12088ADF804006088ADF80600BE
:102D4000A088ADF80800E088ADF80A00A88801ABBB
:102D50006A46002103F01AFFBDF800100829E2D0EE
:102D600003203EBD7FB5634D0446A88868B10020AE
:102D700002900820ADF80800CDF80CD02046FEF7F0
:102D80005AFA20B1102004B070BD0620FBE7A988D4
:102D900002AA4FF6FF7004F03BF90028F3D1BDF80A
:102DA0000810082901D00320EDE7BDF800102180AC
:102DB000BDF802106180BDF80410A180BDF80610B6
:102DC000E180E0E701B582B00220ADF8000049489B
:102DD00002AB6A464088002103F0D8FEBDF800101F
:102DE000022900D003200EBD1CB500210091022154
:102DF000ADF800100190FEF744FA08B110201CBD98
:102E00003C486A4641884FF6FF7004F001F9BDF86E
:102E100000100229F3D003201CBDFEB5354C064638
:102E20001546207A0F46C00705D00846FEF703FA7C
:102E300018B11020FEBD0F20FEBDF82D01D90C20C9
:102E4000FEBD3046FEF7F7F918BB208801A902F055
:102E500098FF0028F4D130788DF80500208801A96A
:102E600003F072FE0028EBD100909DF800009DF861
:102E7000051040F002008DF80000090703D040F073
:102E800008008DF800002088694603F0FAFD00284C
:102E9000D6D1ADF8085020883B4602AA002103F0A5
:102EA00075FEBDF80810A942CAD00320FEBD7CB54E
:102EB00005460020009001900888ADF800000C46FF
:102EC00028460195FEF7FBF918B92046FEF7D9F917
:102ED00008B110207CBD15B1BDF8000060B10548F7
:102EE0006A4601884FF6FF7004F092F8BDF80010B2
:102EF00021807CBDC40100200C20FAE730B50446D7
:102F000093B000200D4601460090142201A80AF05B
:102F10005CFA1C22002108A80AF057FA9DF800006C
:102F2000CDF808D020F00F00401C20F0F000103049
:102F30008DF800009DF8010006AA20F0FF008DF832
:102F400001009DF8200001A940F002008DF820004A
:102F500001208DF8460042F60420ADF8440011A887
:102F600001902088ADF83C006088ADF83E00A08854
:102F7000ADF84000E088ADF842009DF8020020F076
:102F80000600801C20F001008DF802000820ADF83A
:102F90000C00ADF810000FA8059008A803F0EFF999
:102FA000002803D1BDF818002880002013B030BDE0
:102FB0000A4810B5046809490948083108600FF04B
:102FC000DAFE0648001D046010BD064900200860B6
:102FD0004FF0E0210220C1F8800270471005024046
:102FE00001000001FC1F004070B50C46054608F0CA
:102FF000C7FB21462846BDE8704009F0A8BC000088
:103000002CFFFFFFDBE5B15100C001000201FFFF13
:103010007100000090D76A00773D4B16B620AFF9DB
:10302000F4D1D1B6F33F7AC76170DB6D10B50446B9
:10303000FEF701F908B1102010BD2078C0F302108E
:10304000042807D86078072804D3A178102901D86C
:10305000814201D2072010BDE078410706D42179D2
:103060004A0703D4000701D4080701D5062010BD84
:10307000002010BD70B514460D46064605F03AF81E
:1030800080B10178182221F00F01891C21F0F00194
:10309000A03100F8081B21460AF06DF9BDE8704028
:1030A00005F02CB829463046BDE870401322FEF7E3
:1030B00048BB2DE9F047064608A8904690E8300442
:1030C00089461F461422002128460AF07EF9002175
:1030D000CAF80010B8F1000F03D0B9F1000F03D106
:1030E00014E03878C00711D02068FEF7CAF8C0BBDA
:1030F000B8F1000F07D12068123028602068143022
:1031000068602068A8602168CAF8001038788007D5
:1031100024D56068FEF7D3F818BBB9F1000F21D0B1
:10312000FFF715F80168C6F868118188A6F86C11D8
:10313000807986F86E0101F034FAF84FEF6062682A
:1031400062B196F8680106F2691140081032FEF784
:10315000D0FA1022394660680AF00DF90020BDE867
:10316000F08706E0606820B1E8606068C6F8640136
:10317000F4E71020F3E730B5054608780C4620F058
:103180000F00401C20F0F001103121700020607011
:1031900095F8230030B104280FD0052811D0062857
:1031A00014D0FFDF20780121B1EB101F04D295F875
:1031B000200000F01F00607030BD21F0F0002030D2
:1031C00002E021F0F00030302070EBE721F0F00059
:1031D0004030F9E7F0B591B0022715460C46064697
:1031E0003A46ADF80870092103AB05F08CFD049058
:1031F000002810D004208DF804008DF80170E03410
:10320000099605948DF818500AA968460EF07BFCC3
:1032100000B1FFDF012011B0F0BD2DE9F84F0646E7
:10322000808A0C4680B28246FEF788FA0546BB4F7C
:103230003078203F4FF002094FF000080F287CD271
:10324000DFE800F07BA39D082C5B6A7CBADAFD976F
:1032500048979700012150460CF05AFF040000D116
:10326000FFDF97F85C00C00701D0386E0BE0032148
:1032700004F11D0010F097FAD4F81D00A849B0FB26
:10328000F1F201FB1200C4F81D0070686067B068BD
:10329000A0672878252872D0FFDF70E00121504612
:1032A0000CF036FF060000D1FFDF3078810702D531
:1032B0002978252904D040F001003070BDE8F88F4E
:1032C00084F80090307F207106F11D002D36C4E98E
:1032D0000206F3E7012150460CF01AFF050000D169
:1032E000FFDF2878C10604D5072020703D356560D2
:1032F000E4E740F008002870E0E7E87F000700D529
:10330000FFDF307CB28800F0010301B05046BDE819
:10331000F04F092106F08BBD05B9FFDF716821B1BF
:10332000102205F124000AF026F828212846FEF78D
:1033300074F8307A85F82000C0E7F7E001215046A4
:103340000CF0E6FE050000D1FFDF022105F185004B
:1033500010F029FA0420207005F5B4706060B5F80B
:10336000850020826D4810387C356561C4E90270A3
:10337000A4E7012150460CF0CBFE00B9FFDF324636
:1033800029465046BDE8F84F74E605B9FFDF2878B6
:10339000212893D93079012803D1E87F40F0080033
:1033A000E877324629465046FFF764FE2846BDE8D6
:1033B000F84F2321FEF731B83279A28004F10803D7
:1033C0000921504605F09FFCE06010B105202070F7
:1033D00074E74546012150460CF09AFE040000D1E6
:1033E000FFDF04F1620102231022081F0CF029FD07
:1033F00005703179417061E7012150460CF088FE7B
:10340000040000D1FFDF94F8840000F003000128DD
:1034100059D1E87F10F0010003D194F8A010C9073A
:103420002AD0D4F8602132B394F88330117C63F34E
:1034300087011174AA7FD30963F3410100E071E0B1
:10344000D4F860211174D4F8602160F30001117484
:1034500090B1D4F86001102205F12401883409F0FC
:103460008AFF207E40F001002076207820F00100C5
:1034700004F8880919E0C0B994F88810C90714D075
:10348000D4F85C218AB194F88330117C63F387010E
:103490001174AA7FD309D4F85C2163F3410111743C
:1034A000D4F85C2160F30001117494F8880080075F
:1034B00009D594F87C00D4F86421400804F17D011A
:1034C0001032FEF716F98DF8009094F884006A46E1
:1034D00000F003008DF8010094F888108DF80210B8
:1034E00094F8A0008DF803002946504601F042F8F8
:1034F0002878252805D0212807D0FFDF2878222822
:1035000003D922212846FDF788FF012150460CF0FF
:1035100011FE00283FF4DDAEFFDFCFE6F001002012
:1035200040420F00716881F80180C7E6FFDFC5E601
:1035300070B5FE4C002584F85C5025660EF0AFFA9D
:1035400004F11001204604F091FD84F8305070BD64
:1035500070B50D46FEF7F2F8040000D1FFDF4FF41E
:10356000B8720021284609F030FF2434012105F10A
:10357000E0002C610EF094FA002800D0FFDF70BD4F
:103580000A46014602F1E0000EF0ABBA70B50546FE
:10359000406886B00178082906D00B2933D00C2961
:1035A0002FD0FFDF06B070BD46883046FEF7C6F864
:1035B000040000D1FFDF20782128F3D028281BD178
:1035C000686802210C3000F0A0FFA8B168680821EB
:1035D000001D00F09AFF78B104F1240130460BF091
:1035E000CCFC04F0A5FB00B1FFDF06B02046BDE82F
:1035F00070402921FDF711BF06B0BDE8704004F00E
:103600007DBD01218171686886883046FEF796F895
:10361000040000D1FFDF20782128C3D068688179B9
:1036200009B1807808B1FFDFBCE704F067FDA07F37
:10363000000622D5E07FC00705D094F8200000F0F6
:103640001F00102817D0052084F82300207829288F
:1036500015D02428A6D13146042010F08BFB22215E
:103660002046FDF7DAFE012130460CF063FD00280C
:1036700098D0FFDF96E70620E6E70420E4E7012183
:1036800030460CF045FD050000D1FFDF2521204626
:10369000FDF7C3FE03208DF80000694605F1E00048
:1036A0000EF016FA0228BFD00028BDD0FFDF79E760
:1036B0002DE9F04788B09A46164688468146FEF7BF
:1036C0003DF805003AD02878222837D3232835D072
:1036D000E87F000732D40027012148460CF018FD8E
:1036E000040005D10121002248460CF008FD0446E3
:1036F000694600F066FF009800B9FFDF00983CB112
:10370000E03404612878222804D0242802D005E07F
:10371000076103E025212846FDF77FFE009801217F
:103720004170C0F824908680C0E9028A01A90EF099
:10373000EAF9022802D0002800D0FFDF08B00EE529
:1037400070B586B00546FDF7F9FF0078222814D938
:10375000012128460CF0DCFC04002CD1FFDF2AE01C
:10376000B4F85E0004F1620630440178427829B171
:1037700021462846FFF72EFDB0B913E7ADF8042027
:103780000921284602AB05F0BEFA03900028F4D0C8
:1037900005208DF80000694604F1E0000EF098F96C
:1037A000022801D000B1FFDF02231022314604F1CC
:1037B0005E000CF07CFBB4F860000028D0D1F1E68C
:1037C00010B586B00446FDF7B9FF0078222811D95C
:1037D000012120460CF09CFC040000D1FFDF0620F4
:1037E0008DF80000694604F1E0000EF071F9002840
:1037F00000D0FFDF06B010BD2DE9F84F0546007878
:103800000C460027010904F1080090463E46BA46DE
:10381000009002297ED0072902D00A2909D142E06E
:1038200068680178082905D00B292CD00C292AD0EA
:10383000FFDF72E114271C26002C6CD04088A0808A
:10384000FDF77CFF5FEA000900D1FFDF99F8170060
:1038500009F118014008009AFDF74BFF686880895C
:10386000208268684168C4F812108068C4F81600A5
:10387000A07E20F0060040F00100A07699F81E001E
:1038800040F020014FE01A270A26002CD5D080886E
:10389000A080FDF753FF050000D1FFDF2846009907
:1038A000FFF769FC39E10CB1A88BA080287A4FF0B2
:1038B000010B0B287ED006DC01287CD0022808D022
:1038C000032804D137E00D2876D00E2875D0FFDF0D
:1038D00023E11E270926002CAFD0A088FDF72EFF7C
:1038E0005FEA000900D1FFDF287B00F00300012818
:1038F000207A1DD020F001002072297B890861F315
:1039000041002072297BC90861F382002072297B63
:10391000090901E0F7E0AEE061F3C300207299F815
:103920001E0040F0400189F81E10F6E0D001002092
:1039300040F00100E0E713270D26002CA6D0A08858
:10394000FDF7FCFE81460121A0880CF0E1FB05009B
:1039500000D1FFDF686F817801F003010129217A2E
:1039600050D021F00101217283789B0863F341015B
:1039700021728378DB0863F38201217283781B094B
:1039800063F3C3012172037863F306112172437854
:1039900063F3C711217284F809A0C178A17202797A
:1039A000E17A62F30001E1720279520862F34101A7
:1039B000E17203E029E067E04EE05FE002799208FF
:1039C00062F38201E1720279D20862F3C301E1720B
:1039D0004279217B62F3000121734279520862F33C
:1039E000410121734279920862F382012173407987
:1039F000C00860F3C301217399F8000023282AD975
:103A0000262139E041F00101ADE71827102694B3D3
:103A1000A088FDF793FE00900121A0880CF078FBB0
:103A20005FEA000900D1FFDFE868A06099F80000B4
:103A300040F0040189F8001099F80100800708D5CA
:103A400084F80CB000980078232866D927210098C4
:103A500052E084F80CA060E015270F265CB1A08826
:103A6000FDF76CFE81460622E868009909F00BFD1F
:103A700084F80EB085E042E048463DE0162709266E
:103A8000ECB3287B207248E0287B19270E26B4B3BC
:103A9000C4F808A0A4F80CA0012807D0022808D078
:103AA00003280CD004280AD0FFDF15E084F808B002
:103AB00001E002202072607A20F003000BE0697BB5
:103AC000042801F00F0141F080012172F3D1607AE6
:103AD00020F00300401C6072A088FDF72FFE054611
:103AE0000078212819D0232800D0FFDF0121A088E9
:103AF0000CF020FB22212846FDF78FFC0DE0FFE7AC
:103B0000A8F800600EE00CB16888A080287A10B395
:103B1000012809D002283AD0FFDFA8F800600CB1D4
:103B200027806680002007E415270F26002CE7D0A9
:103B3000A088FDF703FE0121A0880CF0E9FA05003A
:103B400000D1FFDFD5F81D000622009909F09BFC8B
:103B500084F80EA0E1E717270926002CD0D0A08812
:103B6000FDF7ECFD81460121A0880CF0D1FA05009B
:103B700000D1FFDF6878800701D5022000E0012036
:103B8000207299F800002328C7D9272174E7192744
:103B90000E26002CB4D0A088FDF7D0FD5FEA000906
:103BA00000D1FFDFC4F808A0A4F80CA084F808A096
:103BB000A07A40F00300A07299F81E10C90961F3C1
:103BC0008200A07299F81F2099F81E1012EAD11FE6
:103BD00005D099F8201001F01F01102925D020F000
:103BE0000800A07299F81F10607A61F3C300607238
:103BF000697A01F0030101298FD140F0040060725D
:103C0000E87A217B60F300012173AA7A607B62F37A
:103C100000006073EA7A520862F341012173A97AC5
:103C2000490861F34100607377E740F00800D8E786
:103C300010B5F84C30B10146102204F1200009F013
:103C40009AFB012084F8300010BD10B5044600F046
:103C5000A8FCF04920461022BDE81040203109F0B0
:103C60008ABB70B5EB4D06004FF0000412D0FDF793
:103C7000E2FA08B110240BE00621304609F0EAFB15
:103C8000411C04D02866012085F85C0000E0072470
:103C9000204670BD0020F7E7007810F00F0204D036
:103CA000012A05D0022A0CD110E0000909D10AE04E
:103CB0000009012807D0022805D0032803D00428D2
:103CC00001D0072070470870002070470620704719
:103CD00005282AD2DFE800F003070F171F00087835
:103CE00020F0FF001EE0087820F00F00401C20F0BC
:103CF000F000103016E0087820F00F00401C20F093
:103D0000F00020300EE0087820F00F00401C20F07A
:103D1000F000303006E0087820F00F00401C20F062
:103D2000F0004030087000207047072070472DE9F0
:103D3000F043804687B00D464FF000090846FDF776
:103D4000C7FAA8B94046FDF7F9FC060003D0307861
:103D500022280BD104E043F2020007B0BDE8F08353
:103D600035B1B07FC10601D4000703D50820F4E7C0
:103D70001020F2E7F07F000701D50D20EDE70027C6
:103D8000012140460CF0C4F9040006D101210022B3
:103D900040460CF0B4F9040005D0694600F011FC6F
:103DA000009818B901E00420D7E7FFDF009802214E
:103DB000E0344170C0F82480446107810121017121
:103DC000297801F00102017E62F3010101762A786F
:103DD000520862F3820101762A78920862F3C301E5
:103DE00001762A78D20862F3041101762421304644
:103DF000FDF713FB01A900980DF085FE022801D004
:103E000000B1FFDF4846A8E72DE9FF4F0E46824983
:103E1000904697B09A4607C914AB4FF0000983E863
:103E200007001798FDF78AFC050006D02878262899
:103E300006D008201BB0BDE8F08F43F20200F9E77E
:103E400026B94046FFF7F2F80028F3D10121179870
:103E50000CF05EF9040000D1FFDF852E27D007DCCF
:103E6000EEB1812E1DD0822E1DD0832E08D11CE0F4
:103E7000862E1ED0882E1ED0892E1ED08A2E1ED0B1
:103E80000F2020710F281CD004F034F9D8B1012084
:103E90008DF83400201D0E902079B0B126E100206D
:103EA000EFE70120EDE70220EBE70320E9E705203B
:103EB000E7E70620E5E70820E3E70920E1E70A2035
:103EC000DFE70720B6E71120B4E798F80000D4E94F
:103ED0001D764208A87F002162F3C710A87798F8E2
:103EE00000008208E87F62F30000E87798F800009D
:103EF000C209607862F34100607098F8000002091E
:103F0000207862F34710207098F80000C2086078AB
:103F100062F30000607098F80100607198F800008A
:103F200000F00102B07862F30100B070AA7FD209FC
:103F300062F38200B070EA7F62F3C300B07062780F
:103F400062F30410B0702278C0F3C00052093270DE
:103F50006278C2F34002727098F80220F2707171B8
:103F60003171B978C1F3C00108405FEA000B2ED06F
:103F70005046FDF760F978BBDAF80C00FDF75BF905
:103F800050BBDAF81C00FDF756F928BBDAF80C0034
:103F9000A060DAF81C00E06060787A7842EA5001AC
:103FA00061F341006070B978C0B200EA111161F3A9
:103FB000000060700020207705F117006061681C28
:103FC000A061B07800F00300012806D046E06078D8
:103FD0007A7802EA5001E3E719E0B87800F00300CC
:103FE00001283BD1321D711D404600F099FA31790C
:103FF000387901408DF8281070797A7910408DF861
:10400000300001432AD05046FDF715F930B1102099
:1040100010E70000D001002098B101000AF1100063
:1040200004F5AE7304F18C028DE80D0000210AAB9B
:104030005A462046FFF73DF80028E9D104F5B07252
:1040400004F1A403CDF800A0CDE9013201210CABAD
:104050005A462046FFF72DF80028D9D1607880070E
:1040600022D4B078B978C0F38000C1F3800108434E
:104070001AD0307814AA397832F810204B00DA4080
:1040800002F00309B9F1030F01D14FF00209BBF1AE
:10409000000F09D0012801D0042805D1012901D041
:1040A000042901D14FF00409A87F40F08000A877CF
:1040B000E97F6BF30001E9776078800706D503207C
:1040C000A071BBF1000F11D100202CE00220B9F14A
:1040D000020F1AD0B9F1010F19D0B9F1040F2AD08B
:1040E0000020A071A87F20F08000A8772521284615
:1040F000FDF793F90DA904F1E0000DF0E9FC10B112
:10410000022800D0FFDF002094E6A071DCE7A07158
:104110000D22002104F1200009F057F9207840F029
:104120000200207001208DF84C0013AA2946179830
:1041300000F020FADAE70120A071D7E72DE9F0437B
:1041400087B09046894604460025FDF7F7FA070038
:1041500004D03878272804D00820FEE543F2020076
:10416000FBE5012120460BF0D3FF040000D1FFDF67
:10417000A6795FEA090005D0012821D0B9F1020F24
:1041800026D110E0B8F1000F22D1012E05D0022E69
:1041900005D0032E05D0FFDF2EE00C252CE00125F5
:1041A0002AE0022528E04046FDF745F8B0B9032E85
:1041B0000ED11022414604F11D0009F0DCF81BE08D
:1041C000012E02D0022E03D104E0B8F1000F13D06B
:1041D0000720C2E54046FDF72EF808B11020BCE5E7
:1041E0001022002104F11D0009F0EFF806214046DD
:1041F00009F030F9C4F81D002078252140F00200B4
:1042000020703846FDF709F92078C10713D020F057
:104210000100207002208DF8000004F11D000290C2
:104220008DF804506946C3300DF052FC022803D0CB
:1042300010B1FFDF00E0257700208EE530B587B0B4
:104240000D460446FDF77AFA60B1012120460BF0D5
:104250005FFF04000CD02846FCF7EDFF28B11020CA
:1042600007B030BD43F20200FAE72078400701D4DE
:104270000820F5E7294604F13D002022054609F013
:104280007AF8207840F01000207001070FD520F058
:104290000800207007208DF80000694604F1E00056
:1042A00001950DF015FC022801D000B1FFDF0020C0
:1042B000D6E770B50D460646FDF740FA18B100780E
:1042C000272817D102E043F2020070BD01213046D9
:1042D0000BF01EFF040000D1FFDFA079022809D1F6
:1042E0006078C00706D02A4621463046FEF772FFA6
:1042F00010B10FE0082070BDB4F860000E280BD29A
:1043000004F1620102231022081F0BF09AFD012123
:1043100001704570002070BD112070BD70B506465B
:1043200014460D460846FCF786FF18B92046FCF7F0
:10433000A8FF08B1102070BDA6F57F40FF380ED051
:104340003046FDF7FBF938B1417822464B08811C15
:104350001846FDF7CEF907E043F2020070BD204693
:10436000FDF759FF0028F9D11021E01D0FF01BFACD
:10437000E21D294604F1170000F033F9002070BD5A
:104380002DE9F04104468AB015460E46002708463E
:10439000FCF79EFF18B92846FCF79AFF18B11020C9
:1043A0000AB0BDE8F0812046FDF7C8F95FEA0008D1
:1043B00004D098F80000272810D102E043F2020050
:1043C000EEE7012120460BF0A3FE040000D1FFDF41
:1043D0002078400702D56078800701D40820DFE705
:1043E000D4E91D01497801B18DB1407800B176B1B1
:1043F000ADB1EA1D06A8E16800F0F3F8102206A9A5
:1044000005F1170008F08AFF18B1042707E007201C
:10441000C6E71022E91D04F12D0008F0ACFF2EB113
:104420001022F11D04F11D0008F0A5FF20782521C0
:1044300040F0020020704046FCF7EFFF2078C107F3
:1044400015D020F00100207002208DF8000004F14A
:104450001D000290103003908DF804706946B3304F
:104460000DF036FB022803D010B1FFDF00E0277704
:10447000002095E770B50D4606460BB1072070BDCC
:10448000FDF75CF9040007D02078222802D3A07F32
:10449000800604D4082070BD43F2020070BDADB1A7
:1044A000294630460AF069FD03F042FC297C4A089F
:1044B000A17F62F3C711A177297CE27F61F300023B
:1044C000E277297C890884F8201004E030460AF05D
:1044D00077FD03F02DFCA17F21F02001A17770BDB5
:1044E00070B50D46FDF72AF9040005D02846FCF703
:1044F000C8FE20B1102070BD43F2020070BD2946F5
:104500002046FEF738FE002070BD04E010F8012BB5
:104510000AB100207047491E89B2F7D201207047C6
:1045200010B5C4780B7864F300030B70C47864088A
:1045300064F341030B70C478A40864F382030B7026
:10454000C478E40864F3C3030B700379117863F350
:104550000001117003795B0863F341011170037965
:104560009B0863F3820111700079C00860F3C301F6
:10457000117010BD70B51546064603F0BBFD040072
:1045800000D1FFDF207820F00F00801C20F0F00029
:104590002030207066802868A060BDE8704003F07D
:1045A000ADBD10B5134C94F83000002808D104F1CB
:1045B0002001A1F110000DF0CDFA012084F83000A7
:1045C00010BD10B190F8B9202AB10A4890F8350012
:1045D00018B1002003E0B83001E00648343008602C
:1045E000704708B50023009313460A460BF08FFF6F
:1045F00008BD0000D0010020F0B5007B059F1E46DD
:1046000014460D46012800D0FFDF0C2030803A20F0
:104610003880002C08D0287A032806D0287B01286F
:1046200000D0FFDF17206081F0BDA889FBE72DE9EE
:10463000F0470D4686B095F80C900E991446B9F1E6
:10464000010F0BD01022007B2E8A9046052807D040
:10465000062839D0FFDF06B0BDE8F0870222F2E776
:10466000E8890C2200EB400002EB40001880332068
:104670000880002CEFD0E8896081002720E00096B8
:10468000688808F1020301AA696900F097FF06EB48
:104690000800801C07EB470186B204EB4102BDF81D
:1046A00004009081F848007808B1012300E000235D
:1046B0000DF1060140460E320DF0B5FA7F1CBFB277
:1046C0006089B842DBD8C6E734200880E889B9F1B0
:1046D000010F11D0122148430E301880002CBAD09F
:1046E000E88960814846B9F1010F00D002202073AB
:1046F00000270DF1040A1FE00621ECE70096688808
:1047000008F1020301AA696900F058FF06EB0800EE
:10471000801C86B2B9F1010F12D007EBC70004EB81
:104720004000BDF80410C18110220AF102011030CE
:1047300008F021FE7F1CBFB26089B842DED88AE74C
:1047400007EB470104EB4102BDF80400D0810AF1F8
:104750000201404610320DF088FAEBE72DE9F047F0
:104760000E4688B090F80CC096F80C80378AF58910
:104770000C20DFF81493109902F10C04BCF1030F24
:1047800008D0BCF1040F3DD0BCF1070F75D0FFDF9E
:1047900008B061E705EB850C00EB4C001880312078
:1047A0000880002AF4D0A8F1060000F0FF0A558125
:1047B00024E01622002101A808F007FE0097708867
:1047C000434601AA716900F0F9FEBDF8040020809B
:1047D000BDF80600E080BDF80800208199F80000CF
:1047E00008B1012300E00023A21C0DF10A0150468C
:1047F0000DF019FA07EB080087B20A346D1EADB24E
:10480000D7D2C5E705EB850C00EB4C0018803220B1
:104810000880002ABCD0A8F1050000F0FF0A5581ED
:1048200037E000977088434601AA716900F0C6FE20
:104830009DF80600BDF80410E1802179420860F37C
:10484000000162F34101820862F38201C20862F34F
:10485000C301020962F30411420962F3451182099E
:1048600062F386112171C0096071BDF807002081D3
:1048700099F8000010B1012301E00EE00023224668
:104880000DF1090150460DF0CEF907EB080087B293
:104890000A346D1EADB2C4D27AE7A8F1020084B228
:1048A00005FB08FC0CF10E00188035200880002A5A
:1048B000A7D05581948100971FFA8CF370880E322F
:1048C000716900F07BFE63E72DE9F84F1E460A9DF3
:1048D0000C4681462AB1607A00F58070D080E0896C
:1048E000108199F80C000C274FF000084FF00E0AC9
:1048F0000D2872D2DFE800F09D070E1B272F3745E9
:10490000546972727200214648460095FFF774FEA2
:10491000BDE8F88F207B9146082802D0032800D0FC
:10492000FFDF3780302009E0A9F80A80F0E7207B1C
:104930009146042800D0FFDF378031202880B9F16C
:10494000000FF1D1E4E7207B9146042800D0FFDF7F
:1049500037803220F2E7207B9146022800D0FFDF2B
:1049600037803320EAE7207B1746022800D0FFDF9C
:104970003420A6F800A02880002FC9D0A7F80A800C
:10498000C6E7207B1746042800D0FFDF3520A6F8B5
:1049900000A02880002FBBD04046A7F80A8012E074
:1049A000207B1746052802D0062800D0FFDF102004
:1049B000308036202880002FAAD0E0897881A7F89F
:1049C0000E80B9F80E00B881A2E7207B9146072837
:1049D00000D0FFDF37803720B0E72AE04FF0120029
:1049E00018804FF038001700288091D0E089788136
:1049F000A7F80E80A7F8108099F80C000A2805D0B7
:104A00000B2809D00C280DD0FFDF81E7207B0A2876
:104A100000D0FFDF01200AE0207B0B2800D0FFDF61
:104A2000042004E0207B0C2800D0FFDF0520387331
:104A30006EE7FFDF6CE770B50C460546FCF77EFEBF
:104A400020B10078222804D2082070BD43F2020071
:104A500070BD052128460BF05BFB206008B10020EB
:104A600070BD032070BD30B44880087820F00F007E
:104A7000C01C20F0F000903001F8080B1DCA81E83E
:104A80001D0030BC03F03ABB100000202DE9FF47A9
:104A900084B00027824602970798904689461230D4
:104AA00006F05FFB401D20F00306079828B907A910
:104AB0005046FFF7C0FF002854D1B9F1000F05D0D0
:104AC0000798017B19BB052504681BE098F80000D6
:104AD000092803D00D2812D0FFDF46E007990325EF
:104AE0004868B0B3497B42887143914239D98AB250
:104AF000B3B2011D0BF091F90446078002E0079C58
:104B0000042508340CB1208810B1032D29D02CE0E5
:104B100007980121123006F056FBADF80C00024652
:104B200002AB2946504604F0EEF8070001D1A01C64
:104B3000029007983A461230C8F80400A8F802A07C
:104B400003A94046029B06F04BFBD8B10A2817D2B6
:104B500000E006E0DFE800F007091414100B0D1464
:104B60001412132014E6002012E6112010E608208B
:104B70000EE643F203000BE6072009E60D2007E6E8
:104B8000032005E6BDF80C002346CDE900702A4657
:104B90005046079900F022FD57B9032D08D1079818
:104BA000B3B2417B406871438AB2011D0BF049F9F1
:104BB000B9F1000FD7D0079981F80C90D3E72DE910
:104BC000FE4F91461A881C468A468046FAB102ABCF
:104BD000494604F098F8050019D04046A61C2788DD
:104BE0000BF0DBFB3246072629463B4600960AF0CF
:104BF000FAFF20882346CDE900504A4651464046F8
:104C000000F0ECFC002020800120BDE8FE8F002099
:104C1000FBE710B586B01C46AAB104238DF800301E
:104C20001388ADF808305288ADF80A208A788DF8DC
:104C30000E200988ADF80C1000236A462146FFF7C4
:104C400025FF06B010BD1020FBE770B50D4605210D
:104C50000BF05EFA040000D1FFDF294604F11200D8
:104C6000BDE8704006F098BA2DE9F8430D4680463D
:104C7000002603F03FFA04462878102878D2DFE8AF
:104C800000F0773B34533131123131310831313159
:104C900031312879001FC0B2022801D0102810D16C
:104CA00014BBFFDF35E004B9FFDF052140460BF000
:104CB0002FFA007B032806D004280BD0072828D021
:104CC000FFDF072655E02879801FC0B2022820D0D8
:104CD00050B1F6E72879401FC0B2022819D0102839
:104CE00017D0EEE704B9FFDF13E004B9FFDF28793E
:104CF00001280ED1172137E0052140460BF008FAB4
:104D0000070000D1FFDF07F11201404606F021FA4B
:104D10002CB12A4621464046FFF7A5FE29E0132183
:104D20004046FDF743FD24E004B9FFDF052140467E
:104D30000BF0EEF9060000D1FFDF694606F1120024
:104D400006F011FA060000D0FFDFA988172901D26A
:104D5000172200E00A46BDF80000824202D901464F
:104D600002E005E01729C5D3404600F047FCD0E734
:104D7000FFDF3046BDE8F883401D20F0030219B183
:104D800002FB01F0001D00E000201044704713B545
:104D9000009858B1002468460AF0E9FF002C04D1BD
:104DA000F749009A4A6000220A701CBD01240020C5
:104DB000F2E72DE9F0470C46154624220021204653
:104DC00008F003FB05B9FFDFA87860732888DFF8D7
:104DD000B0A3401D20F00301AF788946DAF8040043
:104DE0000AF0E3FF060000D1FFDF4FF00008266065
:104DF000A6F8008077B109FB07F1091D0AD0DAF89F
:104E000004000AF0D2FF060000D1FFDF6660C6F89A
:104E1000008001E0C4F80480298804F11200BDE894
:104E2000F04706F087B92DE9F047804601F11200FE
:104E30000D46814606F095F9401DD14F20F0030242
:104E40006E7B1446296878680AF0DAFF3EB104FBED
:104E500006F2121D03D0696878680AF0D1FF0520B8
:104E60000BF002F9044605200BF006F9201A012880
:104E700002D178680AF08EFF49464046BDE8F04707
:104E800006F06EB970B5054605210BF041F9040036
:104E900000D1FFDF04F112012846BDE8704006F0A2
:104EA00058B92DE9F04F91B04FF0000BADF828B094
:104EB000ADF804B047880C460546924605213846B1
:104EC0000BF026F9060000D1FFDF24B1A780A4F87B
:104ED00006B0A4F808B0297809220B20B2EB111F04
:104EE00073D12A7A04F1100138274FF00C084FF0E3
:104EF00012090291102A69D2DFE802F068F2F1F09B
:104F00008008D3898EA03DDCF3EEB7B7307B022852
:104F100000D0FFDFA88908EBC001ADF804103021F4
:104F2000ADF82810002C25D06081B5F80E80002740
:104F30001DE004EBC709317C89F80E10F189A9F84E
:104F40000C10CDF800806888042305AA296900F0B8
:104F500035FBBDF81410A9F8101008F10400BDF8D5
:104F600016107F1C1FFA80F8A9F81210BFB26089D2
:104F7000B842DED80CE1307B022800D0FFDFE9899F
:104F800008EBC100ADF804003020ADF8280095F81A
:104F90000C90002CA9F10400C0B20F90EAD06181FE
:104FA000B5F81080002725E0CDF8008068884B46D2
:104FB00003AA696900F002FB08EB09001FFA80F8F8
:104FC0006F48007818B1012302E0DDE0DAE0002349
:104FD00004EBC702009204A90C320F980CF023FED8
:104FE000009ABDF80C007F1C1082009ABDF80E00DC
:104FF000BFB250826089B842D6D8C9E00AA80090F2
:1050000001AB224629463046FFF711FBC0E0307B5A
:10501000082805D0FFDF03E0307B082800D0FFDF41
:10502000E8891030ADF804003620ADF82800002CD7
:105030003FD0A9896181F189A18127E0307B0928CE
:1050400000D0FFDFA88901460C30ADF804003720FE
:10505000ADF82800002C2CD06181E8890090AB8944
:10506000688804F10C02296955E0E889392110307B
:1050700080B2ADF80400ADF82810002C72D0A989D8
:105080006181287A0E280AD002212173E989E18101
:10509000288A0090EB8968886969029A3BE00121BF
:1050A000F3E70AA8009001AB224629463046FFF7F5
:1050B00055FB6DE0307B0A2800D0FFDFADF804908F
:1050C000ADF828704CB3A9896181A4F810B0A4F898
:1050D0000EB0012020735BE020E002E030E038E019
:1050E00041E0307B0B2800D0FFDF288AADF8287024
:1050F0001230ADF8040084B104212173A9896181C3
:10510000E989E181298A2182688A00902B8A68884E
:1051100004F11202696900F051FA39E0307B0C2881
:1051200000D0FFDFADF80490ADF828703CB3052146
:105130002173A4F80AB0A4F80EB0A4F810B027E0C8
:105140000AA8009001AB224629463046FFF754FAE0
:105150001EE00AA8009001AB224629463046FFF720
:10516000B3FB15E034E03B21ADF80400ADF82810A6
:1051700074B30120E080A4F808B084F80AB007E016
:1051800010000020FFDF03E0297A012917D0FFDF9C
:10519000BDF80400AAF800006CB1BDF8280020801A
:1051A000BDF804006080BDF82800392803D03C28F1
:1051B00001D086F80CB011B00020BDE8F08F3C2182
:1051C000ADF80400ADF8281014B1697AA172DFE7D8
:1051D000AAF80000EFE72DE9F84356880F4680460D
:1051E0001546052130460AF093FF040000D1FFDF89
:1051F000123400943B46414630466A6806F024F972
:10520000B8E570B50D4605210AF082FF040000D113
:10521000FFDF294604F11200BDE8704005F0AEBF83
:1052200070B50D4605210AF073FF040000D1FFDFC1
:10523000294604F11200BDE8704005F0CCBF70B5FE
:10524000054605210AF064FF040000D1FFDF04F1E8
:10525000080321462846BDE870400422AFE470B53B
:10526000054605210AF054FF040000D1FFDF214666
:1052700028462368BDE870400522A0E470B50646C4
:1052800005210AF045FF040000D1FFDF04F1120000
:1052900005F067FF401D20F0030511E0011D0088A7
:1052A0000322431821463046FFF789FC00280BD023
:1052B000607BABB2684382B26068011D0AF0F7FD03
:1052C000606841880029E9D170BD70B50E46054679
:1052D00002F010FF040000D1FFDF0120207266728F
:1052E0006580207820F00F00C01C20F0F0003030E6
:1052F0002070BDE8704002F001BF602801D0072097
:1053000070470878C54900F0010008700020704718
:105310002DE9F0438BB00D461446814606A9FFF7F0
:105320008AFB002814D14FF6FF7601274FF420584E
:105330008CB103208DF800001020ADF8100007A8F4
:10534000059007AA204604A90CF091FC78B107202B
:105350000BB0BDE8F0830820ADF808508DF80E7052
:105360008DF80000ADF80A60ADF80C800CE00698EE
:10537000A17801742188C1818DF80E70ADF80850B4
:10538000ADF80C80ADF80A606A4602214846069BDB
:10539000FFF77CFBDCE708B501228DF8022042F61E
:1053A0000202ADF800200A4603236946FFF731FCEC
:1053B00008BD08B501228DF8022042F60302ADF8BF
:1053C00000200A4604236946FFF723FC08BD00B508
:1053D00087B079B102228DF800200A88ADF8082044
:1053E0004988ADF80A1000236A460521FFF74EFBF5
:1053F00007B000BD1020FBE709B1072309E407202F
:10540000704770B588B00D461446064606A9FFF7EA
:1054100012FB00280ED17CB10620ADF808508DF8A3
:105420000000ADF80A40069B6A460821DC81304640
:10543000FFF72CFB08B070BD05208DF80000ADF81B
:105440000850F0E700B587B059B107238DF8003058
:10545000ADF80820039100236A460921FFF716FBE7
:10546000C6E71020C4E770B588B00C460646002594
:1054700006A9FFF7E0FA0028DCD1069801211230D6
:1054800005F0A1FE9CB12178062921D2DFE801F0C8
:10549000200505160318801E80B2C01EE28880B267
:1054A0000AB1A3681BB1824203D90C20C2E71020C5
:1054B000C0E7042904D0A08850B901E00620B9E76C
:1054C000012913D0022905D004291CD005292AD08E
:1054D0000720AFE709208DF800006088ADF80800CC
:1054E000E088ADF80A00A068039023E00A208DF858
:1054F00000006088ADF80800E088ADF80A00A068F8
:105500000A25039016E00B208DF800006088ADF8A6
:105510000800A088ADF80A00E088ADF80C00A0688B
:105520000B25049006E00C208DF8000060788DF8C3
:1055300008000C256A4629463046069BFFF7A6FA66
:1055400078E700B587B00D228DF80020ADF808107F
:1055500000236A461946FFF799FA49E700B587B074
:1055600071B102228DF800200A88ADF80820498820
:10557000ADF80A1000236A460621FFF787FA37E7DD
:10558000102035E770B586B0064601200D46ADF80F
:1055900008108DF80000014600236A463046FFF7E8
:1055A00075FA040008D12946304601F009FB0021B4
:1055B000304601F023FB204606B070BDF8B51C460E
:1055C00015460E46069F0AF0D6FE2346FF1DBCB2C6
:1055D00031462A4600940AF0D2FAF8BD30B411469A
:1055E000DDE902423CB1032903D0002330BC04F0C2
:1055F0001EBC0123FAE71A8030BC704770B50C4618
:105600000546FFF722FB2146284601F0E8FA284626
:10561000BDE87040012101F0F1BA00001000002047
:1056200018B18178012938D101E010207047018834
:1056300042F60112881A914231D018DC42F601027A
:10564000A1EB020091422AD00CDC41B3B1F5C05F5E
:1056500025D06FF4C050081821D0A0F57060FF3835
:105660001BD11CE001281AD002280AD117E0B0F59E
:10567000807F14D008DC012811D002280FD0032825
:105680000DD0FF2809D10AE0B0F5817F07D0A0F541
:105690008070033803D0012801D0002070470F200C
:1056A00070470A281FD008DC0A2818D2DFE800F06B
:1056B000191B1F1F171F231D1F21102815D008DCC1
:1056C0000B2812D00C2810D00D2816D00F2806D188
:1056D0000DE011280BD084280BD087280FD0032091
:1056E00070470020704705207047072070470F2043
:1056F000704704207047062070470C20704743F223
:105700000200704738B50C46050041D06946FEF7E7
:10571000C3FA002819D19DF80010607861F30200E7
:1057200060706946681CFEF7B7FA00280DD19DF835
:105730000010607861F3C5006070A978C1F3410181
:10574000012903D0022905D0072038BD217821F096
:10575000200102E0217841F020012170410704D0AE
:10576000A978C90861F386106070607810F0380F6E
:1057700007D0A978090961F3C710607010F0380FDD
:1057800002D16078400603D5207840F040002070B8
:10579000002038BD70B504460020088015466068BA
:1057A000FFF7B0FF002816D12089A189884211D8BF
:1057B00060688078C0070AD0B1F5007F0AD840F24F
:1057C0000120B1FBF0F200FB1210288007E0B1F5D8
:1057D000FF7F01D90C2070BD01F20121298000203A
:1057E00070BD10B50478137864F300031370047867
:1057F000640864F3410313700478A40864F382031B
:1058000013700478E40864F3C30313700478240964
:1058100064F3041313700478640964F3451313707C
:105820000078800960F38613137031B10878C107DE
:1058300001D1800701D5012000E0002060F3C713EB
:10584000137010BD4278530702D002F0070306E040
:1058500012F0380F02D0C2F3C20300E001234A78ED
:1058600063F302024A70407810F0380F02D0C0F3A0
:10587000C20005E0430702D000F0070000E001206D
:1058800060F3C5024A7070472DE9F04F95B00D00E6
:10589000824613D012220021284607F096FD4FF6CB
:1058A000FF7B05AA0121584607F057FB0024264636
:1058B00037464FF420586FF4205972E0102015B08D
:1058C000BDE8F08F9DF81E0001280AD1BDF81C101C
:1058D00041450BD011EB09000AD001280CD0022859
:1058E0000CD0042C0ED0052C0FD10DE0012400E0CB
:1058F0000224BDF81A6008E0032406E00424BDF881
:105900001A7002E0052400E00624BDF81A10514583
:1059100047D12C74BEB34FF0000810AA4FF0070A0D
:10592000CDE90282CDE900A80DF13C091023CDF8A4
:10593000109042463146584607F0DFFB08BBBDF8E1
:105940003C002A46C0B210A90CF08FF9C8B9AE814C
:10595000CFB1CDE900A80DF1080C0AAE40468CE8A5
:105960004102132300223946584607F0C6FB40B9CE
:10597000BDF83C00F11CC01EC0B22A1D0CF075F928
:1059800010B103209BE70AE0BDF82900E881062C4E
:1059900005D19DF81E00A872BDF81C0028810020CA
:1059A0008DE705A807F0E5FA00288BD0FFF779FE10
:1059B00085E72DE9F0471C46DDE90978DDF8209000
:1059C00015460E00824600D1FFDF0CB1208818B1C9
:1059D000D5B11120BDE8F087022D01D0012100E0F2
:1059E000002106F1140006F081F9A8F80000024633
:1059F0003B462946504603F086F9C9F8000008B92D
:105A0000A41C3C600020E5E71320E3E7F0B4144653
:105A1000DDE904528DB1002314B1022C09D101E05B
:105A2000012306E00D7CEE0703D025F001050123DC
:105A30000D742146F0BC04F0FAB91A80F0BC70472E
:105A40002DE9FE4F91461A881C468A468046FAB1D7
:105A500002AB494603F057F9050019D04046A61C91
:105A600027880AF09AFC3246072629463B460096CC
:105A70000AF0B9F820882346CDE900504A4651463D
:105A80004046FFF7C3FF002020800120BDE8FE8FC5
:105A90000020FBE72DE9F04786B082460EA890462D
:105AA00090E8B000894604AA05A903A88DE807007C
:105AB0001E462A4621465046FFF77BFF039901B157
:105AC00001213970002818D1FA4904F1140204ABFD
:105AD0000860039805998DE80700424649465046FC
:105AE00006F0B7FCA8B1092811D2DFE800F00508DC
:105AF0000510100A0C0C0E00002006B06AE71120F9
:105B0000FBE70720F9E70820F7E70D20F5E703207A
:105B1000F3E7BDF810100398CDE9000133462A469B
:105B200021465046FFF772FFE6E72DE9F04389B0C2
:105B30001646DDE910870D4681461C4614220021D9
:105B400003A807F042FC012002218DF810108DF807
:105B50000C008DF81170ADF8146064B1A278D20712
:105B600009D08DF81600E088ADF81A00A088ADF8CD
:105B70001800A068079008A80095CDE901104246DA
:105B800003A948466B68FFF785FF09B0BDE8F083BD
:105B9000F0B58BB0002406460694079407270894B6
:105BA00005A80994019400970294CDE903400D469D
:105BB00010232246304607F0A0FA78B90AA806A9B1
:105BC000019400970294CDE90310BDF8143000222F
:105BD0002946304607F02FF8002801D0FFF761FD75
:105BE0000BB0F0BD06F0C0BE2DE9FC410C4680466E
:105BF000002602F07FFA054620780D287ED2DFE8E5
:105C000000F0BC0713B325BD49496383AF959B00E2
:105C1000A848006820B1417841F010014170ADE022
:105C2000404602F099FAA9E0042140460AF070FAD1
:105C3000070000D1FFDF07F11401404605F0EBFF3C
:105C4000A5BB13214046FCF7B1FD97E00421404677
:105C50000AF05EFA070000D1FFDFE088ADF800002F
:105C60000020B8819DF80000010704D5C00602D5C8
:105C7000A088B88105E09DF8010040067ED5A08887
:105C8000F88105B9FFDF22462946404601F0C0FCF5
:105C9000022673E0E188ADF800109DF801100906B6
:105CA0000FD5072803D006280AD00AE024E00421F3
:105CB00040460AF02DFA060000D1FFDFA088F081EF
:105CC0000226CDB9FFDF17E0042140460AF020FA92
:105CD000070000D1FFDF07F1140006F07CFE90F012
:105CE000010F02D1E079000648D5387C022640F049
:105CF0000200387405B9FFDF224600E03DE0294686
:105D0000404601F085FC39E0042140460AF000FAE3
:105D1000017C002D01F00206C1F340016171017C9C
:105D200021F002010174E7D1FFDFE5E7022601213E
:105D3000404602F043FA21E0042140460AF0E8F927
:105D40000546606800902089ADF80400012269468C
:105D5000404602F054FA287C20F0020028740DE03E
:105D6000002DC9D1FFDFC7E7022600214046FFF71B
:105D700057FA002DC0D1FFDFBEE7FFDF3046BDE898
:105D8000FC813EB50C0009D001466B4601AA0020FB
:105D900007F038FA20B1FFF784FC3EBD10203EBD6D
:105DA00000202080A0709DF8050002A900F00700E7
:105DB000FDF78EFF50B99DF8080020709DF8050092
:105DC00002A9C0F3C200FDF783FF08B103203EBD66
:105DD0009DF8080060709DF80500C109A07861F386
:105DE0000410A0709DF80510890961F3C300A0702C
:105DF0009DF80410890601D5022100E0012161F31C
:105E000042009DF8001061F30000A07000203EBD2C
:105E100070B5144606460D4651EA040005D075B12A
:105E20000846FBF74CFA78B901E0072070BD294617
:105E3000304607F04EFA10B1BDE8704031E454B17D
:105E40002046FBF73CFA08B1102070BD21463046D1
:105E5000BDE8704095E7002070BD2DE9FC5F0C4661
:105E600090460546002701780822007A3E46B2EBAC
:105E7000111F7DD104F10A0100910A31821E4FF0F9
:105E8000020A04F1080B0191092A72D2DFE802F03C
:105E9000EDE005F528287BAACE00688804210AF0E9
:105EA00037F9060000D1FFDFB08928B15227072655
:105EB000C3E000003402002051271026002C7DD0C2
:105EC0006888A0800120A071A88900220099FFF7AE
:105ED0009FFF002873D1A8892081288AE081D1E022
:105EE000B5F81290072824D1E87B000621D5512768
:105EF00009F1140086B2002CE1D0A8890022009993
:105F0000FFF786FF00285AD16888A08084F806A091
:105F1000A88920810120A073288A2082A4F81290E9
:105F2000A88A009068884B46A969019A01F04CFB49
:105F3000A8E0502709F1120086B2002C3ED0A889B3
:105F400000225946FFF764FF002838D16888A080F6
:105F5000A889E080287A072813D002202073288A95
:105F6000E081E87BC0096073A4F81090A88A01E082
:105F700085E082E0009068884B4604F11202A9692E
:105F8000D4E70120EAE7B5F81290512709F114008F
:105F900086B2002C66D0688804210AF0B9F88346DE
:105FA0006888A080A88900220099FFF731FF0028A7
:105FB0006ED184F806A0A889208101E052E067E054
:105FC0000420A073288A2082A4F81290A88A009046
:105FD00068884B46A969019A01F0F6FAA989ABF8DD
:105FE0000E104FE06888FBF7A9FB0746688804217C
:105FF0000AF08EF8064607B9FFDF06B9FFDF687BB7
:10600000C00702D05127142601E0502712264CB3B6
:106010006888A080502F06D084F806A0287B5946B7
:1060200001F0E2FA2EE0287BA11DF9E7FE49A889DC
:106030004989814205D1542706269CB16888A080F1
:1060400020E053270BE06888A080A889E08019E051
:10605000688804210AF05CF800B9FFDF552708269C
:10606000002CF0D1A8F8006011E056270726002C7C
:10607000F8D06888A080002013E0FFDF02E001284C
:1060800008D0FFDFA8F800600CB1278066800020F0
:10609000BDE8FC9F57270726002CE3D06888A08026
:1060A000687AA071EEE7401D20F0030009B141437A
:1060B000091D01EB4000704713B5DB4A0020107149
:1060C000009848B10024684609F051FE002C02D126
:1060D000D64A009911601CBD01240020F4E770B578
:1060E0000D461446064686B05C220021284607F07D
:1060F0006CF904B9FFDFA0786874A278218828467B
:1061000001F09DFA0020A881E881228805F11401A0
:10611000304605F064FD6A460121304606F01DFF59
:106120001AE000BF9DF80300000715D5BDF8061062
:106130003046FFF72DFD9DF80300BDF8061040F036
:1061400010008DF80300BDF80300ADF81400FF2324
:106150003046059A07F085F8684606F00AFF0028E1
:10616000E0D006B070BD10B50C4601F1140005F08A
:106170006EFD0146627C2046BDE8104001F094BAF5
:1061800030B50446A84891B04FF6FF75C18905AAFD
:10619000284606F0E2FE30E09DF81E00A0422AD01C
:1061A00001282AD1BDF81C00B0F5205F03D042F6CB
:1061B0000101884221D1002002AB0AAA0CA901905A
:1061C00083E8070007200090BDF81A101023002272
:1061D000284606F092FF38B9BDF828000BAAC0B2D5
:1061E0000CA90BF042FD10B1032011B030BD9DF899
:1061F0002E00A04201D10020F7E705A806F0B9FE65
:106200000028C9D00520F0E770B50546042109F043
:106210007FFF040000D1FFDF04F114010C46284683
:1062200005F0F9FC21462846BDE8704005F0FABCAF
:1062300070B58AB00C460646FBF780FA050014D00C
:106240002878222827D30CB1A08890B101208DF89E
:106250000C0003208DF8100000208DF8110054B1BF
:10626000A088ADF81800206807E043F202000AB0E9
:1062700070BD0920FBE7ADF81800059004213046F9
:1062800009F046FF040000D1FFDF04F1140005F01F
:10629000F4FC000701D40820E9E701F02BFF60B10E
:1062A00008A802210094CDE9011095F8232003A944
:1062B00030466368FFF7EEFBD9E71120D7E72DE9F9
:1062C000F04FB2F802A0834689B015468946504681
:1062D000FBF734FA07460421504609F019FF00265F
:1062E000044605964FF002080696ADF81C6007B903
:1062F000FFDF04B9FFDF4146504603F0E2FE50B92C
:1063000007AA06A905A88DE807004246214650467F
:106310006368FFF74EFB444807AB0660DDE90512F2
:1063200004F11400CDF80090CDE90320CDE901314E
:1063300097F82320594650466B6805F0E7FC0600A5
:106340000AD0022E04D0032E14D0042E00D0FFDF7A
:1063500009B03046BDE8F08FBDF81C000028F7D02A
:106360000599CDE900104246214650466368FFF783
:106370004DFBEDE7687840F008006870E8E72DE92C
:10638000F04F99B004464FF000082748ADF81C8044
:10639000ADF82080ADF82480A0F80880ADF8148016
:1063A000ADF81880ADF82C80ADF82880007916463D
:1063B0000D464746012808D0022806D0032804D0FD
:1063C000042802D0082019B0C4E72046FAF733FFAA
:1063D00070BB2846FAF72FFF50BB6068FAF778FFCA
:1063E00030BB606848B160892189884202D8B1F524
:1063F000007F01D90C20E6E780460EAA06A92846B0
:10640000FFF7C8F90028DED168688078C0F3410042
:10641000022808D19DF8190010F0380F03D0286920
:10642000FAF74DFF20B904E03402002018000020E4
:1064300022E005A92069FFF765F90028C3D120698A
:1064400048B1607880079DF8150000F0380001D54C
:10645000F0B300E0E0BB9DF8140080060ED59DF877
:10646000150010F0380F03D06068FAF728FF18B94C
:106470006068FAF72DFF08B11020A4E70AA9606947
:10648000FFF740F900289ED1606940B19DF82900CE
:1064900000F0070101293CD110F0380F39D00BA9C9
:1064A000A069FFF72FF900288DD19DF828008006FC
:1064B0002FD49DF82C0080062BD4A06950B19DF8F4
:1064C0002D0000F00701012923D110F0380F00E062
:1064D0001FE01ED0E06818B10078D0B11C2818D297
:1064E0000FAA611C2046FFF77CF90121384661F3B1
:1064F0000F2082468DF85210B94642F603000F462F
:10650000ADF850000DF13F0218A928680BF0AFFB61
:1065100008B1072057E79DF8600015A9CDF8009055
:10652000C01CCDE9019100F0FF0B00230BF201220A
:10653000514614A806F03CFCF0BBBDF854000C908A
:10654000FE482A8929690092CDE901106B89BDF8BE
:1065500038202868069906F02BFC01007ED12078AF
:106560004FF0020AC10601D480062BD5CDF80C905D
:10657000606950B90AA906A8FFF764F99DF82900D7
:1065800020F00700401C8DF829009DF8280008A97C
:1065900040F0C8008DF828008DF8527042F60210C5
:1065A000ADF8500003AACDF800A0CDE901210023E9
:1065B00040F2032214A800E01EE00A9906F0F8FB5E
:1065C00001004BD1DD484D4608385B460089ADF8E7
:1065D0003D000FA8CDE90290CDF80490CDF81090C1
:1065E0004FF007090022CDF80090BDF854104FF687
:1065F000FF7006F020FB10B1FFF753F8E3E69DF8BB
:106600003C00000624D52946012060F30F218DF8B7
:1066100052704FF424500395ADF8500062789DF805
:106620000C00002362F300008DF80C006278CDF8B6
:1066300000A0520862F341008DF80C0003AACDE9D6
:10664000012540F2032214A806F0B2FB010005D197
:10665000606888B32069A8B905A900E084E006A8AD
:10666000FFF7F0F86078800706D49DF8150020F059
:1066700038008DF8150005E09DF8140040F040004A
:106680008DF814008DF8527042F60110ADF85000EC
:10669000208940F20121B0FBF1F201FB1202606897
:1066A00009ABCDF80080CDE90103002314A80599BA
:1066B00006F07EFB010057D12078C00728D0039553
:1066C000A06950B90BA906A8FFF7BCF89DF82D00EA
:1066D00020F00700401C8DF82D009DF82C008DF84F
:1066E000527040F040008DF82C0042F60310ADF8D7
:1066F000500007A903AACDF800A0CDE9012100238D
:1067000040F2032214A80B9906F052FB01002BD192
:10671000E06868B32946012060F30F218DF85270BC
:1067200042F60410ADF85000E068002302788DF8BE
:10673000582040788DF85900E06816AA4088ADF8D6
:106740005A00E06800798DF85C00E068C088ADF818
:106750005D00CDF80090CDE901254FF4027214A838
:1067600006F026FB010003D00C9800F0C9FF2AE6D2
:10677000724803210838017156B100893080BDF894
:1067800024007080BDF82000B080BDF81C00F080AF
:10679000002018E670B501258AB016460B46012880
:1067A00002D0022816D104E08DF80E504FF420508C
:1067B00003E08DF80E5042F60100ADF80C005BB11D
:1067C0000024601C60F30F2404AA08A918460BF0EB
:1067D0004EFA18B107204AE5102048E504A99DF8B3
:1067E00020205648CDE90021801E0290002321463A
:1067F00003A802F2012206F0DBFA10B1FEF751FF06
:1068000035E54E4808380EB1C18831800571002049
:106810002DE5F0B593B0074601268DF83E6041F6B0
:106820000100ADF83C0012AA0FA93046FFF7B2FFF5
:10683000002849D1414C0025083CEFB31C2200211F
:1068400002A806F0C2FD9DF808008DF83E6040F0F9
:1068500020008DF8080042F60520ADF83C000E95AA
:106860009DF83A00119520F00600801C8DF83A0042
:106870009DF838006A4620F0FF008DF838009DF83A
:10688000390009A920F0FF008DF839000420ADF887
:106890002C00ADF830000EA80A9011A80D900FA89A
:1068A0000990ADF82E5002A8FFF769FD00280BD122
:1068B000BDF80000608100E008E0BDF80400A081A0
:1068C000401CE0812571002013B0F0BD6581A581D9
:1068D000BDF84800F4E72DE9F74F1849A0B00024AF
:1068E000083917940A79A146012A04D0022A02D055
:1068F000082023B02EE5CA88824201D00620F8E79E
:1069000021988A46824201D10720F2E701202146E0
:1069100060F30F21ADF848004FF6FF780691ADF80F
:106920004A808DF86E0042F6020B8DF872401CA969
:10693000ADF86CB0ADF87040139101E03C0200205E
:10694000ADF8508012A806F043FB00252E462F46D6
:106950000DAB072212A9404606F03DFB78B10A288C
:106960005DD195B38EB3ADF86450ADF866609DF817
:106970005E008DF8144019AC012864D06BE09DF8DE
:106980003A001FB3012859D1BDF8381059451FD11D
:1069900018A809A901940294CDE9031007200090DA
:1069A000BDF8361010230022404606F0A6FBB0BB0F
:1069B000BDF86000042801D006284AD1BDF8241093
:1069C000219881423AD10F2093E73AE0012835D14E
:1069D000BDF83800B0F5205F03D042F601018842CF
:1069E0002CD1BAF80600BDF83610884201D1012733
:1069F00000E0002705B19EB1219881421ED118A860
:106A000009AA01940294CDE90320072000900D46C5
:106A100010230022404606F070FB00B902E02DE092
:106A20004E460BE0BDF86000022801D0102810D1BE
:106A3000C0B217AA09A90BF018F950B9BDF83690E1
:106A400086E7052055E705A917A8221D0BF00FF9C9
:106A500008B103204DE79DF814000023001DC2B2C9
:106A60008DF8142022980092CDE901401BA80699C8
:106A700006F09EF910B902228AF80420FEF711FEF2
:106A800037E710B50B46401E88B084B205AA002136
:106A90001846FEF7A6FE00200DF1080C06AA05A96F
:106AA00001908CE807000720009001230022214676
:106AB0004FF6FF7006F0BFF80446BDF81800012835
:106AC00000D0FFDF2046FEF7ECFD08B010BDF0B5AA
:106AD000F74F044687B038790E46032804D00428BF
:106AE00002D0082007B0F0BD04AA03A92046FEF793
:106AF00051FE0500F6D160688078C0F3410002289D
:106B00000AD19DF80D0010F0380F05D02069FAF772
:106B1000D6FB08B11020E5E7208905AA21698DE898
:106B200007006389BDF810202068039906F040F93A
:106B300010B1FEF7B6FDD5E716B1BDF814003080F0
:106B4000042038712846CDE7F8B50C0006460CD075
:106B500001464FF6FF7500236A46284606F052FBB1
:106B600028B100BFFEF79DFDF8BD1020F8BD6946B5
:106B70002046FEF7C7FD0028F8D1A078314600F086
:106B800001032846009A06F06CFBEBE730B587B0AE
:106B9000144600220DF1080C05AD01928CE82C0082
:106BA000072200920A46014623884FF6FF7006F03E
:106BB00042F8BDF814102180FEF773FD07B030BD18
:106BC00070B50D46042109F0A3FA040000D1FFDFDF
:106BD000294604F11400BDE8704005F047B870B5CF
:106BE0000D46042109F094FA040000D1FFDF294684
:106BF00004F11400BDE8704005F05BB870B50D46B7
:106C0000042109F085FA040000D1FFDF294604F1D0
:106C10001400BDE8704005F073B870B50546042156
:106C200009F076FA040000D1FFDF214628462368E8
:106C3000BDE870400122FEF703BF70B5064604218F
:106C400009F066FA040000D1FFDF04F1140004F03B
:106C5000FEFF401D20F0030511E0011D0088002209
:106C6000431821463046FEF7EBFE00280BD0607C2F
:106C7000ABB2684382B2A068011D09F018F9A068A0
:106C800041880029E9D170BD70B50546042109F09D
:106C90003FFA040000D1FFDF214628466368BDE8C3
:106CA00070400222FEF7CCBE70B50E46054601F0DC
:106CB00021FA040000D1FFDF012020726672658096
:106CC000207820F00F00001D20F0F00040302070F0
:106CD000BDE8704001F012BA10B50446012900D099
:106CE000FFDF2046BDE810400121FEF799BA2DE9EB
:106CF000F04F97B04FF0000A0C008346ADF814A097
:106D0000D04619D0E06830B1A068A8B10188ADF8CC
:106D10001410A0F800A05846FAF710FD070043F23F
:106D2000020961D0387822285CD30421584609F042
:106D3000EFF9050005D103E0102017B0BDE8F08F92
:106D4000FFDF05F1140004F082FF401D20F0030670
:106D5000A078012803D0022801D00720EDE7218880
:106D600007AA584606F0F9F830BB07A806F001F963
:106D700010BB07A806F0FDF848B99DF826000128C9
:106D800005D1BDF82400A0F52451023902D04FF4FA
:106D90005050D2E7E068B0B1CDE902A007200090E2
:106DA00005AACDF804A00492A2882188BDF8143069
:106DB000584605F040FF10B1FEF773FCBDE7A1682F
:106DC000BDF8140008809DF81F00C00602D543F2EC
:106DD0000140B2E70B9838B1A1780078012905D0BD
:106DE00080071AD40820A8E74846A6E7C007F9D0CC
:106DF00002208DF83C00A8684FF00009A0B1697C22
:106E00004288714391420FD98AB2B3B2011D09F091
:106E100004F88046A0F800A006E003208DF83C00AE
:106E2000D5F800804FF001099DF8200010F0380FD0
:106E300000D1FFDF9DF820001E49C0F3C2000844C6
:106E400097F8231010F8010C884201D90F2074E73D
:106E50002088ADF8400014A90095CDE90191434682
:106E600007220FA95846FEF715FE002891D19DF87C
:106E7000500050B9A078012807D1687CB3B27043A4
:106E800082B2A868011D08F0DCFF002055E770B54C
:106E9000064615460C460846FEF7C2FB002805D1FB
:106EA0002A4621463046BDE8704073E470BD12E5C5
:106EB00034020020A2B1010070B51E4614460D0038
:106EC00009D044B1616831B138B1FC49C988814207
:106ED00003D0072070BD102070BD2068FEF7A0FB16
:106EE0000028F9D1324621462846BDE87040FFF718
:106EF00046BA70B515460C0006D038B1EF4909897D
:106F0000814203D0072070BD102070BD2068FEF7BD
:106F100087FB0028F9D129462046BDE87040D6E518
:106F200070B5064686B00D4614461046FAF7A9F924
:106F3000D0BB6068FAF7CCF9B0BBA6F57F40FF384C
:106F400003D03046FAF7FAFB80B128466946FEF7CF
:106F50009BFC00280CD19DF810100F2008293DD271
:106F6000DFE801F008060606060A0A0843F20200F6
:106F700006B070BD0320FBE79DF80210012908D17F
:106F8000BDF80010B1F5C05FF2D06FF4C052D1422D
:106F9000EED09DF8061001290DD1BDF80410A1F521
:106FA0002851062907D200E029E0DFE801F00303B9
:106FB00004030303DCE79DF80A1001290FD1BDF893
:106FC0000810B1F5245FD3D0A1F60211B1F500513C
:106FD000CED00129CCD0022901D1C9E7FFDF6068FA
:106FE00078B9002305AA2946304606F00BF910B1FE
:106FF000FEF757FBBCE79DF81400800601D4102073
:10700000B6E76188224628466368FFF7BFFDAFE711
:107010002DE9F043814687B0884614461046FAF7BA
:1070200030F918B1102007B0BDE8F083002306AA9C
:107030004146484606F0E6F818B100BFFEF731FBBE
:10704000F1E79DF81800C00602D543F20140EAE7D7
:107050000025072705A8019500970295CDE9035063
:1070600062884FF6FF734146484606F046F8060030
:1070700013D16068FAF705F960B960680195CDE948
:10708000025000970495238862884146484606F0DE
:1070900034F80646BDF8140020803046CEE739B1FA
:1070A000864B0A889B899A4202D843F203007047B4
:1070B0001DE610B586B0814C0423ADF81430638909
:1070C00043B1A4898C4201D2914205D943F2030015
:1070D00006B010BD0620FBE7ADF8101000210091AE
:1070E0000191ADF8003002218DF8021005A902913E
:1070F00004A90391ADF812206946FFF7F8FDE7E710
:107100002DE9FC4781460D460846FAF794F888BBFE
:107110004846FAF713FB5FEA00080AD098F8000027
:10712000222829D30421484608F0F2FF070005D1A0
:1071300003E043F20200BDE8FC87FFDF07F1140023
:1071400004F09BFD06462878012803D0022804D0CD
:107150000720F0E7B0070FD502E016F01C0F0BD0A8
:10716000A8792C1DC00709D0E08838B1A068FAF7CB
:1071700062F818B11020DEE70820DCE721882A78C1
:107180000720B1F5847F35D01EDC40F20315A1F253
:107190000313A94226D00EDCB1F5807FCBD003DCEF
:1071A000F9B1012926D1C6E7A1F58073013BC2D010
:1071B000012B1FD113E0012BBDD0022B1AD0032BC2
:1071C000B9D0042B16D112E0A1F20912082A11D26B
:1071D000DFE802F00B04041010101004ABE7022AE1
:1071E000A9D007E0012AA6D004E0320700E0F206A9
:1071F000002AA0DACDB200F07DFF50B198F823004C
:10720000CDE90005FA89234639464846FEF78DFC4C
:1072100091E711208FE72DE9F04F8BB01F461546FF
:107220000C4683460026FAF789FA28B1007822280E
:1072300005D208200BB081E543F20200FAE7B80856
:1072400001D00720F6E7032F00D100274FF6FF7982
:10725000CCB1022D73D32046FAF73AF830B904EBDB
:107260000508A8F10100FAF733F808B11020E1E7AA
:10727000AD1E38F8028CAAB22146484606F015F930
:1072800040455CD1ADB20D49B80702D58889401C94
:1072900000E001201FFA80F8F80701D08F8900E094
:1072A0004F4605AA4146584605F057FE4FF0070ADB
:1072B0004FF00009DCB320460BE000003402002050
:1072C000408810283BD8361D304486B2AE4236D2B4
:1072D000A01902884245F3D351E000BF9DF8170082
:1072E00002074CD594B304EB0608361DB8F80230FB
:1072F000B6B2102B23D89A19AA4220D8B8F8002089
:1073000091421CD1C0061CD5CDE900A90DF1080C95
:107310000AAAA11948468CE80700B8F80010002214
:10732000584605F088FC20B1FEF7BBF982E726E05D
:1073300005E0B8F80200BDF82810884201D00B2003
:1073400078E7B8F80200304486B207E0FFE7C006ED
:1073500004D55846FEF71CFC002888D19DF817007C
:10736000BDF81A1020F010008DF81700BDF81700B6
:10737000ADF80000FF235846009A05F072FF05A8FB
:1073800005F0F7FD18B9BDF81A10B942A6D90421C5
:10739000584608F0BDFE040000D1FFDFA2895AB1B3
:1073A000CDE900A94D46002321465846FEF7BDFB16
:1073B0000028BBD1A5813DE700203BE72DE9FF4F29
:1073C0008BB01E4617000D464FF0000412D0B008D7
:1073D00002D007200FB0B1E4032E00D100265DB12A
:1073E0000846F9F76CFF28B93888691E0844F9F790
:1073F00066FF08B11020EDE7C74AB00701D5D18973
:1074000000E00121F0074FF6FF7802D0D089401E3E
:1074100000E0404686B206AA0B9805F09EFD4FF0AC
:1074200000094FF0070B0DF1140A38E09DF81B001E
:10743000000734D5CDF80490CDF800B0CDF8089011
:10744000CDE9039A434600220B9805F056FE60BB37
:1074500005B3BDF814103A8821442819091D8A4241
:1074600030D3BDF81E2020F8022BBDF8142020F8E0
:10747000022BCDE900B9CDE90290CDF810A0BDF8FE
:107480001E10BDF8143000220B9805F036FE08B12E
:1074900003209FE7BDF814002044001D84B206A815
:1074A00005F067FD20B10A2806D0FEF7FAF891E74B
:1074B000BDF81E10B142B9D934B17DB13888A11CD4
:1074C000884203D20C2085E7052083E7224629461F
:1074D000404605F0EAFF014628190180A41C3C80C3
:1074E000002077E710B50446F9F7CBFE08B110206D
:1074F00010BD8948C0892080002010BDF0B58BB038
:107500000D4606461422002103A805F05EFF012067
:107510008DF80C008DF8100000208DF81100ADF8EA
:1075200014503046FAF70AF948B10078222812D3ED
:107530000421304608F0ECFD040005D103E043F2DD
:1075400002000BB0F0BDFFDF04F11400074604F0A9
:1075500094FB800601D40820F3E7207C022140F050
:107560000100207409A80094CDE90110072203A9A5
:1075700030466368FEF78EFA20B1217C21F00101CC
:107580002174DEE729463046FDF73BFE08A9384660
:1075900004F062FB00B1FFDFBDF82040172C01D2E0
:1075A000172000E02046A84201D92C4602E0172C03
:1075B00000D2172421463046FFF711FB2146304602
:1075C000FDF743FB0020BCE7F8B51C4615460E4608
:1075D000069F08F0D0FE2346FF1DBCB231462A4666
:1075E000009408F0CCFAF8BD70B50C4605460E22A2
:1075F0000021204605F0E9FE002020802DB1012D5C
:1076000001D0FFDF70BD062000E00520A07170BD35
:1076100010B548800878134620F00F00001D20F0B8
:10762000F00080300C4608701422194604F108005E
:1076300005F0A1FE00F062FD3748046010BD2DE9A1
:10764000F047DFF8D890491D064621F003011746A0
:107650000C46D9F8000008F0A8FB050000D1FFDFB8
:107660004FF000083560A5F800802146D9F80000E9
:1076700008F09BFB050000D1FFDF7560A5F80080D6
:107680007FB104FB07F1091D0BD0D9F8000008F009
:107690008CFB040000D1FFDFB460C4F80080BDE8BB
:1076A000F087C6F80880FAE72DE9F0411746491D32
:1076B00021F00302194D064601681446286808F0B7
:1076C0009FFB22467168286808F09AFB3FB104FBD3
:1076D00007F2121D03D0B168286808F091FB04205E
:1076E00008F0C2FC0446042008F0C6FC201A012859
:1076F00004D12868BDE8F04108F04CBBBDE8F0813A
:1077000010B50C4605F0F8FB00B1FFDF2046BDE8E0
:107710001040FDF7C6BF0000340200201800002012
:107720004FF0E0214FF40040C1F88001BFF34F8FCC
:10773000BFF36F8F00F021B810B5044600F01DF8BC
:10774000002C09D0124A124812491432124B012C53
:1077500003D0022C07D0FFDF10BD022404601160AB
:107760004FF0407004E00324046011604FF4000007
:10777000186010BD00B5FFDF00BD054800210160A5
:10778000016005494FF06070091D086070470000F6
:1077900000F500404402002004F501402DE9F05FAF
:1077A000DFF850A44FF000088B4606469AF80940CF
:1077B000474645469AF8019008E0284601F017F838
:1077C000817B407811FB00776D1CEDB24D45F4D103
:1077D0009AF809002044204420440744FF2F01D98F
:1077E0004FF013083068C01C20F0030232605BEADF
:1077F000080021D1FF48FBB2062120300CF0E0F94F
:10780000002408E0062C0FD2DFE804F005030A0A82
:107810000C05F94800E0F9480CF0F2F9054604E0DF
:10782000F748F9E7F748F7E7FFDFA54200D0FFDFA9
:10783000641CE4B2062CE5D3306800EB071030601E
:107840004046BDE8F09F38B50C468288817B19B16F
:107850004189914200D90A462280C188121D90B206
:107860006A4607F091FCBDF80000032800D303200E
:10787000C1B2208800F0DAFF38BD38B50C468288E6
:10788000817B19B10189914200D90A462280C188C1
:10789000121D90B26A4607F077FCBDF8000002287E
:1078A00000D30220C1B2208800F0C0FF401CC0B24B
:1078B00038BD2DE9FF5F82468B46D34814460BF155
:1078C0000302D0E90110CDE9021022F0030201A861
:1078D0004421019208F04BFAC64E002C02D1CB494C
:1078E000019A8A60019901440191B57E05F1010573
:1078F00004D1E8B20AF03CF900B1FFDF019800EBD7
:107900000510C01C20F00301019144B9727A0020D7
:107910000870B08B80B205F04EF900B1FFDF01981E
:10792000F16908440190214601A8FFF737FF80461E
:107930000198C01C20F003000190717A04B100206E
:1079400008F00BFB019908440190214601A800F0C2
:107950007FFFA84800273D4690F801900CE028469C
:1079600000F045FF064681788088FDF705FA7178BA
:107970006D1C00FB0177EDB24D45F0D10198C01CA4
:1079800020F00300019004B100203946FDF7FFF913
:10799000019900270844019096483D4690F80190CF
:1079A0000CE0284600F023FF0646C1788088FEF7E9
:1079B0007AFB71786D1C00FB0177EDB24D45F0D17B
:1079C0000198C01C20F00300019004B1002039464A
:1079D000FEF772FB01994FF00009084401908548B9
:1079E0004D4647780EE0284600F001FF0646807BB2
:1079F00030B106F1080002F0A5F8727800FB029998
:107A00006D1CEDB2BD42EED10198C01C20F0030008
:107A1000019004B100207D494A78494602F096F869
:107A2000019908440190214601A800F0BCFE01988C
:107A3000C01D20F007000190DAF80010814204D345
:107A4000A0EB0B01B1F5803F04DB4FF00408CAF84E
:107A5000000004E0CAF80000B8F1000F02D0404670
:107A600004B0EEE674BB6A490020019A0CF016FAE5
:107A7000FAF770FB5F4C207E0090607E012823D0D7
:107A8000002318B300225B4800210C30FBF73CF8C0
:107A900000B1FFDFE07EFEF7BCFE00B1FFDF55481E
:107AA0004FF4F6720021383005F08FFC5148042164
:107AB000383080F8E91180F8EA11062180F8EB11DE
:107AC000032101710020CBE70123DAE702AADAE7FC
:107AD00070B5484C06463834207804EB4015E07801
:107AE000083598B9A01990F8E80100280FD0A078BF
:107AF0000F2800D3FFDF20220021284605F065FC77
:107B0000687866F3020068700120E070284670BD56
:107B10002DE9F04105460C460027007805219046E6
:107B20003E46B1EB101F00D0FFDF287A50B101288C
:107B30000ED0FFDFA8F800600CB12780668000201F
:107B4000BDE8F0810127092674B16888A08008E0AB
:107B50000227142644B16888A0802869E060A88ABA
:107B60002082287B2072E5E7A8F80060E7E730B5BF
:107B7000204C0120002120706170207260726176BB
:107B8000217621730521A1821F21E182607321A149
:107B900021610A21A176E0761C4D4FF4B060E061CE
:107BA0006868C11C21F00301814200D0FFDF6868D2
:107BB000606030BD30B5154C1568636810339D4268
:107BC00002D20420136030BD0A4B5D785A6802EB84
:107BD0000512107051700320D08017209080012072
:107BE000D0709070002090735878401C5870606876
:107BF000103013E050030020A11F00006D9C000016
:107C0000E92F000063190100A8B101001C00002049
:107C1000000000206E5246357800000060600020B1
:107C200030BD70B50646F8480024457807E0204688
:107C300000F0DDFD0178B14204D0641CE4B2AC4236
:107C4000F5D1002070BDF7B5074608780C4610B393
:107C5000FFF7E7FF0546A7F12006202F06D0052EE7
:107C600019D2DFE806F00F2B2B151A0000F0CBFD20
:107C70000DB1697800E00021401AA17880B2084473
:107C8000FF2808D8A07830B1A088022824D202E0CA
:107C90006088172820D20720FEBD207AE0B16188D5
:107CA0001729F8D3A1881729F5D3A1790029F2D093
:107CB000E1790029EFD0402804D9ECE7242F0BD13B
:107CC000207A48B161884FF6FB70814202D8A188C2
:107CD000814201D90420FEBD65B9207802AA0121A4
:107CE000FFF768FF0028F6D12078FFF79AFF05001C
:107CF00000D1FFDF052E18D2DFE806F0030B0E08D7
:107D00001100A0786870A088E8800FE06088A880E3
:107D10000CE0A078A87009E0A078E87006E054F8BC
:107D2000020FA8606068E86000E0FFDF0020FEBD91
:107D30001A2835D00DDC132832D2DFE800F01B31D1
:107D4000203131272723252D313129313131312F70
:107D50000F00302802D003DC1E2821D107207047F5
:107D60003A3809281CD2DFE800F0151B0F1B1B1B3B
:107D70001B1B07000020704743F20400704743F2CA
:107D800002007047042070470D2070470F20704795
:107D90000820704711207047132070470620704755
:107DA0000320704710B5007800F0010007F0E2F9F9
:107DB000BDE81040BCE710B5007800F0010007F006
:107DC000DEF9BDE81040B3E70EB5017801F001011E
:107DD0008DF80010417801F001018DF80110017853
:107DE000C1F340018DF802104178C1F340018DF8D4
:107DF0000310017889088DF80410417889088DF8FE
:107E0000051081788DF80610C1788DF8071000797B
:107E10008DF80800684606F06EFEFFF789FF0EBD7C
:107E20002DE9F84F784CDFF8E481383400261FE064
:107E3000012000F050FD0120FFF74AFE05464421D5
:107E40004746D8F8080007F0B0FF686000B9FFDFC8
:107E5000686806F049FDA8B12846F9F7DDFD284617
:107E600000F03FFD20B944226968B86807F0C8FFF8
:107E700094F9E9010428DBDA022008F0F5F8074656
:107E80000025A6E044226968D8F8080007F0B8FF8A
:107E9000F2E7B8F802104046491C89B2A8F802106F
:107EA000B94201D3002141800221B8F8020008F054
:107EB0002FF9002865D0B8F80200694607F0D8F815
:107EC000FFF736FF00B1FFDF9DF8000078B1B8F88A
:107ED000020008F062FA5FEA000900D1FFDF4846BD
:107EE00007F0E1FC18B1B8F8020002F0D8F8B8F8D1
:107EF000020008F040FA5FEA000900D1FFDF4846BF
:107F000007F0C9FCE8BB0321B8F8020008F000F94B
:107F10005FEA000B48D1FFDF46E000BFDBF810004E
:107F200010B10078FF2849D0022000F0D4FC0220D4
:107F3000FFF7CEFD8246484607F0B9FDCAF80400B7
:107F400000B9FFDFDAF8040007F081FE002100909D
:107F50000170B8F802105046AAF8021001F0C2FFF2
:107F6000484607F076FE00B9FFDF504600F0B9FC46
:107F700018B99AF80100000704D50099CBF8101041
:107F800012E024E0DBF8100038B10178491C11F050
:107F9000FF01017008D1FFDF06E0002211464846CC
:107FA00000F0FFFB00B9FFDF94F9EA01022805DBCE
:107FB000B8F8020001F05DFF0028AFD194F9E901A3
:107FC000042804DB484607F0A8FE00B101266D1C1A
:107FD000EDB2BD4204D294F9EA010228BFF659AFCE
:107FE000002E7FF423AFBDE8F84F032000F073BCF0
:107FF00010B5064CE06008682061AFF2DB1002F0BB
:10800000D0FF607010BD0000500300201C00002055
:10801000F74800210170F7480170F7494160704747
:1080200070B505464FF080500C46D0F8A410491C9E
:1080300005D1D0F8A810C9430904090C0BD050F899
:10804000A01F01F001012970416821608068A080B3
:10805000287830B970BD062120460BF0A4FB012022
:108060002870607940F0C000607170BD70B54FF04D
:1080700080540D46D4F88010491C0BD1D4F88410DC
:10808000491C07D1D4F88810491C03D1D4F88C10AE
:10809000491C0CD0D4F880100160D4F884104160E1
:1080A000D4F888108160D4F88C10C16002E01021EF
:1080B0000BF079FBD4F89000401C0BD1D4F894005D
:1080C000401C07D1D4F89800401C03D1D4F89C0080
:1080D000401C09D054F8900F286060686860A06860
:1080E000A860E068E86070BD2846BDE870401021D7
:1080F0000BF059BBBE4838300079E9E470B5BC4C90
:108100003834E07830B3207804EB4010407A00F047
:108110000700204490F9E801002800DCFFDF207808
:10812000002504EB4010407A00F00700011991F897
:10813000E801401E81F8E8012078401CC0B22070A0
:108140000F2800D12570A078401CA0700BF0AAF970
:10815000E57070BDFFDF70BD3EB50546032107F039
:10816000D7FF0446284608F006F9054604B9FFDFA4
:10817000206918B10078FF2800D1FFDF01AA694605
:10818000284600F00EFB60B9FFDF0AE0002202A9DA
:10819000284600F006FB00B9FFDF9DF8080000B19B
:1081A000FFDF9DF80000411E8DF80010EED220691F
:1081B0000199884201D1002020613EBD70B505467D
:1081C000A0F57F400C46FF3800D1FFDF012C01D025
:1081D000FFDF70BDFFF78EFF040000D1FFDF2078C6
:1081E00020F00F00401D20F0F0005030207065801E
:1081F0000020207201202073BDE870407EE72DE949
:10820000F04116460D460746FFF774FF040000D103
:10821000FFDF207820F00F00401D20F0F0005030EC
:10822000207067800120207228682061A888A082C1
:108230002673BDE8F04161E77FB5FFF7F2FC04006B
:1082400000D1FFDF02A92046FFF7FDFA054603A98A
:108250002046FFF712FB8DF800508DF80100BDF8A5
:108260000800001DADF80200BDF80C00001DADF8BF
:108270000400E088ADF80600684606F063FF0028B9
:1082800000D0FFDF7FBD2DE9F05F5A4E8146307888
:1082900010B10820BDE8F09F4846F8F7F2FF08B19A
:1082A0001020F7E7524C207808B9FFF760FC647A99
:1082B0004D4600F0A8FAA04207D2201AC1B22A46C1
:1082C0000020FFF777FC0028E4D171684848C91CFA
:1082D000002721F003017160B3463E463D46BA4691
:1082E0003C4690F801800AE0204600F080FA417890
:1082F000807B0E4410FB0155641CE4B27F1C444596
:10830000F2D10AEB870000EBC600DBF8041000EBAB
:10831000850045185C46012229464846FFF7C9FA00
:10832000060013D00020FFF77CFC05000CD005F1FF
:108330001300616820F00300884200D0FFDF2C4862
:108340004178491E417065603046A3E70022294606
:108350004846FFF7AEFA00B1FFDFD9F800006060D1
:108360004FF6FF70608001202070002092E72DE919
:10837000F04104461F4817460E46007810B1082009
:10838000BDE8F0810846F8F756FF08B11020F7E77E
:10839000174D287808B9FFF7EAFB601E1E2807D89A
:1083A000012C22D13078FE281FD8A8760020E7E7DC
:1083B000A4F120001F2805D8E0B23A463146BDE8B6
:1083C000F04140E4A4F140001F2805D83146204682
:1083D000BDE8F04100F0ACBAA4F1A0001F2804D819
:1083E0000020A02C0AD0A12C0DD00720C8E7000047
:1083F000500300201C00002048100020317801F0BC
:108400000101E976BCE731680922F82901D38B071D
:1084100001D01046B4E76B7B03F00303012B04D1BA
:10842000EB8AD7339CB28C42F3D8E961A8E72DE9F7
:10843000F04781460E460846F8F723FF48B94846FC
:10844000F8F73DFF28B909F1030020F00301494581
:1084500002D01020BDE8F087FA484FF0000A81787A
:1084600069B14178804600EB4114083437883246C0
:108470000021204600F043FA050004D027E0A6F8CA
:1084800000A00520E6E7B9F1000F24D03088B842FB
:1084900001D90C251FE0607800F00705284600F0A0
:1084A0001AFA08EB0507324697F8E8014946401CDE
:1084B00087F8E801204607F5F47700F020FA054632
:1084C0003878401E3870032000F005FA2DB10C2DCD
:1084D00001D0A6F800A02846BCE76078DA4E00F08C
:1084E0000701012923D002290CD0032933D0FFDF53
:1084F00098F801104046491CC9B288F801100F29AC
:1085000034D035E0616821B1000702D46088FFF7FC
:1085100023FE98F8EA014746012802D1707802F05C
:108520005FFD97F9EA010428E2DBFFDFE0E761681D
:1085300019B14422B06807F063FC98F8E901474696
:10854000032802D1707802F04BFD97F9E901042865
:10855000CEDBFFDFCCE7C00602D56088FFF7FCFD6D
:1085600098F9EB010628C3DBFFDFC1E780F801A023
:108570008178491E8170617801F0070101EB0800E4
:1085800090F8E811491C80F8E811A4E770B50C4692
:108590000546F8F750FE18B92046F8F772FE08B104
:1085A000102070BD284609F01AFB207008B1002089
:1085B00070BD042070BD70B5054609F029FBC4B23A
:1085C0002846F8F77CFE08B1102070BD35B1287838
:1085D0002C7018B1A04201D0072070BD2046FDF7D5
:1085E000CFFD052805D109F016FB012801D0002098
:1085F00070BD0F2070BD70B5044615460E46084686
:10860000F8F719FE18B92846F8F73BFE08B1102014
:1086100070BD022C03D0102C01D0092070BD2A4659
:108620003146204609F021FB0028F7D0052070BD17
:1086300070B514460D460646F8F7FDFD38B92846D4
:10864000F8F71FFE18B92046F8F739FE08B11020D8
:1086500070BD22462946304609F009FB0028F7D0B4
:10866000072070BD3EB50446F8F70BFE08B1102098
:108670003EBD684606F0CBF9FFF75AFB0028F7D15C
:108680009DF806002070BDF808006080BDF80A0063
:10869000A08000203EBD70B505460C460846F8F7A0
:1086A0000EFE20B93CB12068F8F7EBFD08B11020B0
:1086B00070BDA08828B121462846BDE87040FDF76E
:1086C000B7BD092070BD70B504460D460846F8F7E1
:1086D000B2FD90BB601E1E280ED8032C01D90720C6
:1086E00070BD04B9FFDF594800EB840050F8041C4A
:1086F0002846BDE870400847A4F120001F2805D88F
:1087000029462046BDE87040F9F7B0BCA4F16000EE
:108710001F2805D829462046BDE87040FCF7EDBD6E
:10872000F02C0BD0BF2CDAD1A878298800F00100FA
:1087300001F08EFA78B1002070BD03E0A868F8F768
:108740007AFD08B11020F7E7284606F053FDBDE892
:108750007040FFF7EDBA0820EEE770B504460D460D
:108760000846F8F78EFD30B9601E1E280FD828463F
:10877000F8F761FD08B11020DEE7012C03D0022CD0
:1087800001D0032C01D10620D6E70720D4E7A4F1BD
:1087900020001F28F9D829462046BDE87040F9F787
:1087A000B9BC07F047B81CB500291FD104F02FFE53
:1087B000254800224178C06805F022FF2248103089
:1087C000C0788DF8000010B1012802D004E001202B
:1087D00000E000208DF80000684606F073F91B48A1
:1087E00024380068019001A806F0C6FA1CBD30B517
:1087F000144D0446383D6878A04200D8FFDF686811
:1088000000EB041030BD70B50E48002538382C46FA
:10881000467807E02046FFF7EAFF4078641C2844CA
:10882000C5B2E4B2B442F5D1284685E7021D5143F2
:10883000452900D245210844C01CB0FBF2F0C0B26B
:1088400070470000880300201C000020CCB101000C
:108850002DE9FC5F064676484FF000088B464746F8
:10886000444690F8019022E02046FFF7C0FF050043
:1088700000D1FFDF687869463844C7B22846FEF762
:10888000E2FF824601A92846FEF7F7FF0346BDF83E
:1088900004005246001D81B2BDF80000001D80B2E8
:1088A00007F0B4FC6A78641C00FB0288E4B24C4513
:1088B000DAD13068C01C20F003003060BBF1000F3B
:1088C00000D000204246394607F0AEFC316808442B
:1088D0003060BDE8FC9F5649383108710020C870EF
:1088E000AEE753493831CA782AB10A7801EB421110
:1088F0000831814201D00120A2E70020A0E72DE944
:10890000F04106460078154600F00F040020108064
:10891000601E0F46052800D3FFDF46482A4600EBBD
:108920008400394650F8043C3046BDE8F041184711
:108930002DE9F0413E4E0C46402806D041281AD081
:10894000422822D0432826D11AE0207865780128D1
:1089500001D9132014E5FF2D08D809F0F9FA0746CC
:108960000AF058FD381A401EA84201DA122007E525
:10897000208830810DE0BDE8F041084600F00DB8D8
:108980000878022807D8307603E00878022802D851
:1089900070760020F4E40720F2E438B5044640780D
:1089A00000F00300012803D002280BD0072038BDB7
:1089B000606858B1F8F78CFCD0B96068F8F77FFCB4
:1089C00020B915E06068F8F736FC88B9694620469A
:1089D000FBF762F90028EAD1607800F00300022872
:1089E00008D19DF8000028B16068F8F768FC08B16C
:1089F000102038BD6189F8290DD8208988420AD80D
:108A0000607800F003020A48012A06D1D731C26912
:108A100089B28A4201D2092038BD94E80E0000F1E3
:108A20000C0585E80E000AB900218182002038BDBE
:108A300050030020B4B101002DE9F041074614466F
:108A40008846084601F024FD064608EB88001C22F3
:108A5000796802EBC0000D18688C58B14146384661
:108A600001F025FD014678680078C200082305F171
:108A700020000CE0E88CA8B14146384601F01EFD0C
:108A80000146786808234078C20005F1240007F009
:108A90000EFA38B1062121726681D0E90010C4E9CE
:108AA000031009E0287809280BD005202072668180
:108AB0006868E060002028702046BDE8F04101F0C1
:108AC000C8BC072020726681F4E72DE9F041164604
:108AD0000D460746406801EB85011C2202EBC101EF
:108AE0004418204601F00CFD40B10021708865F368
:108AF0000F2160F31F4105200BF03CF90920207085
:108B0000324629463846BDE8F04195E72DE9F04167
:108B10000E46074600241C21F07816E004EB84037F
:108B2000726801EBC303D25C6AB1FFF7E3FA050098
:108B300000D1FFDF6F802A4621463046FFF7C5FF90
:108B40000120BDE8F081641CE4B2A042E6D8002018
:108B5000F7E770B5064600241C21C0780AE000BF84
:108B600004EB8403726801EBC303D5182A782AB199
:108B7000641CE4B2A042F3D8402070BD282200213A
:108B8000284604F022FC706880892881204670BD48
:108B900070B5034600201C25DC780CE000EB800655
:108BA0005A6805EBC6063244167816B1128A8A4214
:108BB00004D0401CC0B28442F0D8402070BDF0B553
:108BC000044600201C26E5780EE000BF00EB80077D
:108BD000636806EBC7073B441F788F4202D15B787E
:108BE000934204D0401CC0B28542EFD84020F0BD73
:108BF0000078032801D000207047012070470078DA
:108C0000022801D000207047012070470078072813
:108C100001D000207047012070472DE9F041064641
:108C200088461078F1781546884200D3FFDF2C780B
:108C30001C27641CF078E4B2A04201D8201AC4B208
:108C400004EB8401706807EBC1010844017821B18D
:108C50004146884708B12C7073E72878A042E8D1D4
:108C6000402028706DE770B514460B880122A240A1
:108C7000134207D113430B8001230A22011D07F081
:108C8000E0F8047070BD2DE9FF4F81B00878DDE990
:108C90000E7B9A4691460E4640072CD4019807F069
:108CA0007CFB040000D1FFDF07F1040820461FFA17
:108CB00088F106F0CBFC050000D1FFDF20462946F5
:108CC0006A4606F016FF0098A0F80370A0F805A009
:108CD000284606F0BCFF017869F306016BF3C71163
:108CE000017020461FFA88F106F0F3FC00B9FFDF9F
:108CF000019805F02DFC06EB0900017F491C017766
:108D000005B0BDE8F08F2DE9F84F0E469A46914622
:108D10000746032107F0FCF90446008DDFF87C8547
:108D2000002518B198F80000B0421ED1384607F06F
:108D300034FB070000D1FFDF09F10401384689B296
:108D400006F084FC050010D0384629466A4606F035
:108D5000D0FE009800210A460180817005F06DFC6C
:108D60000098C01DCAF8000021E098F80000B04249
:108D700016D104F1260734F8341F012000FA06F951
:108D800011EA090F00D0FFDF2088012340EA090023
:108D900020800A22391D384607F06EF8067006E07A
:108DA000324604F1340104F12600FFF75CFF0A218A
:108DB00088F800102846BDE8F88FFEB515460C4629
:108DC000064602AB0C220621FFF79DFF002827D0A4
:108DD0000299607812220A70801C487008224A802A
:108DE000A07002982988052381806988C180A9889C
:108DF0000181E988418100250C20CDE9000506228A
:108E000021463046FFF73FFF2946002266F31F4107
:108E1000F02310460AF004FF6078801C6070012087
:108E2000FEBD2DE9FE430C46804644E002AB0E2217
:108E300007214046FFF767FF002841D060681C22E9
:108E400067788678BF1C06EB860102EBC1014518E6
:108E500002981421017047700A214180698A0181BA
:108E6000E98A4181A9888180A9898181304601F000
:108E70000FFB029905230722C8806F700420287019
:108E800000250E20CDE9000521464046FFF7FBFEF8
:108E9000294666F30F2168F31F41F02300220520C5
:108EA0000AF0BEFE6078FE49801C60706268204651
:108EB000921CFFF7B2FE606880784028B6D101208E
:108EC000BDE8FE83FEB50D46064638E002AB0E2235
:108ED00007213046FFF717FF002835D068681C23AC
:108EE000C17801EB810203EBC202841802981522BB
:108EF0000270627842700A224280A2894281A2886E
:108F00008281084601F0C4FA014602988180618A94
:108F1000C180E18A0181A088B8B1002020700021C1
:108F20000E20CDE900010523072229463046FFF730
:108F3000AAFE6A68DB492846D21CFFF76EFE686805
:108F4000C0784028C2D10120FEBD0620E6E72DE909
:108F5000FE430C46814644E0204601F0BBFAD0B304
:108F600002AB082207214846FFF7CDFE0028A7D014
:108F700060681C2265780679AD1C06EB860102EB61
:108F8000C10147180298B7F810800621017045709A
:108F900004214180304601F07BFA01460298052306
:108FA0000722C180A0F804807D7008203870002559
:108FB000CDE9000521464846FFF765FE294666F3E0
:108FC0000F2169F31F41F023002205200AF028FE3B
:108FD0006078801C60706268B3492046121DFFF7FC
:108FE0001CFE606801794029B6D1012068E72DE9AF
:108FF000F34F83B00D4691E0284601F06BFA00284C
:109000007ED068681C2290F806A00AEB8A0102EB69
:10901000C10144185146284601F050FAA178CB000E
:1090200069684978CA00014604F1240006F05BFF34
:1090300007468188E08B4FF00009091A8EB208B10B
:10904000C84607E04FF00108504601F00CFA08B995
:10905000B61CB6B2208BB04200D80646B34602AB6F
:10906000324607210398FFF74EFE060007D0B8F1FD
:10907000000F0BD0504601F0F6F910B106E00020C9
:109080003EE60299B8884FF0020908800196E28B0B
:109090003968ABEB09001FFA80F80A4403984E4682
:1090A000009207F07AF9DDE90021F61D43460096AB
:1090B00006F099FDE08B404480B2E083B988884295
:1090C00001D1012600E00026CDE900B6238A07225F
:1090D00029460398FFF7D7FD504601F0C4F910B9AF
:1090E000E089401EE0815EB1A078401CA0706868F5
:1090F000E978427811FB02F1CAB20123816900E0EC
:1091000006E00E3006F09DFE80F800A00020E0830F
:109110006A6866492846921DFFF77FFD6868817975
:1091200040297FF469AF0120EAE570B5064648683A
:109130000D4614468179402910D104EB84011C228C
:1091400002EBC101084401F0FCF9002806D0686870
:10915000294684713046BDE8704048E770BDFEB5D1
:109160000C460746002645E0204601F0B3F9D8B387
:1091700060681C22417901EB810102EBC1014518B5
:10918000688900B9FFDF02AB082207213846FFF7E4
:10919000BAFD002833D00299607816220A70801C2C
:1091A0004870042048806068407901F071F90146F8
:1091B00002980523072281806989C1800820CDE9B2
:1091C000000621463846FFF75EFD6078801C60701F
:1091D000A88969890844B0F5803F00D3FFDFA889DA
:1091E00069890844A8816E81626831492046521D10
:1091F000FFF713FD606841794029B5D10120FEBD1C
:1092000030B5438C458BC3F3C704002345B1838B32
:10921000641EED1AC38A6D1E1D4495FBF3F3E4B280
:109220002CB1008918B1A04200D8204603444FF663
:10923000FF70834200D3034613800C7030BD2DE9CC
:10924000FC41074616460D46486802EB86011C2283
:1092500002EBC10144186A4601A92046FFF7D0FF7E
:10926000A089618901448AB2BDF80010914212D0F0
:10927000081A00D5002060816868407940280AD12A
:10928000204601F054F9002805D068682946467147
:109290003846FFF764FFBDE8FC8100003000002085
:1092A000F18B0000FF8B00000D8C000043A5000037
:1092B0002FA500002DE9FE4F0F4681461546508828
:1092C000032106F025FF0190B9F8020001F0D3F860
:1092D00082460146019801F0FDF8002824D001984B
:1092E0001C2241680AEB8A0002EBC0000C182046E1
:1092F00001F006F9002817D1B9F80000E18A884288
:109300000ED8A18961B1B8420ED10026514601980C
:1093100001F0CDF8218C01EB0008608B30B114E036
:10932000504601F0A0F8A0B3BDE8FE8F504601F012
:109330009AF808B1678308E0022FF5D3B9F8040062
:109340006083618A884224D80226B81B87B2B8F8A5
:109350000400A28B801A002814DD874200DA384608
:109360001FFA80FB688869680291D8F800100A44E7
:10937000009207F000F8F61D009A5B4602990096ED
:1093800006F0FDFBA08B384480B2A083618B88423D
:1093900007D96888019903B05246BDE8F04F01F043
:1093A000EDB81FD14FF009002872B9F802006881AA
:1093B000D8E90010C5E90410608BA881284601F0A7
:1093C00048F85146019801F072F8014601980823C7
:1093D00040680078C20004F1200006F068FD00201B
:1093E000A0836083504601F03EF810B9A089401E6A
:1093F000A0816888019903B00AF0FF02BDE8F04F30
:109400001DE72DE9F041064615460F461C46184655
:10941000F7F711FF18B92068F7F733FF08B11020EC
:109420001AE47168688C0978B0EBC10F01D313207E
:1094300012E43946304601F03AF8014670680823D4
:109440000078C20005F1200006F0FBFCD4E9001210
:10945000C0E90012002005E410B50446032106F01F
:1094600057FE014600F114022046BDE81040A4E476
:1094700070B50446032106F04BFE05460146204622
:10948000FFF765FD002816D029462046FFF767FE46
:10949000002810D029462046FFF714FD00280AD0E6
:1094A00029462046FFF7BDFC002804D02946204667
:1094B000BDE870409BE570BD2DE9F0410C4680464B
:1094C0001EE0E178427811FB02F1CAB28169012302
:1094D0000E3006F0ECFC077860681C22C179491E4A
:1094E000C17107EB8701606802EBC101461839467C
:1094F000204600F0EFFF18B1304600F0FAFF20B12F
:109500006068C1790029DCD18AE7FEF7F3FD050028
:1095100000D1FFDF0A202872384600F0B9FF6881C9
:109520003946204600F0CAFF0146606808234078AB
:10953000C20006F1240006F0BAFCD0E90010C5E92B
:109540000310A5F80280284600F083FFB07800B928
:10955000FFDFB078401EB07062E770B50C4605467C
:10956000032106F0D5FD01464068C2792244C2714C
:109570002846BDE870409FE72DE9FE4F82465078AF
:1095800014460F464FF00008002850D0012807D09D
:10959000022822D0FFDF2068B8606068F860C3E668
:1095A00002AB0E2208215046FFF7ADFB0028F2D097
:1095B0000298152105230170217841700A2141800C
:1095C000C0F80480C0F80880A0F80C80628882810E
:1095D0000E20CDE90008082221E0A678304600F0F0
:1095E00057FF054606EB86012C22786802EBC10185
:1095F0000822465A02AB11465046FFF784FB00286A
:10960000C9D002980721017021784170042141805E
:1096100008218580C680CDE9001805230A46394611
:109620004FEA0A00FFF72FFB87F808807CE6A67850
:10963000022516B1022E13D0FFDF2A1D914602AB80
:1096400008215046FFF75FFB0028A4D002980121B3
:10965000022E0170217841704580868002D005E09D
:109660000625EAE7A188C180E1880181CDE900985B
:109670000523082239465046D4E710B50446032195
:1096800006F046FD014600F108022046BDE8104004
:1096900072E72DE9F04F0F46054687B01446508813
:1096A000032106F035FD4FF000088DF808800646CE
:1096B000ADF80A80042F5CD36A78002A59D0287844
:1096C0004FF6FF794FF01C0A132815D006DC01284D
:1096D0006FD006282BD0072806D16EE0142869D059
:1096E000152868D0162867D0CDF80080CDF8048002
:1096F00068788DF8000037E0B078904239D1307842
:10970000010736D5062F34D120F00800307060886C
:10971000414660F31F4100200AF02CFB02208DF827
:109720000800ADF80C90A888ADF80E00F4E0082F02
:109730001FD1A888EF88814600F09DFE8046014633
:10974000304600F0C7FE18B1404600F08CFE98B1DC
:10975000FA48D0E90010CDE900106878ADF804901F
:109760008DF80000ADF8067060886A463146FFF754
:1097700003FF07B0BDE8F08F716808EB88002C226A
:1097800002EBC000085AB842F3D1EC486A46D0E96F
:109790000210CDE9001068788DF8000008F0FF0590
:1097A0008DF8025060883146FFF7E6FE22462946D2
:1097B00023E097E025E0CEE023E1082FD9D1B5F8EA
:1097C0000480E88800F057FE07460146304600F066
:1097D00081FE0028CDD007EB870271680AEBC2003A
:1097E0000844028A4245C4D101780829C1D1407891
:1097F00069788842BDD1F9B222463046FFF765F953
:10980000B7E70E2F7FF470AFE9886F898B46B5F804
:1098100008903046FFF7BCF9ABF14001402901D375
:10982000092048E0B9F1170F01D3172F01D20B20FF
:1098300041E040280ED000EB800271680AEBC200C4
:1098400008440178012903D140786978884290D092
:109850000A2030E03046FFF77CF940282AD000EBA0
:10986000800372680AEBC30102EB0108012288F849
:1098700000206A7888F801207168AA884989B9426D
:1098800000D93946AD8903232372A282E781218260
:10989000A4F80C90658200F0FBFD6081A8F814909C
:1098A000A8F81870A8F80E50A8F810B0204600F0DC
:1098B000D0FD5EE7042005212172A4F80A80E08132
:1098C000012121739D49D1E90421CDE90021697865
:1098D0008DF80010ADF8020060886A463146FFF747
:1098E0004BFEE3E7062F8BD3B07890421AD1307845
:1098F000010717D520F0080030706088414660F3FA
:109900001F4100200AF036FA02208DF80800A888CE
:10991000ADF80C00ADF80E906088224602A9F8F769
:1099200069FB26E704213046FFF749F90546402840
:10993000BFD002208303009022462946304600F023
:10994000E6FD4146608865F30F2160F31F41052065
:109950000AF010FA0DE70E2FABD104213046FFF7C5
:109960002EF981464028A4D04146608869F30F2132
:1099700060F31F4105200AF0FDF9A8890690688967
:10998000009070682F894089B84200D938468346D4
:10999000B5F80680A8880190484600F079FD6081FE
:1099A000069818B102200090069B24E0B8F1170F2A
:1099B0001ED3172F1CD30420207200986082E781E9
:1099C000A4F810B0A4F80C8009EB890271680AEBC6
:1099D000C2000D18DDE90002A5F81480A5F818B042
:1099E000E8812A82204600F034FD06202870C0E677
:1099F00001200B23009022464946304600F087FDA7
:109A0000B7E6082F8DD1A9883046FFF7C1F8074681
:109A1000402886D000F027FD00289BD107EB870265
:109A200071680AEBC2000844804600F069FD002816
:109A300090D1ED88B8F80E002844B0F5803F05D3EA
:109A400060883A46314600F099FD92E6002DCED06E
:109A5000A8F80E0060883A463146FFF766FB0820FA
:109A60002072384600F014FD6081A5811EE72DE9C3
:109A7000F05F0C4601281ED0957992F80480567943
:109A800005EB85011F2202EBC10121F0030B08EB5E
:109A9000060111FB05F14FF6FF7202EAC10909F157
:109AA000030115FB0611264F21F0031ABB6840B1D4
:109AB00001283ED125E06168E57891F800804E7874
:109AC000DEE75946184606F070F9606000B9FFDF1E
:109AD0005A460021606803F078FCE5705146B8688A
:109AE00006F063F96168486100B9FFDF60684269A8
:109AF00002EB09018161606880F80080606846704F
:109B000017E0606852464169184606F079F95A46EE
:109B10006168B86806F074F9032006F0A5FA0446F7
:109B2000032006F0A9FA201A012802D1B86806F02D
:109B300031F90BEB0A00BDE8F09F0000D8B101003D
:109B40003000002002460021022090E7F7B5FF4CCC
:109B50000A2016462070009860B100254FEA0D00DB
:109B600006F005F90021A1706670002D01D1009961
:109B7000A160FEBD01250020F2E770B50C46154638
:109B800038220021204603F020FC012666700A22BC
:109B9000002104F11C0003F018FC05B9FFDF297A4D
:109BA000207861F301002070A87900282DD02A4682
:109BB00021460020FFF75BFF61684020E34A887080
:109BC0006168C8706168087161684871616888710E
:109BD0006168288808816168688848816068868132
:109BE0009078002811D0616806200877616828887D
:109BF000C8856168288848866068068560686988C5
:109C00009288018681864685828570BDC878002845
:109C100002D0002201202AE7704770B505460021D6
:109C200065F31F4100200AF0A5F80321284606F03D
:109C30006FFA040000D1FFDF21462846FEF766FFD9
:109C4000002804D0207840F010002070012070BD62
:109C500070B505460C46032006F0F8F908B100205F
:109C600070BDBA4885708480012070BD2DE9FF4128
:109C700080460E460F0CFEF73DFA050007D06F80B8
:109C80000321384606F044FA040008D106E004B087
:109C90003846BDE8F0411321F8F788BDFFDF5FEAE1
:109CA000080005D0B8F1050F18D0FFDFBDE8FF812F
:109CB00020782A4620F0080020700020ADF802002D
:109CC00002208DF800004FF6FF70ADF80400ADF8EB
:109CD000060069463846F8F78DF9E7E7C6F307212D
:109CE00001EB81021C23606803EBC202805C042844
:109CF00003D008280AD0FFDFD8E7012000904FF4F6
:109D000040432A46204600F002FCCFE704B02A4632
:109D10002046BDE8F041FEF7D8BE2DE9F05F0546CC
:109D20004089002790460C463E46824600F0A3FB41
:109D30008146287AC01E08286BD2DFE800F00D04A7
:109D4000192058363C4772271026002C6CD0D5E9D4
:109D50000301C4E902015CE070271226002C63D0E5
:109D60000A2205F10C0104F1080003F004FB50E0A5
:109D700071270C26002C57D0E868A06049E07427B2
:109D800010269CB3D5E90301C4E9020168880321C8
:109D900006F0BEF98346FEF7ADF9024668885080AA
:109DA00049465846FEF748FE33E075270A26ECB1CF
:109DB000A88920812DE076271426BCB105F10C007E
:109DC00004F1080307C883E8070022E0772710267C
:109DD00064B1D5E90301C4E902016888032106F0F2
:109DE00097F901466888FFF767FB12E01CE07327CC
:109DF0000826CCB16888032106F08AF9014600786C
:109E0000C00606D56888FEF781FE10B96888F7F7A6
:109E1000E7FDA8F800602CB12780A4F806A06680B2
:109E20006888A080002086E6A8F80060FAE72DE99F
:109E3000FC410C461E4617468046032106F068F991
:109E400005460A2C0AD2DFE804F0050505050505DC
:109E500009090907042303E0062301E0FFDF0023CB
:109E6000CDE90076224629464046FEF70CFFBDE8C4
:109E7000FC81F8B50546A0F57F40FF382BD0284679
:109E800006F079FA040000D1FFDF204605F00FFE4E
:109E9000002821D001466A46204605F02AFE009897
:109EA0000321B0F80560284606F032F90446052E75
:109EB00013D0304600F0DFFA05460146204600F098
:109EC00009FB40B1606805EB85013E2202EBC10150
:109ED000405A002800D00120F8BD007A0028FAD0AE
:109EE0000020F8BDF8B50446408806F044FA0500A5
:109EF00000D1FFDF6A462846616800F0A8FA0146F3
:109F00000098091F8BB230F8032F028042884280EC
:109F10000188994205D1042A08D0052A20D0062AB2
:109F200016D022461946FFF7C5F9F8BD001D0E46AA
:109F30000546014622463046FBF74DF90828F4D184
:109F4000224629463046FCF7BAF9F8BD3000002019
:109F5000636864880A46011D2046F9F7A9FBF4E707
:109F60002246001DFFF795FBEFE770B50D4606464C
:109F7000032106F0CDF8040004D02078000704D5B2
:109F8000112070BD43F2020070BD2A4621463046C2
:109F9000FEF713FF18B9286860616868A06120782F
:109FA00040F008002070002070BD2DE9F04F0E46F3
:109FB00091B08046032106F0ABF80446404606F017
:109FC000ECF907460020079008900990ADF83000A2
:109FD0000A9002900390049004B9FFDF0DF1080984
:109FE000FFB9FFDF1DE038460BA9002205F022FC77
:109FF0009DF82C0000F07F050A2D00D3FFDF6019CB
:10A00000017F491E01779DF82C00000609D52A46DC
:10A010000CA907A8FEF727FE19F80510491C09F836
:10A020000510761EF6B2DED204F13400F84D04F1CC
:10A03000260BDFF8E0A304F12A07069010E058464B
:10A04000069900F08DFA064628700A2800D3FFDF33
:10A050005AF8261040468847E08CC05DB04202D0D6
:10A06000208D0028EBD10A202870EA4D4E46283575
:10A070000EE00CA907A800F073FA0446375D55F806
:10A08000240000B9FFDF55F82420394640469047A8
:10A09000BDF81E000028ECD111B0BDE8F08F10B55E
:10A0A000032106F035F8040000D1FFDF0A22002169
:10A0B00004F11C0003F089F9207840F004002070BE
:10A0C00010BD10B50C46032106F022F82044007F95
:10A0D000002800D0012010BD2DE9F84F8946154613
:10A0E0008246032106F014F8070004D02846F7F74B
:10A0F000A2F840B903E043F20200BDE8F88F4846F9
:10A10000F7F7BFF808B11020F7E7786828B1698839
:10A110000089814201D90920EFE7B9F800001C2429
:10A1200088B100F0A8F980460146384600F0D2F91F
:10A1300088B108EB8800796804EBC000085C01284E
:10A140000BD00820D9E73846FEF703FD80464028AB
:10A1500007D11320D1E70520CFE7FDF7CBFF06009D
:10A160000BD008EB8800796804EBC0000C18B9F834
:10A17000000020B1E88910B113E01120BDE7288864
:10A18000172802D36888172801D20720B5E7686826
:10A1900038B12B1D224641463846FFF732F90028D8
:10A1A000ABD104F10C0269462046FFF729F8288854
:10A1B00060826888E082B9F8000030B10220207027
:10A1C000E889A080E889A0B12BE003202070A8894D
:10A1D000A08078688178402905D180F802803946CE
:10A1E0005046FEF71EFE404600F052F9A9F8000066
:10A1F00021E07868218B4089884200D90846208375
:10A20000A6F802A004203072B9F800007081E0893D
:10A210007082F181208B3082A08AB081304600F0BC
:10A2200018F97868C178402905D180F8038039464B
:10A230005046FEF747FE00205FE770B50D46064624
:10A24000032105F065FF04000ED0284600F013F945
:10A2500005460146204600F03DF918B1284600F0B9
:10A2600002F920B1052070BD43F2020070BD05EB7C
:10A2700085011C22606802EBC101084400F040F92E
:10A2800008B1082070BD2A462146304600F076F914
:10A29000002070BD2DE9F0410C4617468046032191
:10A2A00005F036FF0546204600F0E5F8044695B176
:10A2B0000146284600F00EF980B104EB84011C220F
:10A2C000686802EBC1014618304600F019F938B150
:10A2D0000820BDE8F08143F20200FAE70520F8E724
:10A2E0003B46324621462846FFF78BF80028F0D13E
:10A2F000E2B229464046FEF7A2FF708C08380828D3
:10A3000003D24348407800F06BFE0020E1E72DE9DE
:10A31000F0410D4617468046032105F0F9FE04463C
:10A32000284600F0A8F8064624B13846F6F783FF21
:10A3300038B902E043F20200CBE73868F6F77BFF5A
:10A3400008B11020C5E73146204600F0C3F860B1DF
:10A3500006EB86011C22606802EBC1014518284605
:10A3600000F0CEF818B10820B3E70520B1E7B888AF
:10A37000A98A884201D90C20ABE76168E88C49784A
:10A38000B0EBC10F01D31320A3E73146204600F004
:10A3900095F80146606808234078C20005F1240062
:10A3A00005F04FFDD7E90012C0E90012F2B22146D4
:10A3B0004046FEF7BAFE00208BE72DE9F0470D4638
:10A3C0001F4690468146032105F0A2FE044628461A
:10A3D00000F051F806463CB14DB13846F6F76FFF34
:10A3E00050B11020BDE8F08743F20200FAE7606840
:10A3F00058B1A0F80C8028E03146204600F06AF8F9
:10A4000018B1304600F02FF830B10520EAE700001F
:10A4100030000020F0B1010006EB86011C226068CC
:10A4200002EBC1014518284600F06AF808B108207F
:10A43000D8E7A5F80880F2B221464846FEF7FFFEAD
:10A440001FB1A8896989084438800020CAE705F04F
:10A4500050BB017821F00F01491C21F0F0011031AF
:10A460000170FDF74BBE20B94E48807808B101203D
:10A470007047002070474B498988884201D10020ED
:10A480007047402801D2402000E0403880B2704739
:10A4900010B50446402800D9FFDF2046FFF7E3FF50
:10A4A00010B14048808810BD4034A0B210BD406853
:10A4B00042690078484302EBC0007047C2784068A8
:10A4C000037812FB03F24378406901FB032100EBA0
:10A4D000C1007047C2788A4209D9406801EB810106
:10A4E0001C2202EBC101405C08B101207047002032
:10A4F00070470078062801D9012070470020704776
:10A500000078062801D00120704700207047F0B481
:10A5100001EB81061C27446807EBC6063444049D02
:10A5200005262670E3802571F0BCFEF785BA10B5CC
:10A53000418911B1FFF7DDFF08B1002010BD0120F6
:10A5400010BD10B5C18C8278B1EBC20F04D9C1899E
:10A5500011B1FFF7CEFF08B1002010BD012010BDE2
:10A5600010B50C4601230A22011D05F0A0FC00785D
:10A570002188012282409143218010BDF0B402EB7A
:10A5800082051C264C6806EBC505072363554B68FE
:10A590001C79402C03D11A71F0BCFEF7D8BCF0BC7A
:10A5A000704700003000002070B50B2000F0BDF9AE
:10A5B000082000F0BAF900210B2000F0D4F90021A6
:10A5C000082000F0D0F9F44C01256560A56000205A
:10A5D000C4F84001C4F84401C4F848010B2000F05D
:10A5E000B5F9082000F0B2F90B2000F091F92560D0
:10A5F00070BD10B50B2000F098F9082000F095F917
:10A60000E548012141608160E4490A68002AFCD1E3
:10A610000021C0F84011C0F84411C0F848110B20C7
:10A6200000F094F9BDE81040082000F08FB910B593
:10A630000B2000F08BF9BDE81040082000F086B92F
:10A6400000B530B1012806D0022806D0FFDF002077
:10A6500000BDD34800BDD34800BDD248001D00BD99
:10A6600070B5D1494FF000400860D04DC00BC5F81F
:10A670000803CF4800240460C5F840410820C435D1
:10A6800000F053F9C5F83C41CA48047070BD08B5E4
:10A69000C14A002128B1012811D002281CD0FFDFB7
:10A6A00008BD4FF48030C2F80803C2F84803BB4825
:10A6B0003C300160C2F84011BDE80840D0E74FF4DB
:10A6C0000030C2F80803C2F84803B44840300160C3
:10A6D000C2F84411B3480CE04FF48020C2F80803DC
:10A6E000C2F84803AD4844300160C2F84811AD4893
:10A6F000001D0068009008BD70B516460D46044662
:10A70000022800D9FFDF0022A348012304F1100131
:10A710008B4000EB8401C1F8405526B1C1F84021BF
:10A72000C0F8043303E0C0F80833C1F84021C0F892
:10A73000443370BD2DE9F0411D46144630B1012867
:10A7400033D0022838D0FFDFBDE8F081891E002217
:10A7500021F07F411046FFF7CFFF012D23D00020CD
:10A76000944D924F012668703E61914900203C391A
:10A7700008600220091D08608D49042030390860F6
:10A780008B483D34046008206C6000F0DFF8300432
:10A79000C7F80403082000F0BBF88349F007091F3D
:10A7A00008602E70D0E70120DAE7012B02D00022EA
:10A7B000012005E00122FBE7012B04D0002202204A
:10A7C000BDE8F04198E70122F9E774480068704756
:10A7D00070B500F0D8F8704C0546D4F8400100265A
:10A7E000012809D1D4F80803C00305D54FF48030FF
:10A7F000C4F80803C4F84061D4F8440101280CD11E
:10A80000D4F80803800308D54FF40030C4F80803D7
:10A81000C4F84461012008F01AFAD4F8480101286C
:10A820000CD1D4F80803400308D54FF48020C4F8B5
:10A830000803C4F84861022008F009FA5E48056080
:10A8400070BD70B500F09FF85A4D0446287850B19D
:10A85000FFF706FF687818B10020687008F0F7F974
:10A860005548046070BD0320F8E74FF0E0214FF435
:10A870000010C1F800027047152000F067B84B497E
:10A8800001200861082000F061B848494FF47C10AD
:10A89000C1F808030020024601EB8003C3F84025FD
:10A8A000C3F84021401CC0B20628F5D37047410AC6
:10A8B00043F609525143C0F3080010FB02F000F5C3
:10A8C000807001EB5020704710B5430B48F237649D
:10A8D00063431B0C5C020C60384C03FB0400384BD8
:10A8E0004CF2F72443435B0D13FB04F404EB4020CC
:10A8F00000F580704012107008681844086010BDA0
:10A900002C484068704729490120C1F8000270476F
:10A91000002809DB00F01F0201219140400980005E
:10A9200000F1E020C0F80011704700280DDB00F0B6
:10A930001F02012191404009800000F1E020C0F891
:10A940008011BFF34F8FBFF36F8F7047002809DB73
:10A9500000F01F02012191404009800000F1E02039
:10A96000C0F8801270474907090E002804DB00F187
:10A97000E02080F80014704700F00F0000F1E020A4
:10A9800080F8141D70470C48001F00680A4A0D49E2
:10A99000121D11607047000000B0004004B5004077
:10A9A0004081004044B1004008F501400080004073
:10A9B000408500403C00002014050240F7C2FFFF24
:10A9C0006F0C01000100000110B5EFF3108000F0E2
:10A9D000010472B6FC484178491C41704078012856
:10A9E00001D108F087FD002C00D162B610BD70B512
:10A9F000F54CA07848B90125A570FFF7E5FF08F0F0
:10AA00008AFD20B1002008F054FD002070BD4FF0F9
:10AA10008040E570C0F80453F7E770B5EFF310809D
:10AA200000F0010572B6E84C607800B9FFDF60788D
:10AA3000401E6070607808B908F060FD002D00D1FC
:10AA400062B670BDE04810B5817821B10021C170B7
:10AA50008170FFF7E2FF002010BD10B5044608F03A
:10AA60005AFDD9498978084000D001202060002093
:10AA700010BD10B5FFF7A8FF08F04DFD022201231D
:10AA8000D149540728B1D1480260236103200872DC
:10AA900002E00A72C4F804330020887110BD2DE969
:10AAA000F84FDFF824934278817889F80420002653
:10AAB00089F80510074689F806600078DFF810B3BA
:10AAC000354620B1012811D0022811D0FFDF08F04F
:10AAD00034FD4FF0804498B108F036FDB0420FD1FC
:10AAE000304608F035FD0028FAD042E00126EEE7B6
:10AAF000FFF76AFF58460168C907FCD00226E6E75F
:10AB00000120E060C4F80451B2490E600107D1F899
:10AB10004412B04AC1F3423124321160AD4934319C
:10AB200008604FF0020AC4F804A3A060AA480168B4
:10AB3000C94341F3001101F10108016841F010011E
:10AB4000016001E010F06CF9D4F804010028F9D09C
:10AB5000304608F0FDFC0028FAD0B8F1000F04D10F
:10AB60009D48016821F010010160C4F808A3C4F8F1
:10AB7000045199F805004E4680B1387870B908F054
:10AB8000CAFC804608F0DAFE6FF00042B8F1000F10
:10AB900002D0C6E9032001E0C6E90302DBF80000A9
:10ABA000C00701D008F0B3FC387810B13572BDE8A9
:10ABB000F88F4FF01808C4F808830127A7614FF4F5
:10ABC0002070ADF8000000BFBDF80000411EADF8D8
:10ABD0000010F9D2C4F80C51C4F810517A48C01DC5
:10ABE00008F040FD3570FFF744FF6761794930791F
:10ABF00020310860C4F80483D9E770B5050000D19E
:10AC0000FFDF4FF080424FF0FF30C2F80803002111
:10AC1000C2F80011C2F80411C2F80C11C2F81011E8
:10AC2000694C617008F083FC10B10120A070607065
:10AC300067480068C00701D008F069FC2846BDE8F5
:10AC400070402CE76048007A002800D0012070474F
:10AC50002DE9F04F61484FF0000A85B0D0F800B000
:10AC6000D14657465D4A5E49083211608406D4F8E1
:10AC7000080110B14FF0010801E04FF0000808F0A2
:10AC8000C4FC78B1D4F8240100B101208246D4F884
:10AC90001C0100B101208146D4F8200108B1012730
:10ACA00000E00027D4F8000100B101200490D4F89E
:10ACB000040100B101200390D4F80C0100B101207F
:10ACC0000290D4F8100100B101203F4D0190287886
:10ACD00000260090B8F1000F04D0C4F808610120EC
:10ACE00008F0E7FBBAF1000F04D0C4F82461092092
:10ACF00008F0DFFBB9F1000F04D0C4F81C610A2092
:10AD000008F0D7FB27B1C4F820610B2008F0D1FB75
:10AD10002D48C01D08F0AEFC00B1FFDFDFF8AC80AD
:10AD20000498012780B1C4F80873E87818B1EE7070
:10AD3000002008F0BEFB287A022805D103202872E3
:10AD40000221C8F800102761039808B1C4F8046113
:10AD5000029850B1C4F80C61287A032800D0FFDFB4
:10AD6000C8F800602F72FFF758FE019838B1C4F898
:10AD70001061287A012801D100F05CF86761009821
:10AD800038B12E70287A012801D1FFF772FEFFF743
:10AD900044FE0D48C01D08F083FC1049091DC1F890
:10ADA00000B005B0BDE8F08F074810B5C01D08F031
:10ADB00061FC0549B0B1012008704FF0E021C1F8F5
:10ADC0000002BDE81040FFE544000020340C0040C4
:10ADD0000C0400401805004010ED00E01005024092
:10ADE00001000001087A012801D1FFF742FEBDE809
:10ADF0001040244808F054BC70B5224CE41FA078E1
:10AE000008B908F07BFB01208507A861207A00269D
:10AE1000032809D1D5F80C0120B9002008F098FBCF
:10AE20000028F7D1C5F80C6126724FF0FF30C5F845
:10AE3000080370BD70B5134CE41F6079F0B10128B0
:10AE400003D0A179401E814218DA08F064FB054660
:10AE500008F074FD6179012902D9A179491CA17119
:10AE60000DB1216900E0E168411A022902DA11F10D
:10AE7000020F06DC0DB1206100E0E060BDE870402B
:10AE8000F7E570BD4B00002037490120086070478E
:10AE900070B50D2000F049F8344C0020C4F80001D2
:10AEA0000125C4F804530D2000F050F825604FF040
:10AEB000E0216014C1F8000170BD10B50D2000F054
:10AEC00034F82A48012141600021C0F80011BDE892
:10AED00010400D2000F03AB8254810B50468244908
:10AEE0002448083108602149D1F80001012804D024
:10AEF000FFDF1F48001D046010BD1B48001D0068D7
:10AF00000022C0B2C1F8002108F06FFCF1E710B5D3
:10AF1000164800BFD0F800110029FBD0FFF7DCFF76
:10AF2000BDE810400D2000F011B800280DDB00F046
:10AF30001F02012191404009800000F1E020C0F88B
:10AF40008011BFF34F8FBFF36F8F7047002809DB6D
:10AF500000F01F02012191404009800000F1E02033
:10AF6000C0F880127047000004D5004000D00040B7
:10AF700010050240010000014FF0E0214FF0007089
:10AF8000C1F8800101F5C071BFF34F8FBFF36F8F20
:10AF9000C1F80001394B802283F8002441F8800C6D
:10AFA000704700B502460420354903E001EBC003B9
:10AFB0001B792BB1401EC0B2F8D2FFDFFF2000BDCD
:10AFC00041F8302001EBC00100224A718A71012250
:10AFD0000A7100BD2A4A002102EBC00001717047CE
:10AFE00010B50446042800D3FFDF254800EBC40455
:10AFF0002079012800D0FFDF6079A179401CC0B220
:10B00000814200D060714FF0E0214FF00070C1F834
:10B01000000210BD70B50425194E1A4C16E02178B7
:10B0200006EBC1000279012A08D1427983799A425C
:10B0300004D04279827156F8310080472078401C54
:10B04000C0B22070042801D3002020706D1EEDB224
:10B05000E5D270BD0C4810B504680B490B480831A7
:10B060000860064890F800044009042800D0FFDF7B
:10B07000FFF7D0FF0448001D046010BD19E000E098
:10B080007405002058000020100502400100000156
:10B090000548064A0168914201D100210160044936
:10B0A00001200860704700005C000020BEBAFECAA4
:10B0B00040E501400F4A12680D498A420CD11847F9
:10B0C0000C4A12680A4B9A4206D101B508F008FCF6
:10B0D00008F0DBFEBDE80140074909680958084748
:10B0E00006480749054A064B70470000000000006B
:10B0F000BEBAFECA5C00002004000020B00F002091
:10B10000B00F0020F8B51D46DDE906470E000AD055
:10B1100005F043F92346FF1DBCB231462A46009490
:10B1200004F061FDF8BDD0192246194602F023F95A
:10B130002046F8BD70B50D4604461022002102F0ED
:10B1400044F9258117206081A07B40F00A00A0739C
:10B1500070BD4FF6FF720A800146022008F00ABE59
:10B16000704700897047827BD30701D1920703D4CF
:10B17000808908800020704705207047827B9207F5
:10B1800000D58181704701460020098841F6FE52B2
:10B19000114200D00120704700B50346807BC007F4
:10B1A00001D0052000BD59811846FFF7ECFFC0070C
:10B1B00003D0987B40F004009873987B40F0010026
:10B1C0009873002000BD827B520700D509B14089E9
:10B1D000704717207047827B61F3C3028273704708
:10B1E0002DE9FC5F0E46044601789646012000FAE0
:10B1F00001F14DF6FF5201EA020962684FF6FF7B4A
:10B200001188594502D10920BDE8FC9FB9F1000F12
:10B2100005D041F6FE55294201D00120F4E741EA6C
:10B22000090111801D0014D000232B7094F800C078
:10B23000052103221F464FF0020ABCF10E0F76D201
:10B24000DFE80CF0F909252F47646B77479193B439
:10B25000D1D80420D8E7616820898B7B9B0767D50C
:10B2600017284AD30B89834247D38989172901D3E9
:10B27000814242D185F800A0A5F8010032806168C2
:10B2800088816068817B21F002018173C6E004201F
:10B2900028702089A5F801006089A5F80300318095
:10B2A000BCE0208A3188C01D1FFA80F8414524D3B4
:10B2B000062028702089A5F801006089A5F8030000
:10B2C000A089A5F805000721208ACDE9000163695E
:10B2D00041E00CF0FF00082810D0082028702089D9
:10B2E000A5F801006089A5F8030031806A1D694650
:10B2F00004F10C0006F0BBFC10B15EE01020EDE79D
:10B3000030889DF800100844308087E00A202870BB
:10B310002089A5F80100328044E00C2028702089A3
:10B32000A5F801006089A5F8030031803AE082E0C9
:10B3300064E02189338800EB41021FFA82F843451B
:10B340003BD3B8F1050F38D30E222A700BEA410126
:10B35000CDE90010E36860882A467146FFF7D2FE07
:10B36000A6F800805AE04020287060893188C01C0F
:10B370001FFA80F8414520D32878714620F03F001D
:10B38000123028702089A5F801006089CDE90002FB
:10B3900060882A46E368FFF7B5FEA6F800802878A3
:10B3A00040063BD461682089888037E0A0893288D4
:10B3B000401D1FFA80F8424501D204273DE01620C7
:10B3C00028702089A5F801006089A5F80300A089EC
:10B3D000CDE9000160882A4671462369FFF792FE95
:10B3E000A6F80080DEE718202870207A6870A6F89A
:10B3F00000A013E061680A88920401D405271CE0CC
:10B40000C9882289914201D0062716E01E212970A1
:10B4100030806068018821F400510180B9F1000F8B
:10B420000BD0618878230022022008F0F9FB6168C4
:10B430002078887006E0338003276068018821EA5D
:10B44000090101803846DFE62DE9FF4F85B0174638
:10B45000129C0D001E461CD03078C10703D000F0AE
:10B460003F00192801D9012100E000212046FFF703
:10B47000AAFEA8420DD32088A0F57F41FF3908D04D
:10B480003078410601D4000605D5082009B0BDE892
:10B49000F08F0720FAE700208DF800008DF80100FA
:10B4A00030786B1E00F03F0C0121A81E4FF0050AFA
:10B4B0004FF002094FF0030B9AB2BCF1200F75D286
:10B4C000DFE80CF08B10745E7468748C749C74B537
:10B4D00074BA74C874D474E1747474F174EF74EE53
:10B4E00074ED748B052D78D18DF80090A0788DF8CF
:10B4F00004007088ADF8060030798DF8010070788E
:10B5000000F03F000C2829D00ADCA0F10200092835
:10B5100063D2DFE800F0126215621A621D62200039
:10B52000122824D004DC0E281BD01028DBD11BE00D
:10B5300016281FD01828D6D11FE02078800701E0F8
:10B5400020784007002848DAEEE020780007F9E785
:10B550002078C006F6E720788006F3E720784006DA
:10B56000F0E720780006EDE72088C005EAE72088AC
:10B570004005E7E720880005E4E72088C004E1E70C
:10B580002078800729D5032D27D18DF800B0B6F893
:10B59000010081E0217849071FD5062D1DD381B216
:10B5A0007078012803D0022817D102E0C9E00220F8
:10B5B00000E0102004228DF8002072788DF804201D
:10B5C000801CB1FBF0F2ADF8062092B242438A42F1
:10B5D00003D10397ADF80890A6E079E02078000742
:10B5E00076D598B282088DF800A0ADF80420B0EBB3
:10B5F000820F6DD10297ADF8061095E02178C9064B
:10B6000066D5022D64D381B206208DF800007078D3
:10B6100002285DD3B1FBF0F28DF80400ADF80620EE
:10B6200092B242438A4253D1ADF808907BE0207831
:10B6300080064DD5072003E0207840067FD50820FE
:10B640008DF80000A088ADF80400ADF80620ADF834
:10B65000081068E02078000671D50920ADF80420B4
:10B660008DF80000ADF8061002975DE02188C9054D
:10B6700065D5022D63D381B20A208DF80000707861
:10B6800004285CD3C6E72088400558D5012D56D143
:10B690000B208DF80000A088ADF8040044E021E004
:10B6A00026E016E0FFE72088000548D5052D46D3A3
:10B6B0000C208DF80000A088ADF80400B6F8030057
:10B6C0006D1FADF80850ADF80600ADF80AA02AE0ED
:10B6D00035E02088C00432D5012D30D10D208DF801
:10B6E000000021E02088800429D4B6F80100E08021
:10B6F000A07B000723D5032D21D3307800F03F0035
:10B700001B2818D00F208DF80000208840F400502E
:10B71000A4F80000B6F80100ADF80400ED1EADF885
:10B720000650ADF808B0039769460598F9F79CFAFA
:10B73000050008D016E00E208DF80000EAE7072586
:10B7400010E008250EE0307800F03F001B2809D0FB
:10B750001D2807D00220059908F00CFB208800F472
:10B7600000502080A07B400708D52046FFF70BFD46
:10B77000C00703D1A07B20F00400A073284685E613
:10B780001FB5022806D101208DF8000088B2694655
:10B79000F9F76AFA1FBD0000F8B51D46DDE9064756
:10B7A0000E000AD004F0F9FD2346FF1DBCB231465D
:10B7B0002A46009404F017FAF8BDD019224619461B
:10B7C00001F0D9FD2046F8BD2DE9FF4F8DB09B4615
:10B7D000DDE91B57DDF87CA00C46082B05D0E0699D
:10B7E00001F0FEF850B11020D2E02888092140F085
:10B7F000100028808AF80010022617E0E169012075
:10B800008871E2694FF420519180E1698872E069A2
:10B8100042F601010181E06900218173288811212C
:10B8200040F0200028808AF80010042638780A901A
:10B830000A2038704FF0020904F118004D460C90B0
:10B8400001F0C6FBB04681E0BBF1100F0ED1022D16
:10B850000CD0A9EB0800801C80B20221CDE90010B9
:10B8600005AB52461E990D98FFF796FFBDF81610CE
:10B870001A98814203D9F74800790F9004E003D168
:10B880000A9808B138702FE04FF00201CDE9001995
:10B890000DF1160352461E990D98FFF77DFF1D9876
:10B8A0000088401B801B83B2C6F1FF00984200D283
:10B8B00003461E990BA8D9B15FF00002DDF878C0ED
:10B8C000CDE9032009EB060189B2CDE901C10F984A
:10B8D0000090BDF8161000220D9801F00EFC387093
:10B8E00070B1C0B2832807D0BDF8160020833AE0BB
:10B8F0000AEB09018A19E1E7022011B0BDE8F08FD7
:10B90000BDF82C00811901F0FF08022D0DD09AF826
:10B910000120424506D1BDF82010814207D0B8F180
:10B92000FF0F04D09AF801801FE08AF80180C9480F
:10B9300000680178052902D1BDF81610818009EB55
:10B9400008001FFA80F905EB080085B2DDE90C104C
:10B9500005AB0F9A01F03FFB28B91D980088411BE9
:10B960004145BFF671AF022D13D0BBF1100F0CD1C2
:10B97000A9EB0800801C81B20220CDE9000105ABD3
:10B9800052461E990D98FFF707FF1D98058000206D
:10B9900038700020B1E72DE9F8439C46089E134615
:10B9A0000027B26B9AB3491F8CB2F18FA1F57F4586
:10B9B000FF3D05D05518AD882944891D8DB200E0A2
:10B9C00000252919B6F83C800831414520D82A4481
:10B9D000BCF8011022F8021BBCF8031022F8021B6D
:10B9E000984622F8024B914604F0C5FC4FF00C0C2F
:10B9F00041464A462346CDF800C004F0C0F8F5871A
:10BA0000B16B00202944A41D2144088003E001E01B
:10BA1000092700E083273846BDE8F88310B50B8876
:10BA2000848F9C420CD9846BE018048844B18488CC
:10BA300024F40044A41D23440B801060002010BD9A
:10BA40000A2010BD2DE9F0478AB0002590468946AE
:10BA50008246ADF8185007274BE005980688808885
:10BA6000000446D4A8F8006007A801950097029545
:10BA7000CDE903504FF4007300223146504601F0E7
:10BA80003CFB04003CD1BDF81800ADF8200005983F
:10BA900004888188B44216D10A0414D40195029511
:10BAA000039521F400410097049541F480434288B6
:10BAB0002146504601F0BFF804000BD1059881885B
:10BAC00041F40041818005AA08A94846FFF7A6FF76
:10BAD0000400DCD000970598029501950395049524
:10BAE0000188BDF81C300022504601F0A4F80A2C51
:10BAF00006D105AA06A94846FFF790FF0400ACD07E
:10BB0000ADF8185004E00598818821F40041818047
:10BB100005AA06A94846FFF781FF0028F3D00A2CA2
:10BB200003D020460AB0BDE8F0870020FAE710B540
:10BB30000C46896B86B051B10C218DF80010A18F95
:10BB4000ADF80810A16B01916946FAF74DF8002095
:10BB50004FF6FF71A063E187A08706B010BD2DE905
:10BB6000F0410D460746896B0020069E14460029C9
:10BB700011D0012B0FD1324629463846FFF762FF1C
:10BB8000002808D1002C06D0324629463846BDE8A8
:10BB9000F04100F034BFBDE8F0812DE9FC411446CE
:10BBA000DDE9087C0E46DDE90A15521DBCF800E00F
:10BBB00092B2964502D20720BDE8FC81ACF8002085
:10BBC00017222A70A5F80160A5F803300522CDE9F7
:10BBD00000423B462A46FFF7DFFD0020ECE770B548
:10BBE0000C46154648220021204601F0EEFB04F1E8
:10BBF000080044F81C0F00204FF6FF71E0616184DB
:10BC00002084A5841720E08494F82A0040F00A00DC
:10BC100084F82A0070BD4FF6FF720A8001460320A7
:10BC200008F0A8B830B585B00C460546FFF77FFF91
:10BC3000A18E284629B101218DF800106946F9F737
:10BC4000D3FF0020E0622063606305B030BDB0F830
:10BC5000400070476000002090F84620920703D40F
:10BC6000408808800020F4E70620F2E790F846209C
:10BC70009207EED5A0F84410EBE7014600200988B2
:10BC80000A0700D5012011F0F00F01D040F00200AA
:10BC9000CA0501D540F004008A0501D540F008002E
:10BCA0004A0501D540F010000905D2D540F020002A
:10BCB000CFE700B5034690F84600C00701D0062044
:10BCC00000BDA3F842101846FFF7D7FF10F03E0F53
:10BCD00005D093F8460040F0040083F8460013F8BE
:10BCE000460F40F001001870002000BD90F846207B
:10BCF000520700D511B1B0F84200AAE71720A8E713
:10BD000010F8462F61F3C3020270A2E72DE9FF4F3E
:10BD10009BB00E00DDE92B34DDE92978289D24D085
:10BD20002878C10703D000F03F00192801D901216C
:10BD300000E000212046FFF7D9FFB04215D3287854
:10BD4000410600F03F010CD41E290CD0218811F4CB
:10BD50007F6F0AD13A8842B1A1F57F42FF3A04D001
:10BD600001E0122901D1000602D504201FB0C5E56B
:10BD7000FA491D984FF0000A08718DF818A08DF847
:10BD80003CA00FAA0A60ADF81CA0ADF850A029781D
:10BD9000994601F03F02701F5B1C04F1180C4FF034
:10BDA000060E4FF0040BCDF858C01F2A7ED2DFE8F4
:10BDB00002F07D7D107D267DAC7DF47DF37DF27DEE
:10BDC000F17DF47DF07D7D7DEF7DEE7D7D7D7D7D62
:10BDD000ED0094F84610B5F80100890701D5032E4F
:10BDE00002D08DF818B01EE34FF40061ADF850108A
:10BDF000608003218DF83C10ADF84000D4E2052EA0
:10BE0000EFD1B5F801002083ADF81C00B5F80310A0
:10BE1000618308B1884201D9012079E10020A07234
:10BE200020814FF6FF702084169801F0D1F805208C
:10BE300089F800000220029083460AAB1D9A1699E9
:10BE40001B9801F0C8F890BB9DF82E00012804D083
:10BE5000022089F80100102003E0012089F8010088
:10BE600002200590002203A90BA805F000FFE8BB03
:10BE70009DF80C00059981423DD13988801CA1EBC9
:10BE80000B01814237DB02990220CDE900010DF15F
:10BE90002A034A4641461B98FFF77EFC02980BF1A5
:10BEA000020B801C81B217AA029101E09CE228E0FB
:10BEB00003A90BA805F0DBFE02999DF80C00CDE963
:10BEC000000117AB4A4641461B98FFF765FC9DF8F9
:10BED0000C000AAB0BEB00011FFA81FB02991D9AC3
:10BEE000084480B2029016991B9800E003E001F02C
:10BEF00072F80028B6D0BBF1020F02D0A7F800B04C
:10BF00004FE20A208DF818004BE200210391072E22
:10BF1000FFF467AFB5F801002083ADF81C00B5F859
:10BF20000320628300283FF477AF90423FF674AF5E
:10BF30000120A072B5F8050020810020A073E069FF
:10BF400000F04EFD78B9E16901208871E2694FF493
:10BF500020519180E1698872E16942F6010008810F
:10BF6000E06900218173F01F20841E986062072021
:10BF70006084169801F02CF8072089F80000012051
:10BF8000049002900020ADF82A0028E019E29FE119
:10BF900035E1E5E012E2A8E080E043E00298012804
:10BFA00014D0E0698079012803D1BDF82800ADF8EC
:10BFB0000E00049803ABCDE900B04A4641461B98F9
:10BFC000FFF7EAFB0498001D80B20490BDF82A0038
:10BFD000ADF80C00ADF80E00059880B202900AABE7
:10BFE0001D9A16991B9800F0F6FF28B90298398817
:10BFF000001D05908142D1D20298012881D0E069CC
:10C000008079012803D1BDF82800ADF80E0004980E
:10C0100003ABCDE900B04A4641461B98FFF7BCFB95
:10C020000298BDE1072E02D0152E7FF4DAAEB5F8E6
:10C0300001102183ADF81C10B5F80320628300299C
:10C040003FF4EAAE91423FF6E7AE0121A1724FF014
:10C05000000BA4F808B084F80EB0052E07D0C0B2CB
:10C06000691DE26905F001FE00287FF44AAF4FF632
:10C07000FF70208401A906AA14A8CDF800B081E8B9
:10C0800085032878214600F03F031D9A1B98FFF78F
:10C090009BFB8246208BADF81C0082E10120032E21
:10C0A000C3D14021ADF85010B5F801102183ADF88F
:10C0B0001C100AAAB8F1000F00D00023CDE902033A
:10C0C00004921D98CDF80480009038880022401E0C
:10C0D00083B21B9801F011F88DF8180090BB0B206B
:10C0E00089F80000BDF8280035E04FF0010C052E5E
:10C0F0009BD18020ADF85000B5F801102183B5F830
:10C1000003002084ADF81C10B0F5007F03D9072090
:10C110008DF8180087E140F47C4222840CA8B8F125
:10C12000000F00D00023CDE90330CDE9018C1D982C
:10C1300000903888401E83B21B9800F0DEFF8DF817
:10C14000180018B18328A8D10220BFE00D2189F87A
:10C150000010BDF83000401C22E10000600000200B
:10C16000032E04D248067FF53CAE002018E1B5F856
:10C170000110ADF81C102878400602D58DF83CE07F
:10C1800002E007208DF83C004FF000080320CDE9C5
:10C1900002081E9BCDF810801D980193A6F1030B99
:10C1A00000901FFA8BF342461B9800F044FD8DF877
:10C1B00018008DF83C80297849060DD52088C005E7
:10C1C00006D5208BBDF81C10884201D1C4F824800C
:10C1D00040468DF81880E3E0832801D14FF0020A31
:10C1E0004FF48070ADF85000BDF81C002083A4F817
:10C1F00020B01E986062032060841321CDE0052EDC
:10C20000FFF4EFADB5F80110ADF81C10A28F6AB3C2
:10C21000A2F57F43FE3B29D008228DF83C2000BFC9
:10C220004FF0000B0523CDE9023BDDF878C0CDF8D7
:10C2300010B01D9A80B2CDF804C040F400430092C3
:10C24000B5F803201B9800F0F6FC8DF83CB04FF4D5
:10C2500000718DF81800ADF85010832810D0F8B197
:10C26000A18FA1F57F40FE3807D0DCE00B228DF8CE
:10C270003C204FF6FE72A287D2E7A4F83CB0D2E091
:10C2800000942B4631461E9A1B98FFF784FB8DF8CD
:10C29000180008B183284BD1BDF81C00208353E758
:10C2A00000942B4631461E9A1B98FFF774FB8DF8BD
:10C2B0001800E8BBE18FA06B0844831D8DE888035C
:10C2C0004388828801881B98FFF767FC824668E0F4
:10C2D00095F80180022E70D15FEA080002D0B8F113
:10C2E000010F6AD109208DF83C0007A800908DF855
:10C2F00040804346002221461B98FFF730FC8DF812
:10C3000042004FF0000B8DF843B050B9B8F1010F67
:10C3100012D0B8F1000F04D1A18FA1F57F40FF38F2
:10C320000AD0A08F40B18DF83CB04FF4806000E09F
:10C3300037E0ADF850000DE00FA91B98F9F754FC59
:10C3400082468DF83CB04FF48060ADF85000BAF1F1
:10C35000020F06D0FC480068C07928B18DF818009B
:10C3600027E0A4F8188044E0BAF1000F03D0812040
:10C370008DF818003DE007A80090434601222146B1
:10C380001B98FFF7ECFB8DF8180021461B98FFF770
:10C39000CEFB9DF8180020B9192189F80010012062
:10C3A00038809DF83C0020B10FA91B98F9F71CFCC0
:10C3B0008246BAF1000F33D01BE018E08DF818E088
:10C3C00031E02078000712D5012E10D10A208DF817
:10C3D0003C00E088ADF8400003201B9907F0CAFC40
:10C3E0000820ADF85000C0E648067FF5FAAC4FF0E3
:10C3F000040A2088BDF8501008432080BDF8500082
:10C4000080050BD5A18FA1F57F40FE3806D11E987F
:10C41000E06228982063A6864FF0030A5046A5E400
:10C420009DF8180078B1012089F80000297889F872
:10C430000110BDF81C10A9F802109DF8181089F819
:10C440000410052038802088BDF8501088432080D3
:10C45000E4E72DE9FF4F8846087895B00121814037
:10C460004FF20900249C0140ADF820102088DDF82F
:10C470008890A0F57F424FF0000AFF3A06D039B10C
:10C48000000705D5012019B0BDE8F08F0820FAE7B4
:10C49000239E4FF0000B0EA886F800B018995D4659
:10C4A0000988ADF83410A8498DF81CB0179A0A71A4
:10C4B0008DF838B0086098F8000001283BD00228B9
:10C4C00009D003286FD1307820F03F001D30307044
:10C4D000B8F80400E08098F800100320022904D185
:10C4E000317821F03F011B31317094F84610090773
:10C4F00059D505ABB9F1000F13D0002102AA82E88B
:10C500000B000720CDE90009BDF83400B8F804108D
:10C51000C01E83B20022159800F0EFFD0028D1D193
:10C5200001E0F11CEAE7B8F80400A6F80100BDF844
:10C530001400C01C04E198F805108DF81C1098F840
:10C540000400012806D04FF4007A02282CD00328DA
:10C55000B8D16CE12188B8F8080011F40061ADF899
:10C56000201020D017281CD3B4F84010814218D3D3
:10C57000B4F84410172901D3814212D1317821F047
:10C580003F01C91C3170A6F801000321ADF8341039
:10C59000A4F8440094F8460020F0020084F8460015
:10C5A00065E105257EE177E1208808F1080700F4C0
:10C5B000FE60ADF8200010F0F00F1BD010F0C00F9F
:10C5C00003D03888228B9042EBD199B9B878C00754
:10C5D00010D0B9680720CDE902B1CDF804B00090C1
:10C5E000CDF810B0FB88BA883988159800F023FB85
:10C5F0000028D6D12398BDF82010401C80294ED0A9
:10C6000006DC10290DD020290BD0402987D124E049
:10C61000B1F5807F6ED051457ED0B1F5806F97D156
:10C62000DEE0C80601D5082000E0102082460DA9F2
:10C6300007AA0520CDE902218DF83800ADF83CB0FD
:10C64000CDE9049608A93888CDE9000153460722B0
:10C6500021461598FFF7B8F8A8E09DF81C200121A5
:10C660004FF00A0A002A9BD105ABB9F1000F00D0A8
:10C670000020CDE902100720CDE90009BDF8340003
:10C680000493401E83B2218B0022159800F035FDE3
:10C690008DF81C000B203070BDF8140020E09DF8D0
:10C6A0001C2001214FF00C0A002A22D113ABB9F152
:10C6B000000F00D00020CDE902100720CDE90009CD
:10C6C0000493BDF83400228C401E83B2218B159850
:10C6D00000F013FD8DF81C000D203070BDF84C00EB
:10C6E000401CADF8340005208DF83800208BADF8E3
:10C6F0003C00BCE03888218B88427FF452AF9DF823
:10C700001C004FF0120A00281CD1606AA8B1B8784A
:10C71000C0073FF446AF00E018E0BA680720CDE953
:10C7200002B2CDF804B00090CDF810B0FB88BA8802
:10C73000159800F080FA8DF81C001320307001204D
:10C74000ADF8340093E00000600000203988208BB1
:10C750008142D2D19DF81C004FF0160A0028A06B30
:10C7600008D0E0B34FF6FF7000215F46ADF808B087
:10C77000019027E068B1B978C907BED1E18F0DAB50
:10C780000844821D03968DE80C0243888288018844
:10C7900009E0B878C007BCD0BA680DAB03968DE845
:10C7A0000C02BB88FA881598FFF7F7F905005ED0F0
:10C7B000072D72D076E0019005AA02A92046FFF766
:10C7C0002DF90146E28FBDF80800824201D0002910
:10C7D000F1D0E08FA16B084407800198E08746E024
:10C7E0009DF81C004FF0180A40B1208BC8B1388862
:10C7F000208321461598FFF79AF938E004F11800D4
:10C800000090237E012221461598FFF7A8F98DF8A4
:10C810001C000028EDD1192030700120ADF8340043
:10C82000E7E7052521461598FFF781F93AE02088CA
:10C8300000F40070ADF8200050452DD1A08FA0F578
:10C840007F41FE3901D006252CE0D8F808004FF0D2
:10C85000160A48B1A063B8F80C10A1874FF6FF7113
:10C86000E187A0F800B002E04FF6FF70A087BDF8A6
:10C87000200030F47F611AD078230022032015991C
:10C8800007F0CEF998F8000020712088BDF820103C
:10C89000084320800EE000E007252088BDF8201026
:10C8A00088432080208810F47F6F1CD03AE02188D4
:10C8B000814321809DF8380020B10EA91598F9F721
:10C8C00093F905469DF81C000028EBD086F801A0DE
:10C8D00001203070208B70809DF81C003071052085
:10C8E000ADF83400DEE7A18EE1B118980DAB0088F9
:10C8F000ADF834002398CDE90304CDE90139206B6C
:10C900000090E36A179A1598FFF700FA0546012090
:10C910008DF838000EA91598F9F766F900B10546AB
:10C92000A4F834B094F8460040070AD52046FFF733
:10C93000A4F910F03E0F04D114F8460F20F00400C3
:10C9400020701898BDF83410018028469BE500B58A
:10C9500085B0032806D102208DF8000088B2694610
:10C96000F9F742F905B000BD10B5384C0B782268D4
:10C97000012B02D0022B2AD111E013780BB1052B29
:10C9800001D10423137023688A889A802268CB8897
:10C99000D38022680B891381498951810DE08B88EE
:10C9A00093802268CB88D38022680B8913814B89BE
:10C9B00053818B899381096911612168F9F714F911
:10C9C000226800210228117003D0002800D08120A5
:10C9D00010BD832010BD806B002800D0012070475F
:10C9E0008178012909D10088B0F5205F03D042F693
:10C9F0000101884201D10020704707207047F0B53F
:10CA000087B0002415460E460746ADF8184011E0E1
:10CA100005980088288005980194811DCDE9024180
:10CA2000072104940091838842880188384600F0E9
:10CA300002F930B905AA06A93046FEF7EFFF002833
:10CA4000E6D00A2800D1002007B0F0BD6000002029
:10CA500010B58B7883B102789A4205D10B885BB10F
:10CA600002E08B79091D4BB18B789A42F9D1B0F86D
:10CA700001300C88A342F4D1002010BD812010BDEC
:10CA8000072826D012B1012A27D103E0497801F006
:10CA9000070102E04978C1F3C20105291DD2DFE890
:10CAA00001F00318080C12000AB10320704702209D
:10CAB000704704280DD250B10DE0052809D2801E20
:10CAC000022808D303E0062803D0032803D005205A
:10CAD0007047002070470F20704781207047C0B218
:10CAE00082060BD4000607D5FA48807A4143C01D60
:10CAF00001EBD00080B270470846704700207047B5
:10CB000070B513880B800B781C0625D5F14CA47AE0
:10CB1000844204D843F010000870002070BD95686E
:10CB200000F0070605EBD0052D78F54065F30413FA
:10CB30000B701378D17803F0030341EA032140F22C
:10CB40000123B1FBF3F503FB15119268E41D00FB13
:10CB5000012000EBD40070BD906870BD37B514465D
:10CB6000BDF804101180117841F0040111709DF896
:10CB700004100A061ED5D74AA368C1F30011927AA1
:10CB8000824208D8FE2811D1D21DD2084942184647
:10CB900000F01BFC0AE003EBD00200F007030125C4
:10CBA00010789D40A843994008431070207820F0E9
:10CBB000100020703EBD2DE9F0410746C81C0E460E
:10CBC00020F00300B04202D08620BDE8F081C14DC4
:10CBD000002034462E60AF802881AA72E8801AE0D7
:10CBE000E988491CE980810614D4E17800F003004B
:10CBF00041EA002040F20121B0FBF1F201FB1201F9
:10CC00002068FFF76CFF2989084480B22881381A10
:10CC10003044A0600C3420784107E1D40020D4E7F0
:10CC2000AC4801220189C08800EB400002EB800083
:10CC3000084480B270472DE9FF4F89B01646DDE900
:10CC4000168A0F46994623F44045084600F054FBE7
:10CC5000040002D02078400703D401200DB0BDE8C5
:10CC6000F08F099803F01EFA02902078000606D58E
:10CC70009848817A0298814201D88720EEE72246BF
:10CC800001A90298FFF73CFF834600208DF80C00B5
:10CC90004046B8F1070F1AD001222146FFF7F0FEF7
:10CCA0000028DBD12078400611D502208DF80C0039
:10CCB000ADF81070BDF80400ADF81200ADF81460C6
:10CCC0001898ADF81650CDF81CA0ADF818005FEA22
:10CCD000094004D500252E46A84601270CE02178FE
:10CCE000E07801F0030140EA012040F20121B0FBAD
:10CCF000F1F2804601FB12875FEA494009D5B84549
:10CD000007D1A178207901F0030140EA0120B04267
:10CD100001D3BE4201D90720A0E7A8191FFA80F964
:10CD2000B94501D90D2099E79DF80C0028B103A958
:10CD30000998F8F757FF002890D1B84507D1A07897
:10CD40004FEA192161F30100A07084F804901A9849
:10CD500000B10580199850EA0A0027D0199830B11F
:10CD60000BEB06002A46199900F005FB0EE00BEBD1
:10CD700006085746189E099803F0FDFA2B46F61D43
:10CD8000B5B239464246009502F0F9FE224601A9A5
:10CD90000298FFF7B5FE9DF80400224620F010002F
:10CDA0008DF80400DDE90110FFF7D8FE002055E7FB
:10CDB0002DE9FF4FDFF81C91824685B0B9F80610C7
:10CDC000D9F8000001EB410100EB810440F20120A1
:10CDD000B2FBF0F1174600FB1175DDE9138B4E46EF
:10CDE00029460698FFF77BFE0346FFF719FF184414
:10CDF000B1880C30884202D9842009B02FE7069808
:10CE0000C6B2300603D5B00601D50620F5E7B9F85D
:10CE10000620521C92B2A9F80620BBF1000F01D0E7
:10CE2000ABF80020B00602D5C4F808800AE0B9F8D3
:10CE300008201A4492B2A9F80820D9F80000891AEB
:10CE40000844A0602246FE200699FFF787FEE7709F
:10CE500025712078390A61F301002A0AA17840F08F
:10CE6000040062F30101A17020709AF80200607161
:10CE7000BAF80000E08000252573300602D599F845
:10CE80000A7000E00127B00601D54FF000084E46B9
:10CE900000244FF007090FE0CDE902580195CDF8C5
:10CEA00000900495F1882046129B089AFFF7C3FE74
:10CEB0000028A2D1641CE4B2BC42EDD300209CE760
:10CEC00000B5FFF7ADFE03490C308A88904203D9C4
:10CED000842000BD94050020CA88086802EB420344
:10CEE00000EB8300521C037823F004030370CA8014
:10CEF000002101730846ECE72DE9F047804600F079
:10CF0000FBF9070005D000264446F74D40F2012901
:10CF100016E00120BDE8F087204600F0EDF9027828
:10CF2000C17802F0030241EA0222B2FBF9F309FBE5
:10CF300013210068FFF7D3FD3044641C86B2A4B20D
:10CF4000E988601E8142E7DCA8F10100E8802889B9
:10CF5000801B288100203870DCE710B5144631B101
:10CF6000491E218003F09EF8A070002010BD012012
:10CF700010BD70B50446DC48C188036801E0401C60
:10CF800020802088884207D200EB400213EB820207
:10CF900002D015786D07F2D580B2884216D2AAB1B8
:10CFA0005079A072D08820819178107901F0030126
:10CFB00040EA0120A081A078E11CFFF7A1FD2061DB
:10CFC0002088401C2080E080002070BD0A2070BDB9
:10CFD0000121018270472DE9FF4F85B04FF6FF799F
:10CFE0008246A3F8009048681E460D4680788DF86A
:10CFF000060048680088ADF8040000208DF80A009B
:10D00000088A0C88A04200D304462C8251E038786C
:10D01000400708D4641C288AA4B2401C288208F166
:10D020000100C0B246E0288A401C2882781D696849
:10D03000FFF70EFDD8BB3188494501D1601E308015
:10D040003188A1EB080030806888A04238D3B878D6
:10D05000397900F0030041EA002801A9781DFFF7A3
:10D06000F7FC20BB298949452ED000223946079874
:10D07000FFF706FDD8B92989414518D1E968039120
:10D08000B5F80AC0D7F808B05046CDF800C003F094
:10D0900072F9DDF800C05A460CF1070C1FFA8CFC3F
:10D0A00043460399CDF800C002F033FD60B1641C23
:10D0B000A4B200208046204600F01EF90700A6D149
:10D0C000641E2C820A2098E674807879B071F88802
:10D0D000B0803978F87801F0030140EA01207081CE
:10D0E000A6F80C80504602F0DDFF3A4606F1080132
:10D0F000FFF706FD306100207FE62DE9FF4F87B086
:10D1000081461C469246DDF860B0DDF854800898F0
:10D1100000F0F2F8050002D02878400702D4012080
:10D120000BB09CE5484602F0BDFF2978090605D5FD
:10D130006D49897A814201D88720F1E7CAF309064F
:10D140002A4601A9FFF7DCFC0746149807281CD0E3
:10D1500000222946FFF794FC0028E1D128784006F8
:10D1600013D501208DF808000898ADF80C00BDF823
:10D170000400ADF80E00ADF81060ADF8124002A941
:10D180004846F8F72FFD0028CAD12978E87801F041
:10D19000030140EA0121AA78287902F0030240EA5B
:10D1A0000220564507D0B1F5007F04D9611E8142A7
:10D1B00001DD0B20B4E7864201D90720B0E7801BD0
:10D1C00085B2A54200D92546BBF1000F01D0ABF8CE
:10D1D0000050179818B1B9192A4600F0CCF8B8F1E8
:10D1E000000F0DD03E4448464446169F03F0D5F844
:10D1F0002146FF1DBCB232462B46009402F0F3FCE0
:10D2000000208DE72DE9F04107461D4616460846E9
:10D2100000F072F8040002D02078400701D4012009
:10D22000D3E4384602F03EFF2178090605D52E49A1
:10D23000897A814201D88720C7E422463146FFF728
:10D240005FFC65B12178E07801F0030140EA01203C
:10D25000B0F5007F01D8012000E0002028700020F8
:10D26000B3E42DE9F04107461D461646084600F096
:10D2700043F8040002D02078400701D40120A4E440
:10D28000384602F00FFF2178090605D51649897A3C
:10D29000814201D8872098E422463146FFF75EFCA0
:10D2A000FF2D14D02178E07801F0030240EA02203B
:10D2B00040F20122B0FBF2F302FB130015B900F2B9
:10D2C000012080B2E070000A60F3010121700020AB
:10D2D0007BE410B50C4600F00FF810B10178490757
:10D2E00004D4012010BD000094050020C1882180D5
:10D2F0004079A0700020F5E70749CA88824209D327
:10D3000040B1096800EB40006FF00B0202EB8000B7
:10D3100008447047002070479405002070B504460B
:10D320000D4621462B460AB9002070BD01E0491C7C
:10D330005B1C501E021E03D008781E78B042F6D047
:10D3400008781E78801BF0E730B50C46014623466E
:10D35000051B954206D202E0521E9D5C8D54002AA8
:10D36000FAD107E004E01D780D70491C5B1C521EC9
:10D37000002AF8D130BDF0B50E460146334680EAAA
:10D38000030404F00304B4B906E002B9F0BD13F8D5
:10D39000017B01F8017B521E01F00307002FF4D13D
:10D3A0000C461D4602E080CD80C4121F042AFAD22A
:10D3B00021462B4600BF04E013F8014B01F8014B56
:10D3C000521E002AF8D100BFE0E7F0B50C46014636
:10D3D000E6B204E002B9F0BD01F8016B521E01F0A3
:10D3E0000307002FF6D10B46E5B245EA052545EACD
:10D3F000054501E020C3121F042AFBD2194602E0B2
:10D4000001F8016B521E002AFAD100BFE3E710B504
:10D4100006F001FFFAF784F906F0A6FDBDE810401A
:10D4200006F038BE202801D2012070470020704746
:10D4300001224FF0A043824011B1C3F80C25704780
:10D44000C3F8082570474FF0A04101228240C1F87F
:10D450001825704770B50346002002466FF02F056F
:10D460000EE09C5CA4F130060A2E02D34FF0FF3090
:10D4700070BD00EB800005EB4000521C2044D2B28E
:10D480008A42EED370BD30B50A230BE0B0FBF3F453
:10D4900003FB1404B0FBF3F08D183034521E05F872
:10D4A000014CD2B2002AF1D130BD30B500234FF685
:10D4B000FF7510E0040A44EA002084B2C85C6040B2
:10D4C000C0F30314604005EA00344440E0B25B1C42
:10D4D00084EA40109BB29342ECD330BDF94A1378F2
:10D4E00082F88B30A2F88C0082F88A10012082F832
:10D4F000880092F8640008B192F8600082F88E000B
:10D50000704710B50B46114658B11846FFF7E6FFB5
:10D51000ED488068008802F02EFFBDE8104002F060
:10D52000D5BBBDE810404FF6FF70D7E770B50026B9
:10D5300004464670E44D1120207029682022A01C6A
:10D540006831FFF718FF0121A171286800F8666FA4
:10D550008078002811D1DB48B0F86A20A0F892202A
:10D56000AA68537B80F8943080F89010108802F0FD
:10D5700002FFBDE8704002F0B8BB70BD70B5D24D7F
:10D58000296891F896200024012A11D091F8902062
:10D59000012A1CD091F86620012A22D091F8882017
:10D5A000012A21D091F8A020012A2ED0002070BDA0
:10D5B00044701722027051F8972FC0F802204A6871
:10D5C000C0F806200A7A827201F8014C1BE0447010
:10D5D00005220270D1F89220C0F8022081F8904014
:10D5E00011E0FFF7A3FF0EE091F86620012AF8D0C2
:10D5F00044701422027051F88A2FC0F802208A88E1
:10D60000C28001F8024C012070BD44701A2200F85B
:10D61000022B2222A131FFF7AEFE286880F8A0403D
:10D62000F1E7A948006890F8661011B1B0F86A00F7
:10D6300070474FF6FF70704770B5A34C206800B973
:10D64000FFDF2068417811B10C25284670BD002508
:10D65000C4222946FFF7B9FE2168FF2008707F2009
:10D6600081F8370013204884282081F865000120C4
:10D6700081F85C00002081F85F0007F0C6F906F031
:10D680009BFCE2E770B5904C0546206800B9FFDFCF
:10D690002168002048706560FFF7CEFF002800D0A9
:10D6A000FFDF70BD884909680978814201D10120F6
:10D6B000704700207047844800B5016891F8240045
:10D6C000498CC0F38002C0F340031A4400F001000B
:10D6D0001044132915D004DC102909D0122904D1D3
:10D6E0000FE0152908D01D2904D0FFDF002000BD60
:10D6F000764903E0764800BD7449083131F81000DE
:10D7000000BD72490839F9E76F4840F2712100689D
:10D71000806A484370476C48006890F836000028DB
:10D7200000D00120704710B5664C207B00F074FDDE
:10D7300040B1207D04F115010BF056FB082801D003
:10D74000012010BD207B30B1022804D00120BDE8AB
:10D75000104007F0BEBC0020F9E75A490873704733
:10D760005949096881F83000704770B50646554838
:10D7700090F82D000BF0C6FA050018D010210BF020
:10D7800098FD002813D1504C012032462168C876FC
:10D7900028461C3107F0AAFCD4E900101C310BF01C
:10D7A000E1FF6068BDE8704001210BF0EABF70BD89
:10D7B0002DE9F041434C074694F82D000BF01FFB78
:10D7C000064694F82F0004F10E0528B126B194F80E
:10D7D0002D000BF03AFAA0B194F83000002824D0C4
:10D7E00094F82E00002820D0607B294600F025FD0B
:10D7F000A8B10BF0ACFB3A462946BDE8F04107F072
:10D8000075BC012060733A462946304607F06EFC2D
:10D8100094F82D102846BDE8F0410BF087BB39463F
:10D820002846BDE8F04107F096BCBDE8F08170B530
:10D83000254C2168087BB0B1022814D00120487320
:10D840000E3107F030FC2068007B00F0E5FC216819
:10D8500081F82F00082081F82D00487B0E3100F060
:10D86000E3FC40B901E00020E9E72168487B0E3184
:10D8700000F0E3FC00B10120216881F82E0091F84E
:10D880002F0018B991F82200400706D5087D153100
:10D890000BF0AAFA216881F82D0020680025456068
:10D8A00004F0ADFD216888600020FFF781FF20684B
:10D8B000C57690F8220040070CD5BDE870400020E6
:10D8C00053E70000A00500206800002050B20100CE
:10D8D0009089130070BDFB4A1268137B0370D2F865
:10D8E0000E000860508A8880704778B5F649044673
:10D8F000F44D407B08732A68207810706088ADF87A
:10D90000000080B200F00101C0F3400341EA43018E
:10D91000C0F3800341EA8301C0F3C00341EAC301BD
:10D92000C0F3001341EA0311C0F3401341EA43116D
:10D93000C0F3801041EA80105084E07D012825D09A
:10D94000022825D0FFDF286880F85E60217B80F800
:10D950002410418C1D291DD061688162617D80F891
:10D960003610A17BC1B1022916D00121017554F8EE
:10D970000F1FC0F81510A188A0F81910217B0129EC
:10D9800000D0002180F83410002078BD0126DAE7AD
:10D990000226D8E70021E0E70021E7E7C948006850
:10D9A00090F82200C0F38000704700B5FFF7F6FF43
:10D9B00008B1002000BD1F2000BD00B5FFF7F5FF36
:10D9C000002800D0012000BDBE49002209680A6677
:10D9D0004B8C1D2B02D081F86400704781F86420C5
:10D9E0007047B84A0023126882F85D3042F84C1F35
:10D9F0009080012050747047B24A0023126882F868
:10DA00005C30A2F8580042F8541F01201072704791
:10DA1000AC49096881F835007047AA49096881F85E
:10DA20005F007047A748006890F95F007047A548FD
:10DA3000006890F8220000F001007047A1480068DB
:10DA400090F82200C0F340007047002070479D48C6
:10DA5000006890F82200C0F3C000704701207047B2
:10DA6000012070470120704770B500F0FAFB954C1B
:10DA70002068016E491C016690F83300002530B122
:10DA800006F0C3FF06F098FA206880F8335020684B
:10DA9000457090F8381009B102201AE090F864102F
:10DAA000B1B1006E814213D8022007F0ADFF2068AB
:10DAB00090F82200C00704D0A0684322018801200A
:10DAC00003E043224FF6FF710020BDE8704018E5E7
:10DAD0000020BDE8704007F097BF10B501280DD0B9
:10DAE00002280DD004280FD0FFDF7648006890F898
:10DAF0005E10BDE81040252006F00BBC252000E09C
:10DB0000262006F0E7FCF0E72720FAE7024600208F
:10DB1000D30701D0CB0705D0930705D58B0703D4D6
:10DB200002207047012070475207FCD54907FAD4FC
:10DB3000042070472DE9F041624C86B0206800B99E
:10DB4000FFDF20684178E9BB0178FF2942D000253A
:10DB500080F83150A0F85A50857080F83850284627
:10DB600006F0B4FE182259496846FFF704FC6846DF
:10DB700006F0A0FE06F0D9FB206890F95F0006F0E1
:10DB800099FC52481D3806F09BFC5048203806F09E
:10DB900082FE606806F09DFE2068002190F8240057
:10DBA000FFF7B4FFFFF799FF206880F82C5006F0CC
:10DBB00087FE206890F85E10002006F045FD0F21DA
:10DBC000052000E006E006F04CFC206890F82E10DE
:10DBD00051B902E00C2006B027E690F82F1019B9D1
:10DBE00090F8220040072BD504F009FC80462068FD
:10DBF0004146806805F004F9354F064690FBF7F082
:10DC000007FB10604142404604F0CDF8216888606F
:10DC100096FBF7F04A68104448600BF0E1F8216881
:10DC20004A6890420CD8C1E901580120FFF7C0FDB5
:10DC3000206890F82200400702D50120FFF795FDEB
:10DC40002068417B0E3006F0FEFB206890F85C10E7
:10DC500039B1B0F85810A0F84810416D416480F80F
:10DC60005C5090F85D1041B1B0F85010A0F8401031
:10DC7000C16C40F83C1F80F821500BF01EF90321C5
:10DC800060680BF051F9216881F833000020A2E7A9
:10DC90000C49886070472DE9F0410A4C0746002680
:10DCA00020683146C57E6068068000F0D1FA2068A1
:10DCB000408C132840D00DDC102861D012280DD1E3
:10DCC0005CE0000068000020A005002060B20100B8
:10DCD00040420F00152838D01D2836D0FFDF00BF86
:10DCE00000F0CAFA2068418C1D2907D0152905D0FB
:10DCF000B0F84820416C60680BF04AFD206890F84D
:10DD00002C1090F82400FFF701FF05463FB1FFF704
:10DD1000E4FE01224FF49671002006F033FD2068E6
:10DD200090F82C10294380F82C1090F824208A4376
:10DD30004FF0010129D02DE0002160680BF0E6FCD6
:10DD40000121606800F084FACAE7012160680BF0E5
:10DD5000DDFC0121606800F07BFAD4E9001025B1F8
:10DD60001C310BF0FFFC012104E015310BF0FAFC33
:10DD70002068017D60680BF004FDB1E7062100E03A
:10DD8000022160680BF0C2FCAAE7428C1D2A0BD06E
:10DD900080F831104170418C13290ED007DC102916
:10DDA0000AD0122907D108E080F82C60F2E7152983
:10DDB00003D01D2901D0FFDF37E590F85E20BDE8D4
:10DDC000F0410121084606F072BEF84810B500681F
:10DDD000417841B90078FF2805D00021084600F0BD
:10DDE00059FA002010BD00F03CFA0C2010BD2DE9BE
:10DDF000F041EE4D0446174628680E4690F866003E
:10DE000000B1FFDF2968002F81F868704ED12088AB
:10DE1000A1F86A006088A1F88000A088A1F88200BB
:10DE2000E088A1F8840094F88C0181F8860091F8CC
:10DE30002F0020B1487B0E3100F0FFF940B929686E
:10DE400091F8300060B1487B0E3100F0EDF938B147
:10DE50002868D0F80E104167418AA0F8781003E0D6
:10DE600028684767A0F878706968FF2E0878C0F3C3
:10DE700080106076D1F80300C4F81A00B1F80710DA
:10DE8000E18314D0296801F16E02C1F87A00E08BB9
:10DE9000A1F87E0030466D310AF0BBFF00B9FFDF0C
:10DEA000286810F86D1F41F002010170BDE4286878
:10DEB000C0F87A70A0F87E70617E80F86D10D4F89A
:10DEC0001A1040F86E1FE18B8180AEE470B5FFF749
:10DED000BEFDB64C012538B13C22FF21A068FFF7FA
:10DEE00086FF206880F86650206890F82200C007FE
:10DEF00004D0A0683C220188012003E03C224FF6B8
:10DF0000FF710020FFF7FDFA206880F8385070BDDF
:10DF1000A649096881F83200704770B5002507F0FE
:10DF2000D2FC50B1A14C20684178012908D00229C7
:10DF300001D0032936D0FFDF70BDBDE8704093E506
:10DF400081780029F8D1418C102913D090F8330042
:10DF500020B106F023F8402006F044FD206890F838
:10DF60002210490710D490F83610012904D0032953
:10DF700002D002E0002119E0102590F85E2045F063
:10DF80000E01002006F093FD206890F8340008B1DF
:10DF900006F06CFD0021962006F0C7FC21680220E7
:10DFA000487070BD81780029FBD18178BDE8704050
:10DFB000012000F06FB957E510B57C4C206890F84F
:10DFC000340008B100F07AF9206890F8330018B1F5
:10DFD00006F01BFD05F0F0FF07F075FC88B1206826
:10DFE0004078022800D0FFDF0021012000F052F924
:10DFF00020684178002903D04078012800D0FFDF55
:10E0000010BDBDE810402FE510B50AF0EDFE044646
:10E010000AF09FFF38B120460AF074FE18B11021B3
:10E020000BF047F908B1002010BD012010BD2DE90B
:10E03000F047DFF878910E460746032809D0FFF72E
:10E04000F6FC0446D9F8000090F8320020B1012017
:10E0500003E0FFF7F3FC04460020804606F02CFAAC
:10E060000546032F2BD0012734EA080453D0D9F8F2
:10E0700000004C4690F8330068B10AF004FF30709D
:10E080000146FF2807D06068C01C0AF0D9FE30782E
:10E090000AF003FF054360680178C1F3801221682C
:10E0A0000B7D9A4205D10622C01C1531FFF736F9C7
:10E0B00038B100203178FF290BD0D8B903E002270E
:10E0C000D2E70120F6E7206890F82D00884211D0B1
:10E0D00008E038B1616811F8030BC0F38010FFF756
:10E0E00093FF38B10020216891F82210490703D529
:10E0F000A0B910E00120F6E785B92D4890F8360068
:10E1000008B1B84207D1616811F8030BC0F3801061
:10E11000FFF77AFF10B10020BDE8F0870120FBE790
:10E12000F8B5224C0746002520684078022800D028
:10E13000FFDF206890F8340008B100F0BFF8606895
:10E140000BF006FB06460FB306F087F9F0B1052E7B
:10E150001DD1606890F8240000F01F00102816D927
:10E16000206890F8350090B1FF208DF8000001255F
:10E1700069460520FFF75BFF40B1206880F8A0509A
:10E1800061682222A130C91CFFF7F5F815E060682C
:10E190000BF01EFB88B1062E0FD2DFE806F00E0E44
:10E1A0000E030E0B00F0CDF806E000006800002022
:10E1B000A005002000F091F800B90125206890F832
:10E1C000330018B106F021FC05F0F6FE1DB1002168
:10E1D000012000F05FF820684178002906D04178DE
:10E1E000012903D04078032800D0FFDFF8BD70B5C7
:10E1F0009F4E05460C463068807800280BD106F00B
:10E200003CF803463068214690F85E202846BDE879
:10E21000704007F0D9BD70BD022803D0032801D09B
:10E220000020704701207047012802D148798009F9
:10E2300001D00020704701207047012806D148799D
:10E240000121B1EB901F01D10120704700207047E0
:10E250000278202322F0200203EA41110A430270CF
:10E26000704710B506F0B1FB06F08FFB06F0DEFA42
:10E27000BDE8104006F015BB10B57D4C7D496068C7
:10E280000BF06AFA7B480E38417B6068BDE81040AD
:10E290000BF06EBA764A10B5126892F831303BB185
:10E2A000508C1D2800D1FFDFBDE81040FFF7DCBB1C
:10E2B000002902D1BDE81040EDE410BD10B56C4C52
:10E2C0002068373006F0DDFB18B921687F2081F81F
:10E2D0003700BDE8104006F0BFBB38B5FF208DF811
:10E2E0000000012569460520FFF7A1FE30B3604C10
:10E2F0002068807808BB6268A0681278417BC2F30E
:10E30000401211404173012100F04AF800229DF8AB
:10E310000010A068FFF76BFD2068012100F8661F60
:10E32000827881880120FFF7ECF82168002048708E
:10E33000FFF797FF012007F067FB00E00025284664
:10E3400038BD38B5FF208DF800000125694603204F
:10E35000FFF76DFE464C002820681CD090F8341062
:10E3600031B190F8960018B99DF8000000F04CF813
:10E3700060680021018004210BF0C8F9FFF77CFFE1
:10E380002068B0F84020C16B60680BF011FA21687A
:10E390000320487002E0807800B90025284638BD87
:10E3A00070B5334D0446686850F80F2FC4F80E203E
:10E3B0008288628282792275C27962750289E282DC
:10E3C000428962808289A280C289E2800269A26059
:10E3D000027D2273427D02F01F022276407D4009B9
:10E3E00084F88C0184F8641084F86510002104F12D
:10E3F00030000BF04CFB286890F8651004F8661F9D
:10E4000090F85F00607070BD70B5194C01222168F2
:10E4100081F896200A7881F89720FF280DD001F125
:10E42000990298310AF0F5FC00B9FFDF206810F876
:10E43000981F41F0020101700CE060680278C2F39D
:10E44000801281F89820D0F8032041F8992FB0F875
:10E4500007008880256895F837009F357F2800D110
:10E46000FFDF206810F8371F29707F21017070BD11
:10E4700068000020AE0500202DE9FC470C4606464A
:10E48000694600F019FF002860D1FFF7CAF8B042D2
:10E490005CD02146304609F021F828BB019D95F853
:10E4A0002C01703518B9287F08B1012000E0002048
:10E4B000814695F839004FF000084FF0010AA0B1ED
:10E4C00095F83A00800710D584F8018084F800A000
:10E4D00084F80280A68095F83B10A171A98F218154
:10E4E000E98F618185F839802DE0304601F055FFD4
:10E4F000070000D1FFDF384601F075F940B184F81C
:10E5000001800D212170A680E08084F802A01AE02D
:10E51000304601F030FF070000D1FFDFB9F1000FF6
:10E5200014D0384601F0B7F980B1304606F036FD18
:10E5300084F801800A21217084F80280A680697F16
:10E54000A17185F81C800120BDE8FC870020FBE755
:10E550001CB5694600F0B0FE00B1FFDF684600F070
:10E56000B8FEF94900208968A1F8F2001CBD2DE928
:10E57000FC4104460E46062001F076FD00250746C4
:10E58000A846064417E02088401C80B22080B04294
:10E5900002D34046A4F8008080B2B84204D3B0420F
:10E5A00002D20020BDE8FC81694600F085FE00280B
:10E5B000F8D06D1CEDB2AE42E5D84FF6FF7020806A
:10E5C0001220EFE710B506F05BFD0AF048FBDF48CC
:10E5D0004FF6FF7100234182818203701B2141802D
:10E5E0004FF4A4728280C180028103228275C275B9
:10E5F00082720424C4728181C1810282837610BD3B
:10E6000070B5D14C0D466060217006F0C5FC00F07D
:10E610006CFEFFF7D7FF207809F0B4FD284607F01D
:10E6200065FACA482838FFF72DF82178606809F0A4
:10E630003AF8BDE870400AF012BB10B501240AB1E7
:10E64000002010BD21B1012903D00024204610BDB7
:10E6500002210BF0EDF8F9E7887800B90320C978BA
:10E6600001B90321107019700020704730B587B0D0
:10E6700004460088694600F01FFE002806D1A088E5
:10E6800030B1012804D0022802D0122007B030BDDA
:10E6900005AB04AA21466846FFF7DEFF0400F5D16A
:10E6A0000199012081F8C501019991F81012002506
:10E6B00039B9019991F8C41119B9019991F89710D4
:10E6C00009B13A2415E00199039581F8C401019834
:10E6D0009DF8102080F8C621019B9DF8140083F856
:10E6E000C7018DF80C208DF80D0003AA01200AF057
:10E6F00016FF019880F8C5512046C7E710B50446BB
:10E700000020A17801B90120E2780AB940F00200A6
:10E7100000F0FFFD002803D12046BDE81040A5E72A
:10E7200010BD70B50D4604460189002380880AF0AB
:10E73000EBFE696A81421DD2401A401CA188400844
:10E74000091A8AB2A2802189081A2081668895F860
:10E75000641010460AF0AFFE864200D23046608058
:10E76000E68895F8651020890AF0A5FE864200D259
:10E770003046E08070BDF0B585B00D46064603A971
:10E7800000F09AFD00282AD104990022FB20B1F85C
:10E790004E30FB2B00D30346B1F85040FB20FB2C3E
:10E7A00000D30446DFF8A8C19CE8811000900197CF
:10E7B000CDF808C0ADF80230ADF806406846FFF766
:10E7C000B0FF6E80BDF80400E880BDF808006881E5
:10E7D000BDF80200A880BDF806002881002005B021
:10E7E000F0BD2DE9F04186B004460088694600F08E
:10E7F00063FD002859D12189E08800F0A4FD00289C
:10E8000053D1A188608800F09EFD00284DD1218958
:10E81000E08800F08EFD002847D1A188608800F0D4
:10E8200088FD060041D1208802A9FFF7A4FF00B1AE
:10E83000FFDFBDF8101062880920914235D3BDF882
:10E840000C10E288914230D3BDF81210BDF80E20B2
:10E8500023891144A2881A44914226D3019D01279D
:10E860004FF0000885F8BB71019890F8FC0105F5A0
:10E87000DD7508B13A2615E0E08868806088E88098
:10E88000218940F64800814200D30146A980A18831
:10E89000814200D208462881002228460199FFF7CC
:10E8A00040FF2F7085F80180304606B0BDE8F0814A
:10E8B00097E710B50446FEF761FE002813D02078D4
:10E8C00014280FD1A07868B1A088062101F020FC9F
:10E8D00040B1008806F062FBA088062101F02AFC06
:10E8E00000B1FFDF012010BD2DE9F041060000D18D
:10E8F000FFDF1648022114308046FFF738FE00B1D2
:10E90000FFDF124C0620A78A01F0AEFB0546A08A65
:10E91000A84203D13046FFF7CCFF20B9A08A314688
:10E92000FFF7AAFD30B1304600F01BFD0028EED104
:10E930000120BBE702214046FFF719FE10B9A08A6B
:10E94000B842E4D10020B1E7740000208C0600201A
:10E9500078B2010010B500F08BFC08B10C2010BD9E
:10E960000AF0B8F9002010BD10B50446007818B1BF
:10E97000012801D0122010BD00F08AFC20B10AF05D
:10E980001FFA08B10C2010BD207800F05BFCE21DDE
:10E9900004F11703611CBDE810400AF0BDB910B5C1
:10E9A000044600F065FC08B10C2010BD207818B1B9
:10E9B000012801D0122010BD00F044FC611C0AF0B7
:10E9C00063F908B1002010BD072010BD10B50AF092
:10E9D000FBF908B1002010BD302010BD10B5044671
:10E9E00000F056FC08B10C2010BD20460AF0E4F9F6
:10E9F000002010BD10B500F04BFC20B10AF0E0F98A
:10EA000008B10C2010BD0AF0C9F9002010BDFF218B
:10EA100081704FF6FF718180F94949680A788271E7
:10EA20008A88028149884181012141700020704714
:10EA30001CB50024022A19D015DC12F10C0F15D0D8
:10EA400009DC12F1280F11D012F1140F0ED012F1BF
:10EA5000100F0FD10AE012F1080F07D012F1040FC6
:10EA600004D03AB902E0D31E052B03D8012804D004
:10EA7000032806D0122420461CBD1046FEF7CDFF09
:10EA8000F9E708461446694600F016FC08B102246E
:10EA9000F1E7019880F867400024ECE710B51346D1
:10EAA00001220AF022FC002010BD10B5044600F03F
:10EAB000EFFB08B10C2010BD2146002006F0E1FA62
:10EAC000002010BD10B5044607F0AAF920B1207847
:10EAD00007F018F8002010BD0C2010BD10B504463A
:10EAE00000F0D6FB08B10C2010BD2146012006F035
:10EAF000C8FA002010BD38B504464FF6FF70ADF8D7
:10EB00000000A079E179884216D02079FEF78AFCCE
:10EB100090B16079FEF786FC70B10022A0791146B1
:10EB20000BF0FAFB40B90022E07911460BF0F4FB40
:10EB300010B9207A072801D9122038BD07F07CF9D6
:10EB400048B900216846FFF712FD20B1204605F0C4
:10EB5000B7FB002038BD0C2038BD2DE9FC41817881
:10EB600004461A2925D00EDC16292DD2DFE801F043
:10EB70002C2C2C2C2C212C2C2C2C2C2C2C2C2C2CE0
:10EB80002C2C2C2121212A291ED00BDCA1F11E01C5
:10EB90000C2919D2DFE801F01818181818181818DD
:10EBA0001818180D3A3904290ED2DFE801F00D02C9
:10EBB0000D022088B0F5706F06D20127694600F07B
:10EBC0007BFB18B10220EDE41220EBE4019D6846C6
:10EBD0002E4605F5C87506F2911600F060FB08B1E7
:10EBE000287808B10C20DDE42F70A07830706846DA
:10EBF00000F06FFB0020D5E41CB50C46694600F020
:10EC00005BFB002118B12160217102201CBD01981D
:10EC10000246703080F8421093682360137B2371A2
:10EC200090F84230002BF5D100201CBD10B50446F1
:10EC300000F02EFB20B10AF0C3F808B10C2010BD83
:10EC4000207800F0FFFAE279611C0AF08EF908B131
:10EC5000002010BD022010BD10B5886E60B10022EA
:10EC600041F8682F0120CA71897988400BF048FB70
:10EC7000002800D01F2010BD0C2010BD1CB50C4674
:10EC8000694600F019FB002805D10198B0F8700022
:10EC9000401C208000201CBD1CB50446008869462D
:10ECA00000F00AFB08B102201CBD606828B1DDE954
:10ECB0000001224600F0A3FB1CBDDDE90001FFF7C7
:10ECC000CBFF1CBD10B50078012800D00020FEF756
:10ECD0009FFE002010BDF0B544888188C28803895A
:10ECE00045898089A71F40F67B46B74215D28F1F02
:10ECF000B74212D28C4210D8B2F5FA7F0DD2A3F1EE
:10ED00000A04361FB44208D2521C4A43B2EB830FA6
:10ED100003DA854201D80020F0BD3020F0BDF8B5FF
:10ED200015460E46044607F087F808B10C20F8BDDA
:10ED3000204600F0A3FB0028F9D1A078C1064FF0CF
:10ED40001100F4D5E17D0329F1D0FEF76BFE3070A0
:10ED5000A07555B9FF208DF8000069460020FEF728
:10ED60004BFE69460020FEF73CFE2046BDE8F84019
:10ED7000FEF7BBBD0022D2E70078C10801D0122007
:10ED80007047204988760020704710B50446007807
:10ED9000C00704D1608810B1FEF70FFE80B1207863
:10EDA000618800F00102607800F0B3FB002806D112
:10EDB000FEF7FBFD01466088884203D9072010BD9D
:10EDC000122010BD6168FEF717FE002010BD10B5BF
:10EDD00004460078C00704D1608810B1FEF72EFE0B
:10EDE00090B12078618800F00102607800F091FB1A
:10EDF000002804D160886168FEF7F3FD002010BD93
:10EE0000740000208C0600201220F8E77CB5044630
:10EE100040784225012808D8A078FEF743FC20B1AD
:10EE200020781225012802D090B128467CBDFEF73B
:10EE30000EFE20B1A0880028F7D08028F5D8FEF774
:10EE40000DFE60B160780028EFD02078012808D04E
:10EE500006F094F9044606F01FFE00287FD00C202F
:10EE60007CBDFEF760FC10B9FEF7EFFD90B306F035
:10EE7000E3FF0028F3D1FEF7D4FBA0F57F41FF3973
:10EE8000EDD1FEF7D4FCA68842F210704643A0797B
:10EE9000FEF79AFDFEF7CBFDF8B10022062101A88E
:10EEA00001F008F9040058D0F7480021846020469A
:10EEB0000AF03EF92046FEF7EBFEF44D04F1300077
:10EEC000AA89E989C2830184FEF7CAFD60B1288A54
:10EED00001210DE0FFE712207CBD3146002006F045
:10EEE00014FE88B3FFDF44E0FEF7BCFD0146288A2C
:10EEF00006F0A6FE0146A0620022204606F041F977
:10EF0000FEF7AEFD38B9FEF7ADFD02462146012001
:10EF10000AF003FBD0B1DD4A2146163201200AF087
:10EF2000FEFAE87A0090AB7AEA89A989208801F094
:10EF3000ABF900B1FFDF208806F02FF831462046FC
:10EF400006F0E3FD00B1FFDF13E008E00621BDF8A5
:10EF5000040001F0EFF800B1FFDF09207CBD44B1EF
:10EF6000208806F01BF82088062101F0E3F800B1A4
:10EF7000FFDF00207CBD002148E770B50D4606216B
:10EF800001F0C6F8040003D094F8930110B10AE030
:10EF9000022070BD94F87D00142801D0152802D1FC
:10EFA00094F8E00108B10C2070BD1022294604F548
:10EFB000CA70FEF7E0F9012084F89301002070BDCB
:10EFC00010B5062101F0A4F818B190F8931111B111
:10EFD00007E0022013E790F87D10142903D01529CB
:10EFE00001D00C200BE7022180F89311002006E7E6
:10EFF0002DE9FC410D464BF680321221954213D883
:10F0000095B1694600F058F900280CD1019EB41C56
:10F01000703627882A46394630460AF04AF8208852
:10F02000B842F6D10020CEE50846CCE51CB5044632
:10F030000088694600F040F9002808D10199A378BA
:10F04000084691F82C2070319A4201D10C201CBD49
:10F050007F220A728A720022CA72E17880F82D102B
:10F06000217980F82E10A17880F82C1010461CBD54
:10F070001CB50C46694600F01FF9002806D101981E
:10F0800090F88C0000B10120207000201CBD7CB5E0
:10F090000D461446694600F00FF9002805D1019885
:10F0A00090F82C00012801D00C207CBD019890F82C
:10F0B0007810297090F87900207000207CBD70B520
:10F0C0000D461646062101F023F818B38188012465
:10F0D000C388428804EB4104AC4217D842F2107452
:10F0E0006343A4106243B3FBF2F2521E94B24FF496
:10F0F000FA72944200D91446A54200D22C46491C0B
:10F10000641CB4FBF1F24A43521E91B290F8CC2138
:10F110001AB901E0022070BD01843180002070BD69
:10F1200010B50C46062100F0F3FF48B180F8FF400F
:10F1300024B190F8FD1009B106F099FD00205EE6BB
:10F1400002205CE6017899B1417889B141881B2998
:10F150000ED381881B290BD3C188022908D34B49C0
:10F160000268283941F8322F406848600020704713
:10F170001220704710B506F034FD00203FE610B5B0
:10F1800006F032FD00203AE670B514460A460646FF
:10F1900000250121104606F053FD002800D828461E
:10F1A00005460121304600F054F8064601210020B2
:10F1B00000F04FF83118012296318D4206D901F145
:10F1C0009600691AB1FBF0F0401C82B22280002048
:10F1D00070BD10B5044600F05BF808B10C200EE6D7
:10F1E000601C09F0AFFE207800F00100FEF7B8FACD
:10F1F000002004E610B50446062000F027FF08B101
:10F200000C20FCE52078C00710D000226078114661
:10F210000BF082F808B11220F1E5A06808F0B5FD06
:10F220006078616808F0BAFD0020E8E5002008F089
:10F23000ACFD00210846F5E710B5006805F01AF8A6
:10F240000020DCE518B1022801D001207047002021
:10F25000704710B5012904D0022905D0FFDF2046F0
:10F26000CDE5C000503001E080002C3084B2F6E7DC
:10F2700010B506F0E1FD20B1FEF74DFA08B101200E
:10F28000BDE50020BBE50000740000208C060020D6
:10F2900010B506F0D1FD002800D00120AFE541688F
:10F2A00091F82C0191F88C1021B918B1042801D0E3
:10F2B000012070470020704710B50C46062100F071
:10F2C00027FF606018B101202070002097E5022020
:10F2D00095E5416891F8FD20002A05D0002281F8CB
:10F2E000FD20406806F0C3BC704708B54FF6FF70BC
:10F2F000ADF8000006E00621BDF8000000F01AFF9E
:10F3000000B1FFDF00216846FFF731F90028F2D095
:10F3100008BD70B514460546012200F00EF900281C
:10F3200006D121462846BDE87040002200F005B90C
:10F3300070BDFB2803D840F64800814201D9112056
:10F340007047002070471B38E12806D2B1F5A47F32
:10F3500003D344F29020814201D91220704700204B
:10F3600070471FB58D49897ECA0702D10278192AD4
:10F370000AD08A0702D40278182A24D0490739D43F
:10F380000178122933D035E04088ADF8000002A999
:10F39000FFF792FF00B1FFDF039810F8601F8DF8B0
:10F3A000021040788DF803000020ADF8040001B988
:10F3B000FFDF9DF8030000B9FFDF6846FFF79EF905
:10F3C000D8B1FFDF19E04088ADF8000040F64800F2
:10F3D000FB21ADF80400ADF80800ADF80210ADF85F
:10F3E00006106846FFF764FA38B1FFDF05E0007BDE
:10F3F000C00702D0002004B001E50120FBE7F8B50A
:10F400000646508914460F4640B1B0F5004F05D26C
:10F410000022A07811460AF07FFF08B11220F8BD43
:10F42000B86E394607F1700530B1A07891F86E20BA
:10F43000904201D00C20F8BD012081F86F00A07827
:10F4400081F86E00606841F8680F608988802089C3
:10F45000A884002087F86F0020886946FFF70EFC1B
:10F46000A88CBDF80010081A00B2002804DD394647
:10F470003046FFF7F1FBDDE70020F8BD38B5044664
:10F480000078EF2841D86088ADF80000009800F0BF
:10F4900061F888B36188080708D4D4E90120824262
:10F4A00033D8202A31D3B0F5804F2ED8207B18B323
:10F4B00007282AD8607B28B1012803D0022801D070
:10F4C000032822D14A0703D4022801D0032805D1FA
:10F4D000A07B08B1012818D1480707D4607D28B166
:10F4E000012803D0022801D003280ED1C806E07DF0
:10F4F00003D5012809D104E007E0012801D0032841
:10F5000003D1E07E18B1012801D0122038BD0020BF
:10F5100038BD70B50C460546FF2904D8FEF7A0FAA1
:10F5200018B11F2C01D9122070BD2846FEF7BAF879
:10F5300008B1002070BD422070BD0AB1012200E078
:10F540000222024202D1880802D109B1002070478C
:10F550001120704780B2C1060BD401071CD481066C
:10F560004FEAC07101D5B9B900E099B1800713D451
:10F5700010E0410610D481060ED4C1074FEA807115
:10F5800004D0002902DB400704D405E0010703D4BE
:10F59000400701D401207047002070478C060020EE
:10F5A00030B5058825F4004421448CB24FF4004165
:10F5B00094420AD2121B92B21B339A4201D2A9433F
:10F5C00007E005F40041214303E0A21A92B2A943E7
:10F5D0001143018030BD0844083050434A3108448B
:10F5E00080B2704770B51D4616460B460446294644
:10F5F0003046049AFFF7EFFF0646B34200D2FFDF22
:10F60000282200212046FDF7E0FE4FF6FF70A08281
:10F61000283EB0B265776080B0F5004F00D9FFDFBB
:10F62000618805F13C00814200D2FFDF6088083527
:10F63000401B343880B220801B2800D21B20208041
:10F640000020A07770BD8161886170472DE9F05F6F
:10F650000D46C188044600F12809008921F40046BE
:10F6600020F4004800F063FB10B10020BDE8F09FDB
:10F670004FF0000A4FF0010BB0450CD9617FA8EBA9
:10F680000600401A0838854219DC09EB0600002103
:10F69000058041801AE06088617F801B471A083F1F
:10F6A0000DD41B2F00DAFFDFBD4201DC294600E04C
:10F6B000B9B2681A0204120C04D0424502DD84F883
:10F6C00017A0D2E709EB06000180428084F817B04A
:10F6D000CCE770B5044600F12802C088E37D20F431
:10F6E00000402BB110440288438813448B4201D25E
:10F6F000002070BD00258A4202D30180458008E0C9
:10F70000891A0904090C418003D0A01D00F01FFBD9
:10F7100008E0637F00880833184481B26288A01D26
:10F72000FFF73EFFE575012070BD70B5034600F19F
:10F730002804C588808820F400462644A84202D1C7
:10F740000020188270BD98893588A84206D3401BD6
:10F7500075882D1A2044ADB2C01E05E02C1AA5B242
:10F760005C7F20443044401D0C88AC4200D90D80A1
:10F770009C8924B1002414700988198270BD012469
:10F78000F9E770B5044600F12801808820F40040B4
:10F790004518208A002825D0A189084480B2A0817C
:10F7A00029886A881144814200D2FFDF288869884D
:10F7B00000260844A189884212D1A069807F28715F
:10F7C000698819B1201D00F0C2FA08E0637F28881B
:10F7D0000833184481B26288201DFFF7E1FEA6813C
:10F7E0002682012070BD2DE9F041418987880026DD
:10F7F000044600F12805B94219D004F10A0800BFF7
:10F8000021F400402844418819B1404600F09FFA95
:10F8100008E0637F00880833184481B2628840465C
:10F82000FFF7BEFE761C6189B6B2B942E8D1304618
:10F83000BDE8F0812DE9F04104460B4627892830C8
:10F84000A68827F40041B4F80A8001440D46B74267
:10F8500001D10020ECE70AB1481D106023B1627F9E
:10F86000691D1846FDF787FD2E88698804F1080098
:10F8700021B18A1996B200F06AFA06E0637F6288C5
:10F880000833991989B2FFF78BFE474501D12089CA
:10F8900060813046CCE78188C088814201D1012057
:10F8A00070470020704701898088814201D1012082
:10F8B00070470020704770B58588C38800F1280420
:10F8C00025F4004223F4004114449D421AD0838958
:10F8D000058A5E1925886388EC18A64214D313B1F3
:10F8E0008B4211D30EE0437F08325C1922444088DA
:10F8F00092B2801A80B22333984201D211B103E050
:10F900008A4201D1002070BD012070BD2DE9F04771
:10F910008846C1880446008921F4004604F128077E
:10F9200020F4004507EB060900F001FA002178BB3E
:10F93000B54204D9627FA81B801A002503E06088C5
:10F94000627F801B801A083823D4E28962B1B9F83B
:10F950000020B9F802303BB1E81A2177404518DBA6
:10F96000E0893844801A09E0801A217740450ADB93
:10F97000607FE1890830304439440844C01EA4F84F
:10F980001280BDE8F087454503DB01202077E7E7DB
:10F99000FFE761820020F4E72DE9F74F044600F10C
:10F9A0002805C088884620F4004A608A05EB0A06CC
:10F9B00008B1404502D20020BDE8FE8FE08978B151
:10F9C0003788B6F8029007EB0901884200D0FFDFC4
:10F9D000207F4FF0000B50EA090106D088B33BE0CE
:10F9E0000027A07FB9463071F2E7E18959B1607F05
:10F9F0002944083050440844B4F81F1020F8031D6F
:10FA000094F821108170E28907EB080002EB0801ED
:10FA1000E1813080A6F802B002985F4650B1637F62
:10FA200030880833184481B26288A01DFFF7B8FD02
:10FA3000E78121E0607FE18908305044294408448F
:10FA40002DE0FFE7E089B4F81F102844C01B20F820
:10FA5000031D94F82110817009EB0800E28981B23E
:10FA600002EB0800E081378071800298A0B1A01DF0
:10FA700000F06DF9A4F80EB0A07F401CA077A07D27
:10FA800008B1E088A08284F816B000BFA4F812B0D4
:10FA900084F817B001208FE7E0892844C01B30F8B4
:10FAA000031DA4F81F10807884F82100EEE710B53C
:10FAB000818800F1280321F400442344848AC28809
:10FAC000A14212D0914210D0818971B9826972B17C
:10FAD0001046FFF7E8FE50B91089283220F40040A4
:10FAE000104419790079884201D1002010BD1846D0
:10FAF00010BD00F12803407F08300844C01E10608C
:10FB0000088808B9DB1E136008884988084480B259
:10FB100070472DE9F04100F12806407F1C4608306F
:10FB20009046431808884D88069ADB1EA0B1C01C79
:10FB300080B2904214D9801AA04200DB204687B2DE
:10FB400098183A464146FDF7E9FB002816D1E01B1C
:10FB500084B2B844002005E0ED1CADB2F61EE8E723
:10FB6000101A80B20119A94206D8304422464146F3
:10FB7000BDE8F041FDF7D2BB4FF0FF3058E62DE96C
:10FB8000F04100F12804407F1E460830904643189B
:10FB9000002508884F88069ADB1E90B1C01C80B2F1
:10FBA000904212D9801AB04200DB304685B29918D3
:10FBB0002A464046FDF7DFFB701B86B2A8440020B2
:10FBC00005E0FF1CBFB2E41EEAE7101A80B28119FB
:10FBD000B94206D8211832464046FDF7CCFBA81999
:10FBE00085B2284624E62DE9F04100F12804407F43
:10FBF0001E46083090464318002508884F88069A0C
:10FC0000DB1E90B1C01C80B2904212D9801AB04263
:10FC100000DB304685B298182A464146FDF7ABFB1B
:10FC2000701B86B2A844002005E0FF1CBFB2E41E92
:10FC3000EAE7101A80B28119B94206D82044324648
:10FC40004146FDF798FBA81985B22846F0E5401D0E
:10FC5000704710B5044600F12801C288808820F45E
:10FC600000431944904206D0A28922B9228A12B9CF
:10FC7000A28A904201D1002010BD0888498831B184
:10FC8000201D00F064F800202082012010BD637F59
:10FC900062880833184481B2201DFFF781FCF2E727
:10FCA0000021C18101774182C17581757047038848
:10FCB0001380C28942B1C28822F4004300F12802B5
:10FCC0001A440A60C08970470020704710B5044686
:10FCD000808AA0F57F41FF3900D0FFDFE088A08255
:10FCE000E08900B10120A07510BD4FF6FF7181823F
:10FCF00000218175704710B50446808AA0F57F41C8
:10FD0000FF3900D1FFDFA07D28B9A088A18A8842F1
:10FD100001D1002010BD012010BD8188828A91424E
:10FD200001D1807D08B1002070470120704720F488
:10FD3000004221F400439A4207D100F4004001F44C
:10FD40000041884201D0012070470020704730B543
:10FD5000044600880D4620F40040A84200D2FFDF90
:10FD600021884FF4004088432843208030BD70B57F
:10FD70000C00054609D0082C00D2FFDF1DB1A1B24E
:10FD8000286800F044F8201D70BD0DB100202860E7
:10FD9000002070BD0021026803E0938812681944B6
:10FDA00089B2002AF9D100F032B870B500260D46AC
:10FDB0000446082900D2FFDF206808B91EE0044687
:10FDC00020688188A94202D001680029F7D1818882
:10FDD0000646A94201D100680DE005F1080293B280
:10FDE0000022994209D32844491B0260818021687E
:10FDF000096821600160206000E00026304670BD87
:10FE000000230B608A8002680A600160704700234B
:10FE10004360021D018102607047F0B50F46018802
:10FE2000408815460C181E46AC4200D3641B304473
:10FE3000A84200D9FFDFA019A84200D9FFDF381976
:10FE4000F0BD2DE9F04188460646018840881546F8
:10FE50000C181F46AC4200D3641B3844A84200D99A
:10FE6000FFDFE019A84200D9FFDF708838447080B6
:10FE700008EB0400BDE8F0812DE9F041054600885B
:10FE80001E461746841B8846BC4200D33C442C8047
:10FE900068883044B84200D9FFDFA019B84200D9C1
:10FEA000FFDF68883044688008EB0400E2E72DE952
:10FEB000F04106881D460446701980B217468846F0
:10FEC0002080B84201D3C01B20806088A84200D2A5
:10FED000FFDF7019B84200D9FFDF6088401B6080E7
:10FEE00008EB0600C6E730B50D460188CC189442F1
:10FEF00000D3A41A4088984200D8FFDF281930BDEB
:10FF00002DE9F041BF4D04469046A8780E46A04228
:10FF100000D8FFDF05EB8607786A50F8240000B1AF
:10FF2000FFDFB868002816D0304600F032F90146ED
:10FF3000B868FFF73AFF05000CD0786A072E40F842
:10FF4000245000D3FFDFB0484246294650F82630FF
:10FF5000204698472846BDE8F0812DE9F843050082
:10FF60000C46009524D00026E81C20F00300A8428F
:10FF700000D0FFDFDFF88C820027314688F8007060
:10FF800088F8014088F8024088F8034088F8044067
:10FF900088F8054088F80640684600F003F900201C
:10FFA00042460099C91C21F00301009116B10FE0EF
:10FFB0000126D9E702EB80035962002106E000BF69
:10FFC000D3F824C04CF82170491CC9B2A142F7D320
:10FFD0000099401C01EB8401C0B200910728E0D3D6
:10FFE000481BBDE8F88310B50446F1F74AF908B19B
:10FFF000102010BD2078834A618802EB800092783F
:020000040001F9
:100000000EE0436A53F8213043B14A1C6280A1805C
:10001000406A50F82100A060002010BD491C89B240
:100020008A42EED86180052010BD70B505460C46A9
:100030000846F1F726F908B1102070BD072D01D34D
:10004000072070BD25700020608070BD0EB5694628
:10005000FFF7EBFF00B1FFDF6846FFF7C4FF08B111
:1000600000200EBD01200EBD10B50446072800D3A8
:10007000FFDF6448005D10BD3EB5054600246946BB
:10008000FFF7D3FF18B1FFDF01E0641CE4B268465C
:10009000FFF7A9FF0028F8D02846FFF7E5FF001B6F
:1000A000C0B23EBD57498978814201D9C0B270477C
:1000B000FF2070472DE9F04106291BD1514C002744
:1000C0003B464FF6FF7604EB810514F801C00AE0C9
:1000D000DC19D5F824E0A4B25EF824E0BEF1000FEC
:1000E00004D05B1C9BB29C45F2D834460480204669
:1000F000B44201D100202EE7BDE8F04100E7A0F5B1
:100100007F43FF3B01D0072901D300207047F7E66A
:10011000A0F57F42FF3A0BD0072909D2394A9378DC
:10012000834205D902EB8101496A51F820007047EA
:10013000002070472DE9F04104460D46A4F57F41AB
:1001400043F20200FF3902D0072D01D3072002E756
:100150002C494FF000088A78A242F8D901EB8506B5
:10016000726A52F82470002FF1D0274839461C30AB
:1001700050F8252020469047716A284641F824808F
:1001800000F007F802463946B068FFF739FE002054
:10019000E1E61D49383131F810004FF6FC71C01C02
:1001A000084070472DE9F843164E8846054600245E
:1001B0002868C01C20F0030028602046FFF7E9FFF4
:1001C000315D4843B8F1000F01D0002200E02A68F9
:1001D0000146009232B100274FEA0D00FFF7C7FD3C
:1001E0001FB106E001270020F8E706EB8401009A22
:1001F0008A602968641C0844E4B22860072CD7D3BD
:10020000EFE60000A806002084B2010070B50E469B
:100210001D46114600F0D5F804462946304600F048
:10022000D9F82044001D70BD2DE9F04190460D46DF
:1002300004004FF0000610D00027E01C20F003005F
:10024000A04200D0FFDFE5B141460020FFF78FFD5F
:100250000C3000EB850617B113E00127EDE7624F84
:1002600004F10C00AA003C602572606000EB850080
:10027000206000216068FDF7A8F841463868FFF764
:1002800076FD3046BDE8F0812DE9FF4F564C8046A3
:1002900081B020689A46934600B9FFDF2068027A51
:1002A000424503D9416851F8280020B143F20200C9
:1002B00005B0BDE8F08F5146029800F082F886B292
:1002C00058460E9900F086F885B27019001D87B265
:1002D0002068A14639460068FFF767FD04001FD07B
:1002E000678025802946201D0E9D07465A4601231A
:1002F0000095FFF777F92088314638440123029AA8
:10030000CDF800A0FFF76EF92088C1193846FFF735
:100310009AF9D9F800004168002041F82840C7E761
:100320000420C5E770B5304C0546206800B9FFDFF2
:100330002068017AA9420ED9426852F8251051B1BD
:10034000002342F825304A880068FFF759FD2168EC
:1003500000200A7A08E043F2020070BD4B6853F8AF
:10036000203033B9401CC0B28242F7D80868FFF78A
:1003700011FD002070BD70B51B4E0546002430688D
:1003800000B9FFDF3068017AA94204D9406850F80B
:10039000250000B1041D204670BD70B5124E054603
:1003A0000024306800B9FFDF3068017AA94206D91D
:1003B000406850F8251011B131F8040B441820465C
:1003C00070BD10B50A460121FFF705F9C01C20F0E9
:1003D000030010BD10B50A460121FFF7FCF8C01C50
:1003E00020F0030010BD00008000002070B504461E
:1003F000C2F110052819FCF7BEFF15F0FF0109D066
:10040000491ECAB28020A0542046BDE87040002199
:10041000FCF7DBBF70BD30B505E05B1EDBB2CC5C2A
:10042000D55C6C40C454002BF7D130BD10B500240E
:1004300009E00B78521E44EA430300F8013B11F82F
:10044000013BD2B2DC09002AF3D110BD2DE9F04303
:1004500089B01E46DDE9107990460D00044622D091
:1004600002460846F949FEF719FB10222146384694
:10047000FFF7DCFFE07B000606D5F44A394610237F
:1004800010320846FFF7C7FF102239464846FFF7EB
:10049000CDFFF87B000606D5EC4A49461023103202
:1004A0000846FFF7B8FF102200212046FCF78DFF19
:1004B0000DE0103EB6B208EB060110232246684656
:1004C000FFF7A9FF224628466946FEF7E7FA102EF5
:1004D000EFD818D0F2B241466846FFF787FF1023E5
:1004E0004A46694604A8FFF796FF1023224604A94E
:1004F0006846FFF790FF224628466946FEF7CEFA87
:1005000009B0BDE8F08310233A464146EAE770B5EA
:100510009CB01E460546134620980C468DF80800F0
:10052000202219460DF10900FCF725FF2022214663
:100530000DF12900FCF71FFF17A913A8CDE9000151
:10054000412302AA31462846FFF780FF1CB070BD48
:100550002DE9FF4F9FB014AEDDE92D5410AFBB491C
:10056000CDE90076202320311AA8FFF76FFF4FF066
:1005700000088DF808804FF001098DF8099054F8B3
:10058000010FCDF80A00A088ADF80E0014F8010C98
:100590001022C0F340008DF8100055F8010FCDF87F
:1005A0001100A888ADF8150015F8010C2C99C0F3BE
:1005B00040008DF8170006A88246FCF7DCFE0AA86A
:1005C000834610222299FCF7D6FEA048352308382E
:1005D00002AA40688DF83C80CDE900760E901AA9F9
:1005E0001F98FFF733FF8DF808808DF80990206879
:1005F000CDF80A00A088ADF80E0014F8010C102206
:10060000C0F340008DF810002868CDF81100A888CC
:10061000ADF8150015F8010C2C99C0F340008DF8C9
:1006200017005046FCF7A7FE584610222299FCF707
:10063000A2FE86483523083802AA40688DF83C900F
:10064000CDE900760E901AA92098FFF7FFFE23B09F
:10065000BDE8F08FF0B59BB00C460546DDE92210F1
:100660001E461746DDE92032D0F801C0CDF808C09B
:10067000B0F805C0ADF80CC00078C0F340008DF8AC
:100680000E00D1F80100CDF80F00B1F80500ADF86B
:10069000130008781946C0F340008DF81500108843
:1006A000ADF8160090788DF818000DF119001022A1
:1006B000FCF761FE0DF1290010223146FCF75BFECC
:1006C0000DF1390010223946FCF755FE17A913A881
:1006D000CDE90001412302AA21462846FFF7B6FED4
:1006E0001BB0F0BDF0B5A3B017460D4604461E463C
:1006F000102202A82899FCF73EFE06A820223946BF
:10070000FCF739FE0EA820222946FCF734FE1EA96C
:100710001AA8CDE90001502302AA314616A8FFF716
:1007200095FE1698206023B0F0BDF0B589B0044660
:10073000DDE90E070D463978109EC1F340018DF8B2
:10074000001031789446C1F340018DF8011019680A
:10075000CDF802109988ADF8061099798DF8081037
:100760000168CDF809108188ADF80D1080798DF8F9
:100770000F0010236A46614604A8FFF74CFE22468C
:10078000284604A9FEF78AF9D6F801000090B6F8C9
:100790000500ADF80400D7F80100CDF80600B7F861
:1007A0000500ADF80A000020039010236A46214698
:1007B00004A8FFF730FE2246284604A9FEF76EF98A
:1007C00009B0F0BD1FB51C6800945B680193136805
:1007D000029352680392024608466946FEF75EF9A4
:1007E0001FBD10B588B0044610680490506805908D
:1007F00000200690079008466A4604A9FEF74EF9C5
:10080000BDF80000208008B010BD1FB51288ADF8FB
:1008100000201A88ADF80220002201920292039271
:10082000024608466946FEF739F91FBD7FB5074BFA
:1008300014460546083B9A1C6846FFF7E6FF224629
:1008400069462846FFF7CDFF7FBD0000D2B2010008
:1008500070B5044600780E46012813D0052802D052
:10086000092813D10EE0A06861690578042003F01F
:1008700081FA052D0AD0782300220420616903F053
:10088000CFF903E00420616903F074FA3146204691
:10089000BDE8704001F08AB810B500F12D03C279AF
:1008A0009C78411D144064F30102C271D2070DD03F
:1008B0004A795C7922404A710A791B791A400A7197
:1008C0008278C9788A4200D9817010BD00224A71AD
:1008D000F5E74178012900D00C21017070472DE91E
:1008E000F04F93B04FF0000B0C690D468DF820B01F
:1008F000097801260C2017464FF00D084FF0110A19
:100900004FF008091B2975D2DFE811F01B00C40263
:1009100007031F035E037103A303B803F9031A045B
:1009200062049504A204EF042D0537055505600502
:10093000F3053606390668068406FE062207EB062E
:10094000F00614B120781D282AD0D5F808805FEA77
:1009500008004FD001208DF82000686A02220D9017
:100960008DF824200A208DF82500A8690A90A8880F
:100970000028EED098F8001091B10F2910D27DD246
:10098000DFE801F07C1349DEFCFBFAF9F8F73808E0
:100990009CF6F50002282DD124B120780C2801D036
:1009A0000026F0E38DF82020CBE10420696A03F0F3
:1009B000E1F9A8880728EED1204600F0F2FF0228CE
:1009C00009D0204600F0EDFF032807D9204600F0AB
:1009D000E8FF072802D20120207004E0002CB8D0E4
:1009E00020780128D7D198F80400C11F0A2902D322
:1009F0000A2061E0C4E1A070D8F80010E162B8F804
:100A00000410218698F8060084F83200012028702E
:100A10000320207044E00728BDD1002C99D0207815
:100A20000D28B8D198F8031094F82F20C1F3C00016
:100A3000C2F3C002104201D0062000E0072089075F
:100A400007D198F805100142D2D198F8061001425A
:100A5000CED194F8312098F8051020EA0202114214
:100A6000C6D194F8322098F8061090430142BFD1C5
:100A700098F80400C11F0A29BAD200E008E2617D9B
:100A800081427CD8D8F800106160B8F80410218148
:100A900098F80600A072012028700E202070032014
:100AA0008DF82000686A0D9004F12D000990601DFA
:100AB0000A900F300B9022E12875FCE3412891D178
:100AC000204600F06EFF042802D1E078C00704D170
:100AD000204600F066FF0F2884D1A88CD5F80C8042
:100AE00080B24FF0400BE669FFF745FC32464146C5
:100AF0005B464E46CDF80090FFF741F80B208DF88D
:100B00002000686A0D90E0690990002108A8FFF7AD
:100B10009FFE2078042806D0A07D58B1012809D076
:100B200003280AD04AE305202070032028708DF89E
:100B30002060CEE184F800A032E712202070EAE1C4
:100B40001128BCD1204600F02CFF042802D1E07807
:100B5000C00719D0204600F024FF062805D1E07810
:100B6000C00711D1A07D02280ED0204608E0CCE0BD
:100B700084E072E151E124E103E1E9E019E0B0E150
:100B800000F00FFF11289AD1102208F1010104F1A1
:100B90003C00FCF7F0FB607801286ED0122020703A
:100BA000E078C00760D0A07D0028C8D00128C6D05A
:100BB0005AE0112890D1204600F0F3FE082804D016
:100BC000204600F0EEFE132886D104F16C001022BE
:100BD00008F101010646FCF7CEFB207808280DD06D
:100BE00014202070E178C8070DD0A07D02280AD01B
:100BF0006278022A04D00328A1D035E00920F0E76A
:100C000008B1012837D1C80713D0A07D02281DD014
:100C100000200090D4E9062133460EA8FFF777FCA8
:100C200010220EA904F13C00FCF778FBC8B10420A7
:100C300042E7D4E90912201D8DE8070004F12C03D6
:100C400032460EA8616BFFF770FDE9E7606BC1F3F8
:100C50004401491E0068C84000F0010040F08000D7
:100C6000D7E72078092806D185F800908DF82090E4
:100C700036E32870EFE30920FBE79EE1112899D1C4
:100C8000204600F08EFE0A2802D1E078C00704D189
:100C9000204600F086FE15288CD104F13C0010227D
:100CA00008F101010646FCF766FB20780A2816D0F9
:100CB00016202070D4E90932606B611D8DE80F00A9
:100CC00004F15C0304F16C0247310EA8FFF7C2FC8B
:100CD00010220EA93046FCF721FB18B1F9E20B20D7
:100CE000207073E22046FFF7D7FDA078216AC0F19B
:100CF00010020B1800211846FCF767FB26E3394663
:100D000008A8FFF7A5FD06463CE20228B7D1204619
:100D100000F047FE042804D3204600F042FE0828D5
:100D200009D3204600F03DFE0E2829D3204600F0CE
:100D300038FE122824D2A07D0228A0D10E208DF8E2
:100D40002000686A0D9098F801008DF82400F5E302
:100D5000022894D1204600F024FE002810D020461E
:100D600000F01FFE0128F9D0204600F01AFE0C28E2
:100D7000F4D004208DF8240098F801008DF82500A7
:100D800060E21128FCD1002CFAD020781728F7D186
:100D90006178606A022912D05FF0000101EB410125
:100DA000182606EBC1011022405808F10101FCF79A
:100DB000E2FA0420696A00F0E7FD2670F0E50121FF
:100DC000ECE70B28DCD1002CDAD020781828D7D11A
:100DD0006078616A02281CD05FF0000000EB4002DE
:100DE000102000EBC2000958B8F8010008806078B4
:100DF000616A02280FD0002000EB4002142000EBB3
:100E0000C2000958404650F8032F0A604068486005
:100E100039E00120E2E70120EEE71128B0D1002CF3
:100E2000AED020781928ABD16178606A022912D03F
:100E30005FF0000101EB41011C2202EBC101102215
:100E4000405808F10101FCF796FA0420696A00F0A5
:100E50009BFD1A20B6E00121ECE7082890D1002C78
:100E60008ED020781A288BD1606A98F801200178FA
:100E700062F347010170616AD8F8022041F8012F3E
:100E8000B8F8060088800420696A00F07DFD90E2D1
:100E9000072011E63878012894D1182204F11400B3
:100EA0007968FCF768FAE079C10894F82F0001EA44
:100EB000D001E07861F30000E070217D002974D159
:100EC0002178032909D0C00725D0032028708DF888
:100ED0002090686A0D90412008E3607DA1788842E7
:100EE00001D90620E8E502262671E179204621F0A5
:100EF000E001E171617A21F0F0016172A17A21F0E3
:100F0000F001A172FFF7C8FC2E708DF82090686A7E
:100F10000D900720EAE20420ABE6387805289DD141
:100F20008DF82000686A0D90B8680A900720ADF827
:100F300024000A988DF830B06168016021898180B1
:100F4000A17A817104202070F8E23978052985D1D1
:100F50008DF82010696A0D91391D09AE0EC986E819
:100F60000E004121ADF824108DF830B01070A88C1F
:100F7000D7F80C8080B24026A769FFF70EFA4146E9
:100F80003A463346C846CDF80090FEF72CFE0021C5
:100F900008A8FFF75DFCE07820F03E00801CE070C0
:100FA0002078052802D00F200CE04AE1A07D20B176
:100FB000012802D0032802D002E10720BEE584F810
:100FC0000080EDE42070EBE4102104F15C0002F0FD
:100FD000EAFB606BB0BBA07D18B1012801D00520F1
:100FE000FDE006202870F8486063A063C2E238780C
:100FF000022894D1387908B12875B7E3A07D02287A
:1010000002D0032805D022E0B8680028F5D060633C
:101010001CE06078012806D0A07994F82E100128F1
:1010200005D0E94806E0A17994F82E00F7E7B86802
:101030000028E2D06063E078C00701D0012902D027
:10104000E14803E003E0F8680028D6D0A06306205A
:101050000FE68DF82090696A0D91E1784846C9073E
:1010600009D06178022903D1A17D29B1012903D0DA
:10107000A17D032900D00720287033E138780528A6
:10108000BBD1207807281ED084F800A005208DF859
:101090002000686A0D90B8680A90ADF824A08DF819
:1010A00030B003210170E178CA070FD0A27D022A77
:1010B0001AD000210091D4E9061204F15C03401C0F
:1010C000FFF725FA6BE384F80090DFE7D4E9092302
:1010D000211D8DE80E0004F12C0304F15C02401C7C
:1010E000616BFFF722FB5AE3626BC1F34401491EB7
:1010F0001268CA4002F0010141F08001DAE7387855
:101100000528BDD18DF82000686A0D90B8680A9056
:10111000ADF824A08DF830B0042100F8011B102296
:1011200004F15C01FCF727F9002108A8FFF790FB08
:101130002078092801D0132044E70A2020709AE57E
:10114000E078C10742D0A17D012902D0022927D031
:1011500038E0617808A8012916D004F16C010091EB
:10116000D4E9061204F15C03001DFFF7BBFA0A2064
:10117000287003268DF82080686A0D90002108A849
:10118000FFF766FBE1E2C7E204F15C010091D4E9FC
:10119000062104F16C03001DFFF7A4FA0026E9E71D
:1011A000C0F3440114290DD24FF0006101EBB010DF
:1011B0004FEAB060E0706078012801D01020BDE4F3
:1011C0000620FFE6607801283FF4B6AC0A2050E51F
:1011D000E178C90708D0A17D012903D10B2028702F
:1011E000042030E028702EE00E2028706078616BBB
:1011F000012818D004F15C0304F16C020EA8FFF77B
:10120000E1FA2046FFF748FBA0780EAEC0F11002CD
:1012100030440021FCF7D9F806208DF82000686AD8
:1012200009960D909BE004F16C0304F15C020EA89A
:10123000FFF7C8FAE8E73978022903D1397900299C
:10124000D0D0297592E28DF82000686A0D9056E59D
:1012500038780728F6D1D4E909216078012808D028
:1012600004F16C00CDE90002029105D104F16C0398
:1012700004E004F15C00F5E704F15C0304F14C00C8
:101280007A680646216AFFF763F96078012822D15F
:10129000A078216AC0F110020B1800211846FCF753
:1012A00094F8D4E90923606B04F12D018DE80F0057
:1012B00004F15C0300E05BE204F16C0231460EA82D
:1012C000FFF7C8F910220EA904F13C00FCF726F83C
:1012D00008B10B20ACE485F8008000BF8DF82090A9
:1012E000686A0D908DF824A009E538780528A9D101
:1012F0008DF82000686A0D90B8680A90ADF824A0B7
:101300008DF830B080F80080617801291AD0D4E9D6
:10131000092104F12D03A66B03910096CDE901325A
:1013200004F16C0304F15C0204F14C01401CFFF772
:1013300091F9002108A8FFF78BFA6078012805D001
:1013400015203FE6D4E90912631DE4E70E2028705A
:1013500006208DF82000686ACDF824B00D90A078A2
:101360008DF82800CBE438780328C0D1E079C00795
:1013700070D00F202870072065E7387804286BD1DB
:101380001422391D04F11400FBF7F5FF616A208C6B
:10139000A1F80900616AA078C871E179626A01F078
:1013A00003011172616A627A0A73616AA07A81F834
:1013B000240016205DE485F800A08DF82090696A6D
:1013C00050460D9192E00000D2B201003878052815
:1013D00042D1B868A8616178606A022901D0012110
:1013E00000E0002101EB4101142606EBC101405849
:1013F000082102F0D8F96178606A022901D0012140
:1014000000E0002101EB410106EBC101425802A8B6
:10141000E169FFF70BFA6078626A022801D00120C7
:1014200000E0002000EB4001102000EBC10002238F
:10143000105802A90932FEF7EEFF626AFD4B0EA8B2
:101440000932A169FFF7E1F96178606A022904D0E5
:10145000012103E044E18DE0BFE0002101EB410107
:10146000182606EBC101A27840580EA9FBF783FFAE
:101470006178606A022901D0012100E0002101EBBE
:10148000410106EBC1014158A0780B18C0F11002D0
:1014900000211846FBF799FF05208DF82000686AA7
:1014A0000D90A8690A90ADF824A08DF830B00621FF
:1014B00001706278616A022A01D0012200E00022F4
:1014C00002EB420206EBC202401C89581022FBF7D5
:1014D00052FF002108A8FFF7BBF91220C5F818B089
:1014E00028708DF82090686A0D900B208DF82400EC
:1014F00005E43878052870D18DF82000686A0D90D1
:10150000B8680A900B20ADF824000A9807210170F2
:101510006178626A022901D0012100E0002101EB1B
:101520004103102101EBC30151580988A0F80110B3
:101530006178626A022902D0012101E02FE10021D5
:1015400001EB4103142101EBC30151580A6840F833
:10155000032F4968416059E01920287001208DF857
:10156000300074E6162028708DF830B0002108A8ED
:10157000FFF76EF9032617E114202870AEE63878DD
:1015800005282AD18DF82000686A0D90B8680A9065
:10159000ADF824A08DF830B080F800906278616AD0
:1015A0004E46022A01D0012200E0002202EB420254
:1015B0001C2303EBC202401C89581022FBF7DBFE00
:1015C000002108A8FFF744F9152028708DF8206045
:1015D000686A0D908DF8246039E680E03878052837
:1015E0007DD18DF82000686A0D90B8680A90ADF83A
:1015F0002490092101706169097849084170616985
:1016000051F8012FC0F802208988C18020781C2859
:10161000A8D1A1E7E078C00702D04FF0060C01E0A6
:101620004FF0070C607802280AD000BF4FF000008E
:1016300000EB040101F1090105D04FF0010004E0C5
:101640004FF00100F4E74FF000000B78204413EA5C
:101650000C030B7010F8092F02EA0C02027004D17F
:101660004FF01B0C84F800C0D2B394F801C0BCF159
:10167000010F00D09BB990F800C0E0465FEACC7C37
:1016800004D028F001060670102606E05FEA887C88
:1016900005D528F00206067013262E70032694F84E
:1016A00001C0BCF1020F00D092B991F800C05FEA0E
:1016B000CC7804D02CF001060E70172106E05FEA0A
:1016C0008C7805D52CF002060E70192121700026A9
:1016D0000078D0BBCAB3C3BB1C20207035E012E039
:1016E00002E03878062841D11A2015E42078012834
:1016F0003CD00C283AD02046FFF7EBF809208DF8B3
:101700002000686A0D9031E03878052805D0062061
:10171000387003261820287046E005208DF8200038
:10172000696A0D91B9680A910221ADF8241001216E
:101730008DF830100A990870287D4870394608A83D
:10174000FFF786F8064618202870012E0ED02BE0F1
:1017500001208DF82000686A0D9003208DF8240088
:10176000287D8DF8250085F814B012E0287D80B121
:101770001D202070172028708DF82090686A0D9029
:1017800002208DF82400394608A8FFF761F80646C4
:101790000AE00CB1FE2020709DF8200020B100214D
:1017A00008A8FFF755F80CE413B03046BDE8F08FF9
:1017B0002DE9F04387B00C464E6900218DF80410E6
:1017C00001202578034602274FF007094FF0050C4A
:1017D00085B1012D53D0022D39D1FE2030708DF806
:1017E0000030606A059003208DF80400207E8DF89B
:1017F000050063E02179012925D002292DD0032994
:1018000028D0042923D1B17D022920D131780D1FA0
:10181000042D04D30A3D032D01D31D2917D121899D
:10182000022914D38DF80470237020899DF80410C8
:10183000884201E0CAB2010018D208208DF80000E9
:10184000606A059057E070780128EBD0052007B05A
:10185000BDE8F0831D203070E4E771780229F5D1EE
:1018600031780C29F3D18DF80490DDE7083402F8C3
:1018700004CB94E80B0082E80B000320E7E715781F
:10188000052DE4D18DF800C0656A0595956802952F
:101890008DF8101094F80480B8F1010F13D0B8F14E
:1018A000020F2DD0B8F1030F1CD0B8F1040FCED128
:1018B000ADF804700E202870207E68700021684604
:1018C000FEF7C6FF0CE0ADF804700B202870207EF8
:1018D000002100F01F0068706846FEF7B9FF3770FE
:1018E0000020B4E7ADF804708DF8103085F800C022
:1018F000207E6870277011466846FEF7A9FFA6E7AC
:10190000ADF804902B70207F6870607F00F00100BC
:10191000A870A07F00F01F00E870E27F2A71C00766
:101920001CD094F8200000F00700687194F82100A2
:1019300000F00700A87100216846FEF789FF2868BB
:10194000F062A8883086A87986F83200A0694078CD
:1019500070752879B0700D203070C1E7A971697178
:10196000E9E700B587B004280CD101208DF800000C
:101970008DF80400002005918DF8050001466846A9
:10198000FEF766FF07B000BD70B50C46054602F0D5
:10199000F1F921462846BDE870407823002202F084
:1019A0003FB908B1007870470C20704770B50C0043
:1019B00005784FF000010CD021702146F1F72DFC85
:1019C00069482178405D884201D1032070BD022022
:1019D00070BDF1F722FC002070BD0279012A05D00C
:1019E00000220A704B78012B02D003E004207047DC
:1019F0000A758A6102799300521C0271C15003205A
:101A00007047F0B587B00F4605460124287905EBED
:101A1000800050F8046C7078411E02290AD25249A5
:101A20003A46083901EB8000314650F8043C28461C
:101A3000984704460CB1012C11D12879401E10F0B2
:101A4000FF00287101D00324E0E70A208DF8000090
:101A5000706A0590002101966846FFF7A7FF032CE6
:101A6000D4D007B02046F0BD70B515460A460446EE
:101A700029461046FFF7C5FF064674B12078FE28B8
:101A80000BD1207C30B100202870294604F10C00D5
:101A9000FFF7B7FF2046FEF71CFF304670BD7047CA
:101AA00070B50E4604467C220021FBF78EFC022511
:101AB000012E03D0022E04D0052070BD01206070DD
:101AC00000E065702046FEF704FFA575002070BD9C
:101AD00028B1027C1AB10A4600F10C01C4E70120CA
:101AE000704710B5044686B0042002F043F9207810
:101AF000FE2806D000208DF8000069462046FFF73A
:101B0000E7FF06B010BD7CB50E4600218DF804102D
:101B10004178012903D0022903D0002405E004699B
:101B200000E044690CB1217C89B16D46014628462C
:101B3000FFF753FF032809D1324629462046FFF715
:101B400093FF9DF80410002900D004207CBD04F10F
:101B50000C05EBE730B40C460146034A204630BC86
:101B6000024B0C3AFEF751BE10B30100CAB201009D
:101B700070B50D46040011D085B122010021284620
:101B8000FBF723FC102250492846FBF7F4FB4F4893
:101B90000121017044704560002070BD012070BDBE
:101BA00070B505460024494E11E07068AA7B00EB31
:101BB0000410817B914208D1C17BEA7B914204D120
:101BC0000C222946FBF7AAFB30B1641CE4B2307842
:101BD0008442EAD3002070BD641CE0B270BD70B5D1
:101BE0000546FFF7DDFF002805D1384C20786178E5
:101BF000884201D3002070BD6168102201EB001003
:101C00002946FBF7B8FB2078401CC0B2207070BD9D
:101C10002E48007870472D490878012802D0401ED0
:101C200008700020704770B50D4600219170144671
:101C30001180022802D0102815D105E0288890B123
:101C40000121A17010800CE0284613B1FFF7C7FFF7
:101C500001E0FFF7A5FFA07010F0FF0F03D0A889E7
:101C60002080002070BD012070BD0023DBE770B52F
:101C7000054614460E0009D000203070A8780128CF
:101C800006D003D911490A7890420AD9012070BDC3
:101C900024B1287820702888000A5070022008702B
:101CA0000FE064B14968102201EB001120461039A1
:101CB000FBF761FB287820732888000A60731020E6
:101CC0003070002070BD00001FB3010084000020B0
:101CD0002DE9F04190460C4607460025C2EB48111D
:101CE000FE48072F00EB410607D2DFE807F00707A1
:101CF000070704040400012500E0FFDF06F8147064
:101D0000002D13D0F5487C3000EB880191F82700B6
:101D10001F2803D006EB4000447001E081F8264004
:101D200006EB44021F20507081F82740BDE8F08187
:101D3000F0B51F4614460E4605461F2A00D1FFDFA8
:101D4000E648C7EB471100EB410CE4490CEB4400BB
:101D50007C3101EB87021F2E07D00CEB4601407847
:101D60004B78487018461F210AE092F825304078D9
:101D700082F82500F6E701460CEB4100057040783B
:101D8000A142F8D192F827401F2C03D00CEB440459
:101D9000637001E082F826300CEB41041F2363706E
:101DA00082F82710F0BD30B50D46CD4B4419002206
:101DB000181A72EB020100D2FFDFCA48854200DD2B
:101DC000FFDFC8484042854200DAFFDFC448401CBC
:101DD000844207DA002C01DB204630BDC048401C9D
:101DE000201830BDBE48C043FAE710B5044601686C
:101DF000407ABD4A52F82020114450B102200844D4
:101E000020F07F40F8F753FD94F90810BDE810402A
:101E1000C9E70420F3E72DE9F047B04E7C3696F889
:101E20002D50DFF8B89206EB850090F8264036E09A
:101E3000C5EB451109EB41074FF0070817F81400EF
:101E4000012806D004282ED005282ED0062800D040
:101E5000FFDF01F045F9014607EB4400427806EB4D
:101E6000850080F8262090F82720A24202D11F2268
:101E700080F82720084601F03EF92A462146012035
:101E8000FFF726FF9948414600EB04100268204600
:101E9000904796F82D5006EB850090F826401F2CB1
:101EA000C6D1BDE8F087022000E003208046D0E7DD
:101EB00010B58A4C1F217C3484F8251084F8261034
:101EC00084F82710002084F8280084F82D0084F876
:101ED0002E10411EA16044F8100B20746074207312
:101EE0006073A0738249E077207508704870002104
:101EF0007A4A103C02F81100491CC9B21F29F9D3D3
:101F00000120F8F7C4FB0020F8F7C1FB012084F89A
:101F10002200F9F731F87748F9F743F8744CA41E1A
:101F200020707548F9F73DF86070BDE81040F8F78B
:101F30003BBB10B5F8F75DFB6D4CA41E2078F9F79C
:101F400049F86078F9F746F8BDE8104001F000B9AB
:101F50001F2070470020F8F773BB70B505460124B9
:101F60000E46AC405AB1FFF7F5FF0146634800EB5F
:101F7000C500C0F81015C0F81465614801E060485C
:101F8000001D046070BD2DE9F34F544D00247C35D5
:101F900005EB810A89B09AF825001F2823D0611E1D
:101FA00002915249009401EB0017391D03AB07C998
:101FB00083E8070005F11400A0460189ADF81C1064
:101FC000807A8DF81E009DF81500C8B1022646499A
:101FD00051F820400399A219114421F07F41019149
:101FE00084B102210FE00120F8F751FB0020F8F73F
:101FF0004EFBF8F71CFB01F0ABF885F82F40A9E089
:102000000426E4E700218DF81810022801D00128E9
:1020100020D1039801190998081A801C9DF81C10FA
:1020200020F07F4001B10221353181420BD20320E3
:102030008DF815000398C4F13201401A20F07F405A
:10204000322403900CE095F8240018B901F063FAEB
:10205000002863D0322C03D214B101F06DF801E0F6
:1020600001F076F8224A107818B393465278039B11
:10207000121B00219DF81840994601281AD0032808
:1020800018D000208DF81E00002A04DD981A039055
:1020900001208DF818009DF81C0000B10221039862
:1020A000184A20F07F40039003AB099801F05CF8D8
:1020B00010B110E00120E5E79DF81D0018B99BF86C
:1020C0000000032829D08DF81C80CDF80C908DF8E5
:1020D00018408DF81E809DF8180015E0D8080020E3
:1020E000FF7F841E0020A10730B30100E806002016
:1020F0008E000020CF3A0100171E010000F00140C1
